:1000000000800020BD010000A9D7000061D70000DA
:1000100061D7000061D7000061D7000061D7000000
:1000200061D7000061D7000061D70000A9D70000A8
:10003000A9D7000061D7000029CE00002DCF000015
:10004000A9D70000A9D70000A9D70000A9D70000B0
:10005000A9D70000A9D70000A9D70000A9D70000A0
:10006000A9D70000A9D70000A9D70000A9D7000090
:10007000A9D70000A9D70000A9D70000A9D7000080
:10008000A9D70000A9D70000A9D70000A9D7000070
:10009000A9D70000A9D70000A9D70000A9D7000060
:1000A00065B3000071B30000A9D70000A9D7000014
:1000B000A9D70000A9D70000A9D70000A9D7000040
:1000C000A9D70000A9D70000A9D70000A9D7000030
:1000D000A9D70000A9D70000A9D70000A9D7000020
:1000E000A9D70000A9D70000A9D70000A9D7000010
:1000F000A9D70000C5FB0000A9D7000095E20000C9
:10010000A9D7000031E50000A9D70000A9D7000059
:10011000A9D70000A9D70000A9D70000A9D70000DF
:10012000A9D70000A9D70000A9D70000A9D70000CF
:10013000A9D70000A9D70000A9D70000A9D70000BF
:10014000A9D70000A9D70000A9D70000A9D70000AF
:1001500019D000002DD0000041D0000055D0000083
:10016000A9D700004DE80000A9D70000A9D70000DA
:10017000A9D70000A9D70000A9D70000A9D700007F
:10018000A9D70000A9D70000A9D70000A9D700006F
:10019000A9D70000A9D70000A9D70000A9D700005F
:1001A000A9D70000A9D70000A9D70000A9D700004F
:1001B000A9D70000A9D70000A9D70000564B4CF2E0
:1001C000205210B51A804DF628121A8000BF00BFC9
:1001D0000DF0EEFA514B4FF010621A60504A9A60DF
:1001E000504ADA60504A136813F4807304D14F49BF
:1001F0000B604FF4A85313604D4B1A78110703D5C9
:100200001A7842F008021A704A4B4B492A221A7097
:100210004A4A4B4B8B4204D252F8040F43F8040B6A
:10022000F8E7484B484900228B4202D243F8042B9E
:10023000FAE74649464A002352F8230041F82300D2
:1002400001336F2BF8D1434B434A802103F8011B44
:100250009342FBD1414B3D4A1A60414B8A221A70AE
:10026000A3F5805324225A70A0221A709A7992071B
:10027000FCD59A79D406FCD43A4A937903F00C035E
:10028000082B384BF9D103221A7140225A719A79FE
:100290009006FCD5334A9179324B4906FBD5324A58
:1002A000324911600221516020221A709A7902F0BD
:1002B0000C020C2AFAD12E4B2E4A1A602E4B2F4AD2
:1002C0001A6000225A60072243F8042C2C4AC3F813
:1002D0000C2D62B60DF01CFE144B1B68DA0705D519
:1002E00028480DF0E9FB284B284A1A60284B1B7858
:1002F0005B0609D5244C254B22689A4204D121483B
:100300000DF0DAFB0023236010F016FF0DF056FA13
:100310000DF084F9FEE700BF0E2005403080044058
:10032000823F04000100002B10D0034014D0034092
:1003300002D0074000E00740549CFF1F244D0100FD
:100340004088FF1F549CFF1F7CA4FF1F0082FF1FDB
:100350000000000000E400E05FE400E008ED00E0E1
:100360000050064000400640448004400000030165
:1003700004800440C010050014E000E0FF76010096
:10038000000020201D2631601CE00340A5C3945AC4
:1003900000F00740FFFFFFFFFFFFFFFFFFFFFFFF32
:1003A000FFFFFFFFFFFFFFFFFFFFFFFFFFFFFFFF5D
:1003B000FFFFFFFFFFFFFFFFFFFFFFFFFFFFFFFF4D
:1003C000FFFFFFFFFFFFFFFFFFFFFFFFFFFFFFFF3D
:1003D000FFFFFFFFFFFFFFFFFFFFFFFFFFFFFFFF2D
:1003E000FFFFFFFFFFFFFFFFFFFFFFFFFFFFFFFF1D
:1003F000FFFFFFFFFFFFFFFFFFFFFFFFFFFFFFFF0D
:10040000FFFFFFFFFFFFFFFFFFFFFFFFDEF9FFFF23
:1004100010B5054C237833B9044B13B10448AFF33E
:1004200000800123237010BD549CFF1F00000000BA
:10043000284D0100084B10B51BB108490848AFF31F
:1004400000800848036803B910BD074B002BFBD0A0
:10045000BDE81040184700BF00000000589CFF1F77
:10046000284D0100549CFF1F0000000038B50446D1
:10047000104621700A491D4610F040FC01464FF01D
:100480007E5010F0EFFC074910F038FCE56060602A
:10049000256165610DF0CCFCE061204638BD00BFF0
:1004A000DB0FC9400024744938B50446104621705A
:1004B00009491D4610F022FC01464FF07E5010F015
:1004C000D1FC064910F01AFCE560606025616561A9
:1004D0000DF0AEFCE06138BDDB0FC940002474496B
:1004E00038B503780446032B20D8DFE803F01A1848
:1004F0001002C168406910F0F7FA0D4905466068BE
:1005000010F0B0FC0146284610F0ACFC38BD08499C
:10051000406810F0A7FCE16810F0F0FB38BDC0683F
:1005200038BDC168406910F0DFFA38BD002038BD21
:100530000024744970B504460E460DF079FC05465A
:10054000E069281A10F086FBE3682361E5616661C3
:10055000A0610146606810F085FC0146A06010486B
:1005600010F080FC0FF056FF0FF0F6FB10F068FA69
:10057000054601464FF07E5010F0B6FA616910F062
:10058000BDFB21690646284610F0B8FB01463046FF
:1005900010F0ACFAE0602046BDE87040FFF7A0BF65
:1005A000000080BF08B50E200CF012FF114B1B8815
:1005B000012B19D0104B1B88984213DB40F6FF71BA
:1005C0008842D4BFC3EB0001C3EB0101C1EB013191
:1005D000C3F57F630F33282091FBF3F1BDE808409A
:1005E0000DF07CBA0021F3E70146BDE80840142075
:1005F0000DF074BAB09EFF1F449DFF1F10B5044656
:100600000CF0E8FC204610BD70B44C88A04220D904
:1006100001230133DBB21CB2660031F8144084427E
:100620001D46F6D3A04211D005F10045013D965B71
:1006300031F8151032F81530401AF21A00FB02F0AA
:10064000641A90FBF4F4E01870BC7047905B70BCC7
:10065000704702260125E5E700280CDA064A4342E6
:1006600082FB0320DA17C2EB600000EB4000A3EB33
:100670008000C0F10C007047ABAAAA2A38B5234B02
:100680001B78002B2CD015200CF0A2FE204B1860FC
:10069000204B1B88984203DA1F4C237863BB38BD7C
:1006A0001E4A1488A042A4EB0302A8BF20467F2A5A
:1006B0001CDDC01AC001541C90FBF4F4002CEBD0DC
:1006C000154B1A780AB901221A70154D2B689C42F5
:1006D00004D0144BE1B2187808F0EEFE2C6038BD5F
:1006E00011200DF091FF0A4B1860D1E7C01AC0EB42
:1006F000C01090FBF2F4E1E70A4B0021187808F0F3
:10070000DBFE0023064A2370136038BDC29EFF1F24
:10071000809CFF1FFE9CFF1F389FFF1FDC9EFF1F5A
:10072000349FFF1FD49CFF1F38B50F200DF06CFFC6
:100730001B4A1C4B12881860C0F53B600830904281
:1007400020DB194B1B889842A3EB0204A8BF184674
:10075000801A7F2CC6BFC0010134C0EBC01090FBD3
:10076000F4F47CB1114B1A780AB901221A70104DB9
:100770002B689C4204D00F4BE1B2187808F09CFE25
:100780002C6038BD094C237803B938BD094B0021D2
:10079000187808F091FE0023054A2370136038BDD5
:1007A000489DFF1F989CFF1FC89EFF1FEC9EFF1FC8
:1007B000089DFF1FF69CFF1FF0B40E8886420DD2E5
:1007C00003F10043013B31F81350854202D9F0BCDC
:1007D000FFF71ABF32F81300F0BC70471088F0BC66
:1007E000704700BF094B1B880C2B09D8084A80B200
:1007F00052F8232028B143F6FE73984203D9108C97
:100800007047108870470349FFF7FEBEAE9CFF1F7C
:1008100040270100DC2801004B4B4C4A2DE9F047F2
:100820001E8814684A4BB442B3F80080494B33DB4E
:100830004445A8BF4446A6421C60C8BF00202DDD29
:10084000C6EB0807B7F5804F33DB80037B1C90FBBA
:10085000F3F0FFF7C7FF404A404B15881B88C0F3F1
:10086000C61909FB05F57F2D8246A8BF7F252BB34E
:10087000A64253DC4445D4BFC6EB0404C6EB0804CF
:100880009F42CCBF03FB04445C43354BC8BF0137D8
:1008900094FBF7F71F6013E034461E60C6EB0807B1
:1008A000A045D4BFC6EB0800C6EB0400B7F5804FE7
:1008B000CBDAC0EB803090FBF7F0CAE7284A136030
:1008C000284C2368994508D0274B1B88002B34D12E
:1008D000264B1B886BBBC4F80090254C23689A45B7
:1008E00006D0214B1B885A1F032A19D9C4F800A02F
:1008F000204C23689D420FD01F4B188848B11A4BDB
:100900001E4A1B88D35C834203D0C0B2E9B208F010
:10091000D3FD2560BDE8F087BDE8F0870024AFE790
:10092000164AD05C2030C0B20AF07F0108F0C4FD46
:10093000DCE7484608F060FECDE7104A4946D05C47
:1009400008F0BAFDC4E700BF449DFF1FAC9EFF1F27
:100950000E9FFF1F789CFF1F889CFF1F8A9CFF1F14
:10096000149FFF1FF09CFF1F929EFF1F3A9DFF1FC9
:10097000A89CFF1F3C9DFF1FA29EFF1F9C89FF1F7D
:100980002DE9F04F17208BB00DF03EFEDFF870B36D
:10099000DFF870A3CBF8000016200DF035FEBA4B3F
:1009A000CAF800001B880C2B00F05E82B74EB84AD4
:1009B0003188B84B52F8214000221A70B64BB74A22
:1009C0001B88B7491288013B012A31F9133005937E
:1009D00000F0AE81B34B0193B34B0293B34FDFF8FA
:1009E000288300230093B24B1B88012B00F0F48175
:1009F000DFF81893AF4B0393D9F80050AE4B049334
:100A00000023AE4A1288013A032A00F24982DFE845
:100A100012F0A500ED000400C9002846059310F06F
:100A200019F9A74910F06AF9059B0546184610F018
:100A300011F9A44910F062F90146284610F056F861
:100A400010F022FB0546C9F80050386810F002F992
:100A50009B4910F053F98146009810F0FBF8994932
:100A600010F04CF90146484610F040F810F00CFB2D
:100A70003860954A954B17881988954BDBF800200C
:100A80001B88DFF88CE2C7EB050C3D44039FC7F8D9
:100A900000C0471A084404990D6001990F6002993B
:100AA000BEF8007008609A4280F2E7800025C3EB30
:100AB000070E7445DAF8000080F2D380611C98427A
:100AC00005FB01F50EF1010E95FBFEF5C0F25F830B
:100AD0008742A8BF0746FF1A01FB07F494FBFEF408
:100AE0009A4200F3A780984200F3A480794C2068D2
:100AF00010F0B0F8784910F001F978490FF0F6FFDE
:100B000010F0C2FAA0F5FF531C3B082B98BF4FF41E
:100B10000050D8F80030184400282060C0F29F80B0
:100B2000B0F5804F80F2F6806D4B1B781BB1B0F5AD
:100B3000005F40F0F7806B4D2B78002B40F0AB81CD
:100B4000694D20682B68634C984204D080B208F04D
:100B500083FC23682B600BB0BDE8F08F284605931B
:100B600010F078F8614910F0C9F8059B0546184661
:100B700010F070F85E4910F0C1F8014628460FF0F9
:100B8000B5FF10F081FA0546C9F80050386810F03A
:100B900061F8564910F0B2F88146009810F05AF802
:100BA00053495DE72846059310F054F84A4910F080
:100BB000A5F8059B0546184610F04CF84D4910F075
:100BC0009DF8014628460FF091FF10F05DFA0546AA
:100BD000C9F80050386810F03DF83F4910F08EF821
:100BE0008146009810F036F8424939E728460593C7
:100BF00010F030F8404910F081F8059B0546184682
:100C000010F028F83D4910F079F8014628460FF019
:100C10006DFF10F039FA0546C9F80050386810F039
:100C200019F8354910F06AF88146009810F012F86A
:100C3000324915E73388002B3FF458AF2B1B002BAC
:100C4000B8BF5B42092B00F32D81D8F80030214C4E
:100C50004FF40050184400282060BFF661AF002216
:100C60005AE0984205FB04F5B8BF002195FBFEF55C
:100C700080F2848291FBFEF432E7BA42D4BFC3EB28
:100C80000205C3EB070512E7DE9EFF1FE49CFF1F72
:100C90005889FF1F7E9CFF1F2089FF1FB29EFF1FE8
:100CA0006C2B0100D89CFF1F189DFF1F709CFF1F1D
:100CB000409EFF1FD09EFF1F449EFF1F2E89FF1FD7
:100CC000CDCC4C3FCDCC4C3EA889FF1F2C89FF1FBB
:100CD000A89EFF1F9089FF1F9A99193FCDCC4C45C4
:100CE000EA9FFF1F399DFF1F2489FF1F3333733F86
:100CF000CDCC4C3DCDCCCC3E6666663FCDCCCC3D1C
:100D0000E09CFF1FA49CFF1FE89EFF1FCC9EFF1FBF
:100D1000C09CFF1F43F6FF72C04B22601B78002B64
:100D20003FF409AF05F068FCBD4B01221A7007E7DC
:100D3000BC4BBD4A1B88BD491278013B31F91350A9
:100D4000002A40F0C78011200DF05EFC0090B84BE7
:100D50000193D3F80080009B984540F3C080B54BC9
:100D6000B54F1B88B54A012B3B68B2F80090B44AD6
:100D700002922046A3EB050500F0E2800FF06AFF27
:100D8000029A52F829100FF0B9FF014600200FF027
:100D9000ABFE10F079F9009BC8EB05029D42B8BF8D
:100DA0001D469042C8EB050580F2DE8000FB05552C
:100DB000013295FBF2F5A34BDFF8B4820293D8F829
:100DC00000302B4403EBD3735B10C8F800309E4B0C
:100DD0001B88012B7FF40CAE9C4B03931D460F2008
:100DE0000DF012FC2A6804929042034680F2CC80F7
:100DF000904A1288012A00F03F81904A0790128899
:100E00008F4D069220460FF025FF069ADFF8649278
:100E100055F82210D9F800500FF070FF014600205D
:100E20000FF062FE059BEA1A059210F02DF9059A63
:100E3000079B04999A42C1EB020EB8BF1A4670454F
:100E400080F24481521A00FB02220EF1010192FB52
:100E5000F1F2D8F800107E4804900A4402EBD272F6
:100E60005210C8F80020CCE57A4B1B78002B3FF4D9
:100E70009DAD794E794A3188794B52F82100012293
:100E80001A700FF0E7FE4FF07C510FF037FF10F0B3
:100E9000FBF8044692E505F0ABFB00232B704FE610
:100EA0003868E6E505F500500130001B0FF0D2FE72
:100EB0006C496D4C0FF022FF054620680FF0CAFE0A
:100EC0006A490FF01BFF014628460FF00FFE10F095
:100ED000DBF81EE615200CF07BFA009037E7594B43
:100EE0000293D3F80080009B984542DA514B524F51
:100EF0001B88524A012B3B68B2F80090504A03927B
:100F000020461D4400F0E9800FF0A4FE039A52F839
:100F100029100FF0F3FE10F0B7F8009B9D42C8EBCC
:100F20000502A8BF1D46C8EB05059042BABF00FBED
:100F300005550132454395FBF2F5DFF834813EE774
:100F40000FF088FE029A52F829100FF0D7FE10F029
:100F50009BF8009BC8EB05029D42B8BF1D4682422C
:100F6000C8EB05053FF722AF00FB05F595FBF2F551
:100F700021E7DFF8FC80304FD8F8003003EBD37363
:100F80005B10C8F800302EE5314A049212680692D0
:100F9000904237DD274A1288012A00F0BC80274A98
:100FA00009901188264A0891204607920FF052FEB8
:100FB000079A0899DFF8BC9052F82110D9F8005030
:100FC0000FF09CFE059B2B44059310F05DF80599EE
:100FD000099B069A9942C2EB010EA8BF19467045BB
:100FE00080F2BE80891A00FB01110EF1010291FB13
:100FF000F2F2D8F800100A4402EBD2725210C8F88C
:101000000020FEE4D8F80020DFF8689002EBD272EE
:101010005210D9F80050C8F80020F2E4EA9FFF1FF0
:10102000399DFF1FAC89FF1FC29EFF1F942801003E
:10103000D89CFF1F1E9DFF1F709CFF1FC89CFF1F99
:10104000842B0100189DFF1F409EFF1FD09EFF1F95
:10105000449EFF1F909EFF1FE49CFF1F5889FF1FA7
:101060007E9CFF1FCDCCCC3E9089FF1F9A99193FE3
:10107000E89EFF1FCC9EFF1F464A08901188464AF3
:101080000791204606920FF0E5FD069A0799DFF8D2
:101090000C9152F82110D9F800500FF02FFE059B4B
:1010A000E91A05910FF0F0FF0599089B049A9942FF
:1010B000C2EB010EB8BF1946704558DA891A00FB19
:1010C00001110EF1010291FBF2F2C2E60499521AEB
:1010D00000FB02F292FBFEF2BBE60FF0BBFD039AAF
:1010E00052F829100FF00AFE014600200FF0FCFC18
:1010F0000FF0CAFF009A9542C8EB0503A8BF15463A
:10110000C8EB05059842BABF00FB055501334543BE
:1011100095FBF3F511E71F491F4A089020460D88FB
:1011200007920FF097FD079ADFF8709052F825109C
:10113000D9F800500FF0E2FD014600200FF0D4FC7A
:10114000059B2B4405930FF09FFF0599089B069A7A
:101150009942C2EB010EA8BF19467045FFF642AF97
:10116000069A891A00FB01F191FBFEF241E7049A0D
:10117000891A00FB01F191FBFEF26AE6B842D4BF86
:10118000C3EB0001C3EB070104FB01F172E51F464D
:10119000A1E400BFC89CFF1F842B0100CC9EFF1F51
:1011A00008B5244B1B88FBB1234B1B78FBB1234BA9
:1011B0001B78E3B1224B1B78CBB1224B1B78B3B128
:1011C000214B22481A78C2B9214A22490088128844
:1011D00009680244B1EB620F09DD01221A70642034
:1011E000BDE8084005F01CBA174A117801B908BDDE
:1011F0001370BDE8084008F0D3B9154A16490088B5
:10120000128809680244B1EB620FF0DD00221A7007
:1012100008F0C6F9642005F003FA642005F000FA2E
:10122000642005F0FDF94FF41670BDE808400CF09D
:1012300021BE00BF509EFF1F3C9FFF1F089FFF1F46
:10124000099FFF1F0A9FFF1FAC9CFF1FC09CFF1F31
:10125000A89EFF1FE09CFF1FA49CFF1F38B5114CE8
:10126000232025780CF0B4F80F4A42F82500131F0C
:1012700002F1C400002253F8041F83420A44FAD149
:1012800023780A4907480A4C0133DBB2322B81FB31
:10129000025108BF0023D217C2EB21120370226053
:1012A00038BD00BF8C9CFF1F549DFF1F1F85EB5155
:1012B000A49EFF1F2DE9F04FB84CB94D2068B94FDF
:1012C00083B00FF0C7FCB8490FF018FD0646102098
:1012D0000DF09AF90FF0BEFCB4490FF00FFD314646
:1012E0000FF004FC0FF0D0FE2988206088423B8874
:1012F00043DA9E465B1A7F2B4FF0000247DDD20196
:101300005E1C92FBF6F2AA4EDFF8C882B6F800C067
:10131000C8F80020BCF1190F00F0DF80BCF11A0FF3
:1013200000F01881BCF11E0F00F021810126B146AA
:10133000A04A1288002A00F09D808842C0F20881ED
:101340007045D4BFC1EB0000C1EB0E009A42BABF9A
:1013500002FB00000133504390FBF3F3964A136005
:10136000964B1888C0B9964A1288AAB9954B197835
:1013700001B11A7003B0BDE8F08F9842D4BFC1EB41
:101380000002C1EB03029E465B1A7F2BB7DCC2EB67
:10139000C21292FBF3F2B6E72988D4F800E0DFF836
:1013A0000082DFF8F8A171456CDCDFF818C29CF808
:1013B0000020002A2ED14FF0010B04288CF800B039
:1013C00028D1002E40F095817D4B18880028D1D07F
:1013D000B9F1000FCED023682C883A88A34280F25E
:1013E00066810023141B7E2C774DD5BFC3EB83137E
:1013F000C3EBC3135B00013493FBF4F42B6801349B
:10140000A34203D0C0B2E1B208F056F82C6003B09A
:10141000BDE8F08F012800F0F780022800F0EC8092
:101420000328D1D1694B1B88092BCDD0002ECBD0FE
:1014300023682E883A88B34280F27C810023961B71
:101440007E2EDFF88CA1D5BFC3EB8313C3EBC31390
:101450005B00013693FBF6F6DAF800300136B34252
:1014600003D0F1B24A2008F027F8CAF80060ABE7D1
:1014700091460126BCF11E0F7FF472AF0022DFF807
:1014800058817FE04F4B1A78002A3FF473AF002455
:1014900001281C7000F0A480022840F00F81002E6B
:1014A00000F0A3804A4D2B68002B00F09E800420A2
:1014B000214608F001F8424B2C60188800283FF4C0
:1014C00059AFB9F1000F3FF455AFC0B2002107F09A
:1014D000F3FF3D4B00221A604CE7DFF8FC8098F8E0
:1014E0000020C2B1DFF8D890B9F800A0BAF1000F1F
:1014F00011D0DFF8E89099F800B0934578D05FFA02
:101500008AF07F2107F0D8FF98F80030B6F800C0C5
:1015100089F8003010E0DFF8C49099F800A09245F7
:1015200066D0274B0021187807F0C6FF98F80030E6
:10153000B6F800C089F800301E4B1A88002A97D0F0
:10154000BCF11E0F40F0078101264FF0000919E0A1
:101550000020FBE6DFF8808098F80020002A0BBF0F
:10156000012600264FF000094FF00109E0E6DFF800
:101570006880104B98F800601A88B6FA86F67609EB
:101580004FF0000998F80030002B3FF4E7AE2988AF
:10159000B7F800E02068C1EB0E03CEE6D09CFF1F39
:1015A000569EFF1F529EFF1F9A99193FCDCCCC3EED
:1015B000DE9EFF1F189FFF1F4C9DFF1FDE9CFF1F1D
:1015C000F09EFF1FE59EFF1FB49CFF1F929EFF1F12
:1015D000509DFF1FC49EFF1F909EFF1F929CFF1FE8
:1015E0001EB1624D2B68002B7CD1614B188865E7DA
:1015F00001264FF000099BE6002E3FF4E5AEDFF830
:101600006CA1DAF800202EE0002E3FF4DDAEB7F832
:101610000080F045D4BFC1EB0802C1EB0E02C1EB64
:101620000808B8F17E0FDFF844A1D5BFC2EB8212E3
:10163000C2EBC212520008F1010892FBF8F8DAF886
:10164000002008F10108424506D05FFA88F1012028
:10165000009307F031FF009B1888CAF80080022829
:101660007FF4DEAE42462168B5F8008038884145F7
:1016700059DA0021C8EB0008B8F17E0FD3BFC1EBE7
:101680008111C1EBC11108F10108490091FBF8F883
:1016900008F10108904506D05FFA88F10420009314
:1016A00007F00AFF009B1888CAF80080B8E693424A
:1016B000D4BFC4EB0303C4EB020393E6032827D192
:1016C0002C4B1B88092B90D0002E8ED0274D2B68D9
:1016D000002B8AD04A20214607F0EEFE244B2C60D6
:1016E0001888EBE6214607F0E7FE214B2C601888AE
:1016F000E4E640207F218DE80C0007F0DDFE019B31
:10170000009A188858451CD002287FF489AE76E7E5
:1017100004287FF46AAF002E3FF467AF21464020D3
:1017200007F0CAFE61E78142D4BFC8EB0101C8EBF4
:1017300000019FE79342D4BFC6EB0303C6EB02034D
:101740007DE6B8F80010DAF800E0B7F800808E45C2
:10175000FFF665AF5DE72988B7F800E02068C1EBC8
:101760000E0301264FF00009E7E500BF509DFF1F63
:10177000F09EFF1F929EFF1F08B5114B1B88022B86
:1017800009D0052B07D0032B15D0042B0BD00D4B04
:1017900001221A7008BD7F21412007F08DFE094B00
:1017A00001221A7008BD7F21092007F085FE054B34
:1017B00001221A7008BD4021092007F07DFEE6E7EE
:1017C0004A9DFF1F009DFF1F38B5074B074D1B8823
:1017D000052B044606D02B68834203D0C1B20520F6
:1017E00007F06AFE2C6038BD4A9DFF1FF49EFF1F64
:1017F00038B5124D124C2B88052B12D022684AB9ED
:10180000022B0ED0033B012B13D90E4A0023137079
:10181000236038BD0021052007F04EFE2B88022BE7
:1018200004D10021412007F047FEEEE7052BE9D166
:10183000F7E70021092007F03FFEE6E74A9DFF1F7A
:10184000F49EFF1F009DFF1F464B1B881D2B70B58C
:1018500041D0454D0024454B1B88022B16D0444BEC
:101860001B88022B54D02888424B002C1B780ADBA3
:101870008442A8BF044634B1002B3AD02046BDE8CC
:101880007040FFF7A1BF002B2FD170BD3A4B1B78E2
:10189000002B37D015200BF09BFD384B1860384AD1
:1018A0001288002ADBD0374A186811888142D6DCBA
:1018B000354B2A881B888342A3EB0106A8BF034649
:1018C0005B1AB242BABF02FB03330136534393FBA8
:1018D000F6F31C44C3E72A4B1C888CB12B4B224DDA
:1018E0001C78002CB7D02C88B5E7BDE87040FFF716
:1018F0007FBFFFF741FF2046BDE87040FFF764BFA0
:10190000194DA8E711200CF07FFE1C4B1860C6E7AC
:101910000F200CF079FE1A4B1D4A1B881060002B1B
:10192000A1D01C4AC0F53B63118808338B429ADB77
:10193000194A288812889342A2EB0105A8BF1346D2
:10194000A842A3EB010306DA00FB0333013593FB46
:10195000F5F31C4488E700FB03F292FBF5F31C440B
:1019600082E700BFDE9EFF1FE29EFF1FB29EFF1FA9
:10197000409EFF1F009DFF1FC29EFF1F809CFF1FF8
:101980004A9DFF1FFE9CFF1FDC9EFF1F909EFF1FB6
:10199000989CFF1F489DFF1FC89EFF1F38B5102051
:1019A0000CF032FEC830B0F5FA7FC0F2EE80B0F530
:1019B0007A6F0146A8BF4FF47A6101F51673B3F54B
:1019C0007A6FA8BF4FF47A639BB289B28E4A8F4C6C
:1019D00011802220238007F0C9FE21888C4D8D4C78
:1019E000242007F0C3FE0E200BF0F2FC40F6FF713E
:1019F000C8308842A8BF084620EAE07000F2DC52F6
:101A000083B28A42A8BF0A460220194622802B8050
:101A100007F0ACFE2188042007F0A8FE17200CF088
:101A2000F3FD044616200CF0EFFDA042B8BF20469F
:101A300000F1C801B1F5FA7FC0F2A280B1F57A6F6A
:101A4000A8BF4FF47A6101F54873B3F57A6FA8BF68
:101A50004FF47A639BB289B26F4A704C11800A20AE
:101A6000238007F083FE21880C2007F07FFE0F20E3
:101A70000CF0CAFDC0F53F610431B1F5AF6F7CDBFE
:101A8000B1F5FA6FA8BF4FF4FA6189B2644BC0F5A3
:101A90004360B0F5AF6F19806CDBB0F5FA6FA8BF8B
:101AA0004FF4FA6083B25F4CA420238007F05EFEFF
:101AB000A620218807F05AFE0B200CF0A5F900287B
:101AC00068D011200CF0A0FD00F1C801B1F52F7F06
:101AD0006EDA40F214534FF42F71534A1180534C75
:101AE0000620238007F042FE2188082007F03EFEF2
:101AF00000244FF4AF75E1B24D4809F0A7FC013462
:101B00008542A8BF05460C2CF5D101200CF07CFDC8
:101B1000044600200CF078FD323CA0F13203454928
:101B20006FF4957000FB03F300FB04F081FB0342AC
:101B300081FB0041DB17C017C3EB6223C0EB6120C0
:101B400003F5AF7200F5AF739342A8BF13469D42F1
:101B5000A8BF1D46A5F11401312938DC40F26C7391
:101B600032213548354A018013602A20BDE83840CB
:101B700007F0FCBD4FF4AF6395E74FF4AF6185E725
:101B800040F214534FF4FA7166E740F24C434FF4BD
:101B9000FA711BE715200BF01BFC00F59671B1F5EF
:101BA0002F7F96DB41F25C2399421FDD194694E7B3
:101BB00041F25C239942F9DC1B4A00F5487089B276
:101BC000B0F52F7F118019DA4FF42F7387E740F2B9
:101BD0003A72A5F5B9751A4B02FB05F583FB05238F
:101BE000ED17A5EB631389B23233BAE70E4A00F55D
:101BF000617089B2B0F52F7F1180E5DB8342A8BF09
:101C000003469BB26BE700BF569EFF1F529EFF1F0D
:101C1000449DFF1F0E9FFF1FA89EFF1FC09CFF1F1C
:101C2000489DFF1FC89EFF1FFE9CFF1FDC9EFF1FDD
:101C3000389DFF1F67BBCF46069FFF1F9889FF1F78
:101C4000B5814E1B2DE9F84F0C200BF08DFB0C20BD
:101C50000CF042F8C149DFF88CA314200CF04CF8CA
:101C6000BF49C04809F084F8022103200CF0DAF8DB
:101C7000022104200CF0D6F8022105200CF0D2F845
:101C8000022106200CF0CEF801210A200CF0CAF83F
:101C9000012109200CF0C6F801210D200CF0C2F83A
:101CA000012128200CF0BEF8012114200CF0BAF814
:101CB00002210B200CF0B6F801210C200CF0B2F838
:101CC00000210C200CF09AF8012121200CF0AAF838
:101CD00002211C200CF0A6F801211B200CF0A2F818
:101CE00000211B200CF08AF81C200CF08DF8B0FAB3
:101CF00080F35B091A208AF800300CF029FA1F20C3
:101D000000210CF0EBF904200CF07EF8002800F024
:101D1000EA8005200CF078F8002800F017810023F5
:101D2000914C062023700CF06FF8B0FA80F35B0939
:101D30004FF0000B8D4A137006F096F82378002BB5
:101D400040F0CD80584607F03BFD894B894A1B88FF
:101D500089491488894D8A4840F23A72A3F5AF73D5
:101D600002FB03F381FB0312DB17A3EB6213323395
:101D70002B60844B5A211C7009F0A4FB002800F052
:101D80003781814A81481268DFF85C920023012183
:101D9000FEF78AFB0B200CF037F8011E0CBF012365
:101DA000002389F8003000F0B780794F794D7A4EE2
:101DB000DFF8388200233B602B60336004240F205F
:101DC0000CF022FC336803440E2033600BF000FB60
:101DD0003B6899F8002018443860002A78D0152014
:101DE0000BF0F6FA2B681844286004F0010080F02C
:101DF000010004F005FCB8F80030002B14BF4B20A4
:101E0000DC200CF037F8013CD9D133683968604ADE
:101E10002868624F002BB8BF03330029B8BF0331D5
:101E2000891011605E495F4A098814889B10002858
:101E30003360B8BF03305C4E8210581A19442A60D0
:101E400031603860594D5A485A49161B22442E6059
:101E500002600B60BBF1000F62D1B8F80030002BBC
:101E60004DD0554B012404201C600BF0CDFF18B958
:101E7000524B444A1C701070514B1B881C2B56D07F
:101E8000504C04F1C80523200BF0A2FA44F8040FCB
:101E900001200BF0EFFFAC42F5D19AF800301BB1F6
:101EA000494B1B78002B4CD1002121200BF0A6FFC1
:101EB000464A474B1078187007F08AFA04F098FBEE
:101EC00045F6BF5243494448BDE8F84F0BF038B8D7
:101ED00011200CF099FB2B681844286085E7BDE8B9
:101EE000F84F08F055BE06200BF08EFF00287FF457
:101EF00010AF1D4C034620704FF0010B1AE74FF452
:101F0000FA7004F08DFB04F077FB06F001FB4FF450
:101F1000AF600BF0AFFFA4E711200BF083FF44E7A5
:101F2000FFF73CFDB8F80030002B9AD1E7E72B4BC8
:101F300018880028A4D02A4BC0B2197807F0BCFA40
:101F40009EE7012121200BF059FFB1E703200BF0A0
:101F50005BFFB0FA80F35B09E2E600BF001B374687
:101F600040420F005C91FF1FB29CFF1F489EFF1F65
:101F7000069FFF1FE09EFF1FB5814E1B9889FF1F24
:101F8000389DFF1F149DFF1F2889FF1F709EFF1F94
:101F9000849CFF1F709CFF1FCC9EFF1FD09EFF1FC5
:101FA000A889FF1F2C89FF1F449EFF1FD89CFF1F7D
:101FB000189DFF1F209FFF1FD89EFF1F9C9CFF1F87
:101FC000DE9EFF1F509DFF1F589EFF1F5A9EFF1F42
:101FD0003E9EFF1FA5050000FC9EFF1F1C9DFF1FCE
:101FE000CC9CFF1F429EFF1FC29EFF1F9E9EFF1F95
:101FF00003200BF009FF0028FAD104200BF004FFA6
:102000000028F5D105200BF0FFFE0028F0D10620B6
:102010000BF0FAFE0028EBD10CF016FC2DE9F04F86
:1020200089B005ADA14F2C4608AE611BC9B2A048CE
:1020300009F00CFA3B88834294BF0020012004F889
:10204000010BA642F1D19B489B4A9DF814E09B49A5
:1020500080F800E09DF81600994D10709DF818204A
:102060009DF81C30974E984C0A709DF81A102970F4
:1020700000253370257073B9002940F00F81934F0C
:102080001AB13B78002B40F01F82002800F0F2814B
:102090000222227005E0002A40F0B08005228B4F1A
:1020A00022708B4BDFF888929DF815109DF819006F
:1020B000DFF880A2DFF880B2864DDFF88082864E9E
:1020C0003A709DF81EE019709DF81F209DF81D10B4
:1020D0009DF817C09DF81B7089F80000012000933F
:1020E0008BF800E088F8001032708AF800C02F707A
:1020F0000CF08AFA79497A4AD1F800E0009B7045E1
:10210000CCBF0121002111707CDD764A1288182A8B
:1021100078D875490F880C3A002F78D1734993F815
:1021200000C00B7899F800909AF800109BF80070A6
:1021300095F800B02478A3EB4C03A9EB890A5B1A4D
:102140005344C7EB877AC7EB8A07DFF8A8A11F447F
:1021500098F80030BAF800A007EB4B0796F800B0EB
:102160003B440BFB0A33624F4FF00C0A1AFB043A54
:10217000C7F800A0B9F1000F0BD033784BB15D4B1D
:102180001B88042B0CBF0AF1020A0AF1040AC7F8E3
:1021900000A0594B594CDFF8A8B11B882488DBF804
:1021A00000B0574F574E3F883688033BC4EBC404FA
:1021B0005C4403EB4303DFF88CB10AEB83033B443D
:1021C000DBF800B0504FC6EBC60657F824404F4F1F
:1021D0005E440C3B134457F826601A193244BCF194
:1021E000000F27D02B782BB300295BD1B9FA89F9DE
:1021F000474B4FEA591983F8009023E006222270DA
:10220000324F4EE738490F880022002F86D0012F29
:1022100000F0CF80022F00F0FB80032F00F09480AD
:10222000334F9AF8001093F800C099F80090D7F84F
:1022300000A09FE7364B00241C7011B198F80030C5
:1022400023BB0021334B70451970C8BF324B334953
:10225000C8BFC3F800A00B689A4213D0304B314C72
:1022600018680390039820601B6804932E4C049B0D
:1022700024880A601B1AA34284BF2C4B1A6009B041
:10228000BDE8F08F2748264B0068EDE7BCF1000F52
:10229000D7D1B9F1000FD4D10121D3E704222270A4
:1022A0000A4FFEE61A4B00211970CAE7069FFF1F6E
:1022B000389DFF1F089FFF1F099FFF1F0A9FFF1FD9
:1022C0000B9FFF1F0C9FFF1F4A9EFF1F549EFF1F67
:1022D000399FFF1F3D9FFF1FE49EFF1F9889FF1F2F
:1022E000909EFF1FDE9EFF1F7C9CFF1FAA89FF1F81
:1022F000989EFF1FEC9CFF1FB69EFF1FD49EFF1FE2
:102300008E9CFF1F029DFF1F482901000024010031
:102310001A9FFF1F1B9FFF1F249FFF1FF89CFF1F7B
:1023200028A0FF1FE89CFF1FEE9EFF1F2C9FFF1F92
:102330003B9FFF1F3A9FFF1F3C9FFF1F3E9FFF1FBA
:102340004C9DFF1F149FFF1F664993F800C00B7838
:1023500099F800909AF800109BF8007094F800A08B
:102360002C78A3EB4C03A9EB890B5B1A5B444FF071
:10237000050B1BFB0733009398F800300193009B7B
:10238000DFF86CB1C7EBC707BA440533019FBBF850
:1023900000B003EB440334783B4404FB0B33524C52
:1023A000524F54F82A400C3303EB040AC7F800A03C
:1023B000E0E64C4993F800C00B7899F800909AF841
:1023C00000109BF8007095F800A02478A3EB4C0354
:1023D000A9EB890B5B1A5B44C7EB877BC7EB8B07C9
:1023E000DFF80CB13B4498F80070BBF800B003EB89
:1023F0004A0A3378BA44C4F1060403FB0BA3E4B2DF
:102400004FF00C0A394F1AFB043AC7F800A0B1E6A6
:10241000344993F800C00B7801932B780093019B0B
:102420009AF8001099F800909BF800A02478A3EB8C
:102430004C03A9EB890B5B1A5B44A3F1020B2C4BF9
:10244000CAEBCA0A54441B88DFF8C8A00193BDF840
:1024500000305AF824A098F8004017FB03BB3778E7
:10246000019B5C4407FB03431833204F9A44C7F891
:1024700000A07FE6BEF1000F29D13A78012A2FD9BA
:102480001C4B22701B882BB31B4B1B88013B9BB240
:10249000062B1FD8194B1B78E3B1194B1B68012B76
:1024A0007FF4FFAD1749184B0968184D83FB0130C5
:1024B000CB17C3EB600303EB4303A1EB83032B8038
:1024C000134B03211970ECE503222270E9E5012288
:1024D0002270E6E50A4B1B68012B7FF4E2ADEFE7C3
:1024E0007246DEE5AA89FF1FCC2C0100989EFF1FD3
:1024F000EC9CFF1FC09EFF1F5C9EFF1F469DFF1FA1
:10250000D89EFF1F2C9FFF1FABAAAA2A9C9EFF1FCD
:102510008C89FF1F342B01002DE9F04F3A4B1B78BB
:102520008BB0002B6BD10E200AF052FF0EF092FB05
:1025300001463648364E374DFDF7FCFF3348FDF770
:10254000CFFF0EF0A1FD80F30C003060FFF766FDB9
:102550002C68012C7AD0022C00F01283032C00F09E
:1025600038842D4E2D4C33682D4A2E4E0993099BED
:10257000316812882360591A013A9142274F00F2BC
:10258000FA82294E32689A1A0D2A00F2E382274E07
:1025900032689A1A132A00F2D882254E32689A1AA3
:1025A000252A1AD9234B1B88002B40F06481224B2B
:1025B0001B78002B40F05F81FEF750FE1F4B1B88FD
:1025C0001B3B9BB2022B04D81D4B1B78002B40F009
:1025D000558104F037F8236833601A4D2A689B1A36
:1025E000502B00F21982184B1B88012B00F031820E
:1025F00006F0E6FE06F0CAFD0BB0BDE8F08F08F06D
:102600004FF90BB0BDE8F08FB29CFF1F709EFF1F0B
:10261000AC9EFF1FD89EFF1F28A0FF1F6C9EFF1FB0
:102620009489FF1F409DFF1F2C9DFF1F0C9DFF1FC6
:10263000109DFF1F509EFF1FAC9CFF1FDE9EFF1FC3
:10264000909EFF1F609EFF1FB09EFF1FDFF8389314
:10265000A44AB9F800001378834204D0C3B21846E4
:10266000137006F09FFEDFF81C839F4AB8F8003015
:102670001178994204D09D4F3978002940F04E8757
:102680009B4A336812889B4E9A42C0F201819A4A53
:102690001278002A40F0FC80DFF8F0A2BAF800308F
:1026A00023B9964B1B88002B00F06585944A954B07
:1026B00011881B88944A0B4412685B109342934A1A
:1026C000126880F2078500219342B4BF01230B46B4
:1026D00004910093ACBF4FF0010B8B4605910E2087
:1026E0000AF076FE8A4B8B4A1B6817680393013306
:1026F000A7F25232002B8446029240F32087802BAF
:10270000A8BF8023844A854912780191002A00F0ED
:10271000C9800978914200F0C580B8F80010DFF850
:1027200064E2994201F00A817049AEF800307C4BB6
:102730004FF0010E81F800E01978DFF854E2019BB8
:102740008EF800101A70009B002B00F02381BAF85D
:102750000030002B00F01E81724B1B685A1C002AAF
:1027600040F3F186802A00F3ED866F4C6F49704884
:102770002488098800682144B0EB610FC1F25083BE
:10278000A3F148020F2A02D8473BA9F800300E20D7
:102790000AF01EFE6FF454731F44874202DC654B3F
:1027A00000221A7000200BF02FFF634A634B116860
:1027B000634C1B888842D4BF002201222270002B68
:1027C00000F07E845F4B1C78944243D0884241DD08
:1027D0005D490C78002C00F07A875C4991F800C0C4
:1027E000BCF1000F40F07187594F0097594F5A487C
:1027F0000297574F007887F800C0564F4FF0010EF0
:1028000087F800C081F800E0002841F0E7805349D4
:102810000978002901F03B80514903910C46097861
:10282000002941F031804F484A4F0078397001212A
:102830000297217070B14648444900904A480327E6
:102840000770002008700099029F08700399012406
:102850003C7008701A70454B1B88A3F11B02012ABB
:1028600040F222861D2B7FF47DAE3E4A404B12780B
:102870001A70404C77E6FEF793FC9DE63E4B1B78C2
:10288000002B3FF4A6AE2B68012B7FF4A2AEA2E68C
:1028900031683A4A069106983949106002220B6065
:1028A0002A60F9E61E49DFF8E8E0097800293FF4DC
:1028B00046AF9EF8000081423FF441AF03984B2899
:1028C00041F303801833802BB8F80000A8BF8023A1
:1028D00098423FF434AF2B4803800448012303702F
:1028E0002DE700BF3E9EFF1F149DFF1F9C9CFF1FF6
:1028F000449DFF1F28A0FF1FAC9CFF1F329DFF1FA0
:10290000C09CFF1FA89EFF1FE09CFF1FA49CFF1FF1
:10291000249FFF1F849CFF1F1A9FFF1FF49CFF1F13
:102920001B9FFF1F989EFF1F569EFF1F529EFF1F5B
:10293000D09CFF1F499EFF1F9889FF1F5C9EFF1FB1
:10294000C69CFF1F749CFF1F3C9FFF1FA09EFF1F84
:10295000F29EFF1F469DFF1F3D9FFF1F399FFF1FD8
:10296000759CFF1F909EFF1F8C89FF1FDE9EFF1F1F
:10297000929CFF1F6C9EFF1FE49EFF1F049DFF1F84
:10298000689EFF1FE09EFF1F5A9EFF1FFC9CFF1FBB
:10299000F59CFF1F029B9C45BFF6F9AEA54B1B881B
:1029A000002B3FF4F4AEBBF1000F7FF4D5AEA24B89
:1029B0001B881BB1059B002B7FF4CEAE049B002B24
:1029C0003FF4E5AE9D4B1A78002A7FF4E0AEDFF8C5
:1029D000109399F8004001221A70002C40F098835F
:1029E000974B1B78002B02F0BB80964B1B78002B7B
:1029F00002F09083944B1B78002B7FF4C8AE934B6E
:102A00001B78002B3FF4C3AEB8F8003090490A3B66
:102A1000A8F800300A70BAE605F06EFA8D4B1B7804
:102A200073B98D4B1B785BB98C4B1B7843B98C4BBE
:102A30001B782BB98B4B1B7813B903F0D9FD01E040
:102A400003F0E2FD23682B60874B1B88012B7FF48A
:102A5000CFAD864B864A1B6886481178183B2A22E0
:102A600002FB03F303608448A9B10268934200F3B8
:102A7000C58310DA814D2978002940F09C87804970
:102A80000D68D5F17F0548BF0335AD100135521BE8
:102A90009342B8BF13467B4A1268A92101FB02F298
:102AA000002ABCBF02F57F523F3277499213543A55
:102AB00009881344036051B3744A246852F8211002
:102AC000B4FBF1F2782901FB124200F35883C2EB08
:102AD0000212D20092FBF1F26D4C6E4954F82220A2
:102AE00009686D4CA2F2FF7201FB02F202F57D3221
:102AF00002F5607202EB4201C2EBC10284FB0241AB
:102B00001144D217C2EBA1420B3A1344036063494C
:102B1000634A0C88118804F65C72B2F57C6FA1F1EF
:102B20006400BABF04F65D725E495F4903FB02F2BE
:102B300081FB02311144D317C3EBE123C11881F3A8
:102B40000C0128200AF0CAFF52E5FEF77DFE23683B
:102B5000336022E5FDF714FFFEF7ACFB534B1B88F7
:102B6000032B00F01085524B1B88032B00F00785C8
:102B7000236833600BE5FDF74FFE3B68336000E5EB
:102B80004C4A34681288A24204DB364B1B78002B77
:102B900000F06083484E494833680793484B0799D3
:102BA00000681B88091A994200F2C180002B00F0CE
:102BB000BE80444B198800293FF4D4AC424B4348B3
:102BC0001B680088A342B8BF23469A4241F3218183
:102BD0003F4B1A60DFF80C8188F80010234FFDF797
:102BE0001BFE38687F2840F362853A4B7F3883FBB1
:102BF0000032C317C3EB620303EB4303A0EB830074
:102C00007330354B01931B883860002B40F07D8674
:102C1000124B00931B78002B00F0C7832F4C2378B6
:102C2000002B00F0C283DFF8C090DFF8A8A04FF0BF
:102C3000000B68E0329DFF1F649EFF1F499EFF1F2F
:102C4000399FFF1F3A9FFF1F3B9FFF1F3C9FFF1FA6
:102C50009C9CFF1F469DFF1FA09EFF1FF29EFF1F13
:102C6000759CFF1FAC9CFF1FB09EFF1F2C9FFF1F7A
:102C7000009DFF1F249DFF1F349DFF1FF89EFF1F17
:102C8000F49EFF1F9089FF1F909CFF1F00290100E9
:102C9000FC210100C49EFF1F4D261281309FFF1FA3
:102CA000049FFF1F81DFFF8183200882B29EFF1FE8
:102CB000409EFF1F449DFF1F28A0FF1F049DFF1F74
:102CC000309DFF1F949CFF1F689EFF1F0E9FFF1FDC
:102CD000789CFF1FABAAAA2ADC9CFF1F5489FF1F08
:102CE0004A9EFF1F209DFF1F2C89FF1F03F17300C9
:102CF000C0B298F8001006F00FFC23780BF1010B1E
:102D00005B4540F352833B6859F8040F1844A0F127
:102D10007F038AFB0321DA17C2EB610202EB420256
:102D20007F28A3EB8203E1DCFDF796FCE0E7554B3F
:102D300055491B6808885549A342B8BF23469A42A3
:102D400000F36F82524C09888342A8BF0346236078
:102D500000297FF43FAF9A42C8BF0B4640F3688218
:102D6000801AB0F5804FAABF9B03C3EB83330130B9
:102D700093FBF0F0FDF736FDC0F3C6100DF06AFFCF
:102D8000444B044618880DF065FF4349074620462A
:102D90000DF0B4FF014638460DF0B0FF21460DF0AE
:102DA000A5FE4FF07E5104460EF046F9002841F092
:102DB00025803A4920460EF05DF9002840F008864B
:102DC00020460EF087F9C0B2DFF8F08088F80000E6
:102DD00004E7334B34681988A14273DD314B1B780B
:102DE000002B6FD1DFF8D89099F800007F2840F3CE
:102DF000DE85A3F155337F3803F1004383FB0032B6
:102E0000C317C3EB620303EB4303A0EB83007330F0
:102E1000254B01931B88C0B289F80000002B40F0BD
:102E2000D887224B00931B78002B00F07D84204C28
:102E30002378002B00F078841E4FDFF87C804FF061
:102E4000000A0AE003F17300C0B206F089FB2378A0
:102E50000AF1010A534540F3678457F8043F99F893
:102E600000001844A0F17F0388FB0321DA17C2EBAE
:102E7000610202EB42027F28A3EB8203E2DCFDF752
:102E8000EBFBE1E7689EFF1F0E9FFF1F949CFF1F57
:102E9000789CFF1F1C9FFF1FCDCCCC3D0000FE4245
:102EA000449DFF1FAC9CFF1FDC9CFF1FF29EFF1F79
:102EB0005489FF1F2C89FF1FABAAAA2A209DFF1F40
:102EC000949EFF1FB24F38687F2840F3B881B14B02
:102ED0007F3883FB0032C317C3EB620303EB43036A
:102EE000A0EB83007330DFF8049399F800A08245CB
:102EF00000F00182A84B1B88002B43D1A74AA848A9
:102F000012680088914205DC8242D4BFC1EB020303
:102F1000C1EB0003411AB1F5804FA6BF9B030131FD
:102F2000C3EB833393FBF1F0FDF75CFCC0F3C610F9
:102F30000DF090FE9B4B044618880DF08BFE9A49CD
:102F4000804620460DF0DAFE014640460DF0D6FEE2
:102F500021460DF0CBFD4FF07E5104460EF06CF88B
:102F6000002840F0A686914920460EF083F80028FC
:102F700040F02B8520460EF0ADF8C0B2DFF870822D
:102F800088F80000BAF17F0F40F38D838148AAF1E1
:102F90007F0A80FB0A304FEAEA73C3EB600000EB64
:102FA0004000AAEB80007330814B00931B78C0B2C5
:102FB00089F80000002B40F0ED827E4B03931B78D4
:102FC000002B40F0D7847C4B02931B78002B40F001
:102FD00018877A4B0193029B1B78FBB1784B1B88B7
:102FE000012B00F0E485022B00F07087032B01F029
:102FF0008A81042B01F01183052B01F02D84062B0F
:1030000001F08285072B01F03587082B02F03B8009
:10301000092B02F07F810A2B02F09482009B1B781F
:10302000002B00F04484019B644C1988002900F0B7
:103030009A8438687F2840F3AA82564B7F3883FBF6
:103040000032C317C3EB620303EB4303A0EB83001F
:1030500073303860002940F04F84009B1B78002BB0
:1030600000F05581574C2378002B00F05081DFF899
:1030700084A1DFF87C814FF0000B0CE003F17300BA
:10308000C0B298F8001006F047FA23780BF1010B54
:103090005B4540F33C813B685AF8040F3D4A1844B5
:1030A000A0F17F0382FB0321DA17C2EB610202EB7E
:1030B00042027F28A3EB8203E0DCFDF7CDFADFE7D5
:1030C0003D4C41483A493B4A237003700B701370E2
:1030D000FFF7C1BB93424FF0000B80F2B380012396
:1030E000CDF800B0CDF814B00493FFF7F8BA374B21
:1030F0001B78002B7FF44BAB039B354A243B83F3B7
:103100004703D9B25B20136006F0D6F999F8004066
:10311000032C30D1DFF8E08098F80030002B42F02B
:1031200041812C4F3B78002B42F02F81274C237894
:10313000002B42F01D81284B1B78002B42F00B81A5
:10314000264A1380264B1B78002B42F0D181124B6C
:103150007F221A8098F800306BB93B785BB92378EE
:103160004BB9204A7F210720138006F0A5F97F2163
:103170000B2006F0A1F91C4B1F68FFF708BBC2EB40
:103180000214013102EBC40292FBF1F2A4E400BF8D
:103190002C9FFF1FABAAAA2A949CFF1F789CFF1F9D
:1031A0000E9FFF1F1C9FFF1FCDCCCC3D0000FE4299
:1031B000F29EFF1F759CFF1F469DFF1FDC9CFF1F9B
:1031C0005C9EFF1F5489FF1FA09EFF1F3C9FFF1F97
:1031D000BC9CFF1F3B9FFF1F3A9FFF1F3A9DFF1F95
:1031E0003D9FFF1F929EFF1F849CFF1F949EFF1F09
:1031F000209DFF1F2C89FF1F399FFF1FB3490D78AA
:10320000002D40F03783B2490968D1F17F0148BFF2
:10321000033102EBA1014A1C93420260A8BF13468E
:1032200039E4AC4B09881A6000297FF4D3AC13460B
:103230009842D4BFC2EB0003C2EB030390E5FDF755
:103240000BFA50E60123CDF810B0CDF800B005938D
:10325000FFF745BA01232B60FFF783B9029B1B7868
:10326000FBB19D4B1B88012B00F01A84022B00F050
:10327000AB86032B00F0CE87042B01F0F381052BE6
:1032800001F06E82062B01F03784072B01F03F8599
:10329000082B01F0AF86092B02F005800A2B02F003
:1032A0007681019B1B88002B00F02083009B1B78FC
:1032B0003BB9039B1B7823B9029B1B78002B00F0C2
:1032C0008987864B1B78002B00F0FE8084490B78A1
:1032D000082B00F2F98083483A680068824C013379
:1032E000DBB25F1E101A44F827000B707F4B346866
:1032F000198889F80020A1427D4EBFF633A93268B3
:103300007C4B0892089A7C4C1A60FFF72CB9039BFF
:103310001B78002BA2D03B68A3F10C007F2840F360
:10332000408376488B3B80FB0320DA17C2EB6000BA
:1033300000EB4000A3EB800303F17300DFF8D081C2
:10334000C0B298F8001006F0E7F8009B1B78002B3D
:1033500084D0634C2378002B80D0DFF8B8A14FF0E5
:10336000000B0CE003F17300C0B298F8001006F0F7
:10337000D3F823780BF1010B5B457FF76FAF3B6808
:103380005AF8040F5D4A1844A0F18B0382FB032115
:10339000DA17C2EB61020C3802EB42027F28A3EB82
:1033A0008203DFDCFDF758F9DEE74C4B1B78002B7E
:1033B00040F0B2823B68524A1278002A45D0A3F10D
:1033C0000C007F2840F3F0824C4A8B3B82FB0321A8
:1033D000DA17C2EB610202EB4202A3EB820303F1B4
:1033E0007300C0B298F8001006F096F8009B1B78A6
:1033F00053B33B4C23783BB3DFF81891DFF8FCA0C4
:103400004FF0000B0BE003F17300C0B298F800100E
:1034100006F082F823780BF1010B5B4514DD3B6865
:1034200059F8040F1844A0F18B038AFB0321DA1723
:10343000C2EB61020C3802EB42027F28A3EB82034D
:10344000E1DCFDF709F9E0E73B682E4A1278FAB1B2
:10345000214A1288012A00F02F84022A00F03586C2
:10346000032A00F0CA87042A01F02081052A01F00E
:103470005582062A01F06D83072A01F0A383082AEA
:1034800001F05B86092A01F0D1860A2A02F0BD808C
:10349000019A1288002A00F04A821B4A164C1370C7
:1034A00003232B60FFF75FB8DFF86C8098F80030DB
:1034B000002B40F00081154F3B78002B40F0B38487
:1034C0000D4C3B70FFF74FB83A680FE7F89EFF1FAF
:1034D000F49EFF1F789CFF1F5C9EFF1FA09EFF1F96
:1034E0005489FF1FA09CFF1F3089FF1F449DFF1FB1
:1034F00028A0FF1FD49FFF1F6C9EFF1FABAAAA2A04
:10350000759CFF1F469DFF1F949EFF1F929CFF1FEF
:10351000209DFF1F2C89FF1F909EFF1FDBB21846C6
:10352000137006F087F8A54BA5491A46A54B184617
:1035300000230B703B7013700370FFF7A1B80123D9
:10354000FFF7E0B88024A049A04BA14A09881B8856
:1035500012680B44B2EB630FBFF619A99D4B1B78A1
:10356000002B40F0F181B8F800309B4AA3423FF4B1
:103570000EA99A4B148001221A70FFF708B9FDF7C3
:10358000D3F8FFF7F5BAFDF779F8FFF7ECBAFDF7D6
:1035900063F85EE5924B01931B8863BB894B0393F1
:1035A000904B0293904C23787BB3DFF85882DFF87E
:1035B0003CA24FF0000B09E003F17300C0B205F02C
:1035C000CFFF23780BF1010B5B451EDD58F8043F5C
:1035D00099F800001844A0F17F038AFB0321DA1751
:1035E000C2EB610202EB42027F28A3EB8203E3DC21
:1035F000FDF732F8E2E7734B03937A4B029305F041
:10360000AFFF009B1B78002BCCD1039B1B78002BBA
:103610003FF4E1AC99F80030A3F10C007F2840F3AF
:10362000BD8172488B3B80FB0320DA17C2EB600040
:1036300000EB4000A3EB800303F17300C0B205F080
:103640008FFF009B1B78002B00F09D81664C237838
:10365000002B01F06282DFF8AC81DFF890A14FF01F
:10366000000B0AE003F17300C0B205F079FF237884
:103670000BF1010B5B457FF7AEAC58F8043F99F8AE
:1036800000001844A0F18B038AFB0321DA17C2EB78
:1036900061020C3802EB42027F28A3EB8203E1DCDB
:1036A000FCF7DAFFE0E75046FCF7D6FF7CE4FCF7D6
:1036B000D3FFFFF7A6BA4E4A1278002A40F09B814A
:1036C0004C4F4D4C3B70FEF74EBF002008704B49ED
:1036D000087840B1394900910978002900F07B81D0
:1036E000009F002139704649097800297FF494A889
:1036F000002C40F0CC80002840F0C980354C2F4F82
:1037000094F800E02F4C0394364C02942D4C2C4935
:103710002070344C0097087038702070BEF1000F94
:103720007FF48CA8FFF796B8264B1B78002B6BD044
:1037300099F80030A3F10C007F2840F399832B4ABD
:103740008B3B82FB0321DA17C2EB610202EB4202E0
:10375000A3EB820303F17300C0B205F001FF009BED
:103760001B78002B50D0204C2378002B4CD0254FB9
:10377000DFF878804FF0000A09E003F17300C0B26F
:1037800005F0EEFE23780AF1010A53453CDD57F8B7
:10379000043F99F800001844A0F18B0388FB032133
:1037A000DA17C2EB61020C3802EB42027F28A3EB6E
:1037B0008203E2DCFCF750FFE1E700BFF29EFF1F4F
:1037C000A09EFF1F759CFF1F569EFF1F529EFF1F4E
:1037D000D09CFF1F909EFF1FE09EFF1F9C9CFF1F21
:1037E000DC9CFF1F469DFF1F5489FF1FABAAAA2A1E
:1037F000E49EFF1F929CFF1F6C9EFF1F3D9FFF1FBB
:10380000399FFF1F2C89FF1F914B1B78FBB1914BF8
:103810001B88012B00F07A86022B00F07487032BA3
:1038200001F0ED80042B01F08381052B01F0C183B1
:10383000062B01F0E584072B01F0C085082B01F071
:103840001887092B01F091870A2B01F06F87019BE4
:103850001B88002B00F0B8827F4B1B78002B40F0B8
:10386000AE827E4B7E4A19883468002001231060A6
:103870002B6040E50135EDB2022D86BF00230B70B1
:103880000D701346FFF707B90398002101707549C1
:10389000097800293EF4DEAF6D49029109780029CC
:1038A00000F05787029800210170FEF7D3BF039BF9
:1038B0001B78002B7FF4B7AB029B1B78002B7FF4A7
:1038C000B2AB019B1988FFF7B4BB243B002BB8F8BF
:1038D000000040F3798498423EF431AF9BB26248D5
:1038E000A8F8003001230370FEF729BF5F4B38783A
:1038F000197805F011FED9E4DFF87081C0B298F8AC
:10390000001005F009FEFFF7A8BBC0B298F8001040
:1039100005F002FEFFF77CB97F21402005F0CCFDC9
:103920005349544A3B680B600021117043E5D8B2FB
:1039300098F8001005F0F0FD3B68AEE54E4BDFF85F
:1039400058E11978FEF7FBBE4B2C40F34682183441
:10395000802CB8F80030494AA8BF8024A3427FF4E5
:1039600008AEFEF714BF99F8000005F0F9FD2188B4
:10397000FFF75FBB424B01931B88002B41F036875A
:10398000334B029346E6029B1B78002B7FF426AB59
:10399000039B1B78002B7FF446AB92E7FCF75CFEA1
:1039A0004CE6FCF759FEC9E4FCF756FE19E5FCF7B6
:1039B00053FEFFF72DBA4B1CDBB2022B40F25B82A9
:1039C00000232B701346FFF766B87F20FFF7D6BAA7
:1039D0007F20FFF7F9B91E4F1F4902974FF0000CE7
:1039E00081F800C0009F02994FF0010E87F800E0B7
:1039F00081F800C077E6234F387802F073FE224B3F
:103A00001B78002B00F045823B887E2B00F2418220
:103A10001E4CDFF888902268D9F80010521A0F2A3D
:103A200040F22E821A4A0133108899B23980002858
:103A300000F04882C9B2C0B205F03EFD154F2268C1
:103A400098F80030C9F800203B70FEF78CBD00BF2D
:103A5000469DFF1F5C9EFF1FA09EFF1F449DFF1FF2
:103A6000789CFF1F909EFF1F9C9CFF1F209DFF1FA7
:103A7000A09CFF1F5489FF1F1B9FFF1FE09EFF1F7D
:103A8000DC9CFF1FCC9CFF1F3E9FFF1F6C9EFF1FF7
:103A90001C9DFF1F929CFF1FF59CFF1F289FFF1F6F
:103AA000DFF8B4A33868BAF80030E44AE44CC31A2B
:103AB00082FB031ED917C1EB6E0101EB4101A3EBA1
:103AC000810303EB430354F8233018447F2840F369
:103AD00090847F3882FB0032C317C3EB620303EB91
:103AE0004303A0EB83007330DFF87083DFF870B31B
:103AF00098F80010C0B205F00FFDBBF80030022BA3
:103B00007FF6CFAB3968BAF80030CC4ACB1A82FBCB
:103B1000030ED817C0EB6E0000EB4000A3EB800350
:103B200003EB430304EB8303586808447F2840F306
:103B300058877F3882FB0032C317C3EB620202EB67
:103B40004202A0EB82007330C0B298F8001005F07A
:103B5000E3FCBBF80030032B7FF6A3AB3968BAF85F
:103B60000030B64ACB1A82FB030ED817C0EB6E00AA
:103B700000EB4000A3EB800303EB430304EB83045F
:103B8000A06808447F2840F381817F3882FB00329F
:103B9000C317C3EB620202EB4202A0EB8200733058
:103BA00098F80010C0B205F0B7FCFFF77ABBDFF859
:103BB000A8A299F80000BAF80030A04AA04CC31A95
:103BC00082FB031ED917C1EB6E0101EB4101A3EB90
:103BD000810303EB430354F8233018447F2840F358
:103BE00083847F3882FB0032C317C3EB620303EB8D
:103BF0004303A0EB83007330DFF864B2C0B205F07A
:103C0000AFFCBBF80030022B7FF608AA99F8001031
:103C1000BAF80030894ACB1A82FB030ED817C0EBE2
:103C20006E0000EB4000A3EB800303EB430304EBC7
:103C30008303586808447F2840F3D7867F3882FB87
:103C40000032C317C3EB620202EB4202A0EB820018
:103C50007330C0B205F084FCBBF80030032B7FF654
:103C6000DDA999F80010BAF80030744ACB1A82FB2B
:103C7000030ED817C0EB6E0000EB4000A3EB8003EF
:103C800003EB430304EB8304A06808447F2840F35C
:103C9000E9807F3882FB0032C317C3EB620202EB7C
:103CA0004202A0EB82007330C0B205F059FCFFF76E
:103CB000B5B90120FFF762B9DFF89CA15F49BAF8F6
:103CC00000205F4C9A1A81FB020ED017C0EB6E00E9
:103CD00000EB4000A2EB800202EB420254F822000B
:103CE00018447F2840F30484A0F17F0381FB032163
:103CF000DA17C2EB610000EB4000A3EB80007330E9
:103D0000DFF85CB198F80010C0B205F005FCBBF814
:103D10000030022B50D93968BAF80030474ACB1A24
:103D200082FB030ED817C0EB6E0000EB4000A3EB44
:103D3000800303EB430304EB8303586808447F28A4
:103D400040F3C0867F3882FB0032C317C3EB6202A8
:103D500002EB4202A0EB82007330C0B298F8001070
:103D600005F0DAFBBBF80030032B25D93868BAF828
:103D70000030324AC31A82FB031ED917C1EB6E0111
:103D800001EB4101A3EB810303EB430304EB830449
:103D9000A36818447F2868DD7F3882FB0032C31790
:103DA000C3EB620202EB4202A0EB82007330C0B2AE
:103DB00098F8001005F0B0FB3B68FFF769BB0021E5
:103DC000402005F079FB4CE599F8000005F0C8FBB0
:103DD00042E505F0C5FBFFF724B8243C002CB8F8F9
:103DE000003040F30686A3423EF4D1ACA4B2154B9A
:103DF000A8F8004001221A70FEF7C9BC0120FEF7A6
:103E0000E3BF114B01931B88002B3FF4E4A8FFF79D
:103E1000F6BB0E4A8342A8BF03461360FEF7DABE24
:103E20001446FFF79BBB0A4B0A4C19886A2005F021
:103E30009DFC98F800303B70FEF795BBABAAAA2A10
:103E4000042801009C9CFF1FDC9CFF1F789CFF1F27
:103E5000CC9CFF1F6C9EFF1F9C9EFF1F209DFF1F81
:103E6000B09CFF1FFCF7F8FB1EE7FCF7F5FB9EE795
:103E7000FCF7F2FB70E42B701346FEF70CBEDA4C35
:103E8000DA4F98F800303B70FEF76DBBFCF7E4FBAF
:103E900086E6D74B1B78002BF1D03B88D54F002B03
:103EA000EDD0D14CDFF85C932268D9F80010521A9B
:103EB0000F2AE5D9D04A013B108899B239800028F1
:103EC0007FF4B8ADC8B205F097FBB7E5DFF838A3CB
:103ED00099F80000BAF80030C84AC94CC31A82FBEE
:103EE000031ED917C1EB6E0101EB4101A3EB810366
:103EF00003EB430354F8233018447F2840F3FA833C
:103F00007F3882FB0032C317C3EB620303EB43032A
:103F1000A0EB83007330DFF8F4B2C0B205F020FBF1
:103F2000BBF80030022B7FF679A899F80010BAF898
:103F30000030B24ACB1A82FB030ED817C0EB6E00DA
:103F400000EB4000A3EB800303EB430304EB83038C
:103F5000586808447F2840F3E7857F3882FB0032A9
:103F6000C317C3EB620303EB4303A0EB830073307F
:103F7000C0B205F0F5FABBF80030032B7FF64EA86F
:103F800099F80010BAF800309C4ACB1A82FB030E55
:103F9000D817C0EB6E0000EB4000A3EB800303EBEF
:103FA000430304EB8304A06808447F287FF75AAFDB
:103FB0007F3882FB0032C317C3EB620303EB43037A
:103FC000A0EB830073306FE6DFF83CA23868BAF8E4
:103FD00000308A4A8A4CC31A82FB031ED917C1EBF0
:103FE0006E0101EB4101A3EB810303EB430354F8A2
:103FF000233018447F2840F380837F3882FB0032CF
:10400000C317C3EB620303EB4303A0EB83007330DE
:10401000DFF8FC81DFF8F4B198F80010C0B205F0C9
:104020007BFABBF80030022B7FF63BA93968BAF85F
:104030000030724ACB1A82FB030ED817C0EB6E0019
:1040400000EB4000A3EB800303EB430304EB83038B
:10405000586808447F2840F374857F3882FB00321B
:10406000C317C3EB620303EB4303A0EB830073307E
:10407000C0B298F8001005F04FFABBF80030032BDF
:104080007FF60FA93868BAF800305C4AC31A82FB81
:10409000031ED917C1EB6E0101EB4101A3EB8103B4
:1040A00003EB430304EB8304A36818447F287FF7E2
:1040B000EDAE7F3882FB0032C317C3EB620303EB24
:1040C0004303A0EB830073306AE5DFF83CA14B4962
:1040D000BAF800204A4C9A1A81FB020ED017C0EBA6
:1040E0006E0000EB4000A2EB800202EB420254F8AB
:1040F000220018447F2840F30383A0F17F0381FB53
:104100000321DA17C2EB610000EB4000A3EB800053
:104110007330DFF8F8B098F80010C0B205F0FCF981
:10412000BBF80030022B7FF647AE3968BAF8003092
:10413000324ACB1A82FB030ED817C0EB6E0000EB9D
:104140004000A3EB800303EB430304EB83035868B5
:1041500008447F2840F3F9847F3882FB0032C3177C
:10416000C3EB620303EB4303A0EB83007330C0B2E5
:1041700098F8001005F0D0F9BBF80030032B7FF65B
:104180001BAE3868BAF800301C4AC31A82FB031E03
:10419000D917C1EB6E0101EB4101A3EB810303EBE6
:1041A000430304EB8304A36818447F287FF75DAEC4
:1041B0007F3882FB0032C317C3EB620303EB430378
:1041C000A0EB83007330F2E501283EF4B8AA012386
:1041D000FFF785BB4FF47A43013BFDD199F800000E
:1041E00005F0BEF9FFF76DB86C9EFF1F929CFF1F94
:1041F0003D9FFF1FCC9CFF1F1C9DFF1FABAAAA2A3F
:10420000F0290100289FFF1F9C9EFF1FB09CFF1FED
:10421000209DFF1FDFF8E8A23868BAF80030B64AE0
:10422000B64CC31A82FB031ED917C1EB6E0101EB1A
:104230004101A3EB810303EB430354F823301844FB
:104240007F2840F3DB817F3882FB0032C317C3EB4A
:10425000620202EB4202A0EB82007330DFF8A4821C
:10426000DFF8A4B298F80010C0B205F055F9BBF819
:104270000030022B7FF615A83868BAF800309E4A45
:10428000C31A82FB0321DA17C2EB610202EB42027E
:10429000A3EB820303EB430304EB83035B68184443
:1042A0007F2840F31C847F380C2290FBF2F302FB42
:1042B00013007330C0B298F8001005F02DF9BBF868
:1042C0000030032B7EF6EDAF3868BAF800308A4A2A
:1042D000C31A82FB0321DA17C2EB610202EB42022E
:1042E000A3EB820303EB430304EB8304A3681844AA
:1042F0007F287FF7CBAD7F380C2290FBF2F302FBD7
:10430000130073304CE4DFF8F8A199F80000BAF814
:104310000030794A794CC31A82FB031ED917C1EBCE
:104320006E0101EB4101A3EB810303EB430354F85E
:10433000233018447F2840F364817F3882FB0032A9
:10434000C317C3EB620202EB4202A0EB82007330A0
:10435000DFF8B4B1C0B205F003F9BBF80030022BAE
:104360007EF65CAE99F80000BAF80030624AC31AD3
:1043700082FB0321DA17C2EB610202EB4202A3EBDC
:10438000820303EB430304EB83035B6818447F2839
:1043900040F39C837F380C2290FBF2F302FB130066
:1043A0007330C0B205F0DCF8BBF80030032B7EF6AA
:1043B00035AE99F80000BAF800304F4AC31A82FBB4
:1043C0000321DA17C2EB610202EB4202A3EB820384
:1043D00003EB430304EB8304A36818447F287FF7AF
:1043E00041AD7F380C2290FBF2F302FB13007330D7
:1043F0005AE4FCF731F9FFF777BBDFF804A13E4937
:10440000BAF800203D4C9A1A81FB020ED017C0EB7F
:104410006E0000EB4000A2EB800202EB420254F877
:10442000220018447F2840F3EF80A0F17F0381FB36
:104430000321DA17C2EB610101EB4101A3EB81001B
:104440007330DFF8C4B098F80010C0B205F064F81B
:10445000BBF80030022B7FF6AFAC3868BAF80030FA
:10446000254AC31A82FB0321DA17C2EB610202EB71
:104470004202A3EB820303EB430304EB83035B6879
:1044800018447F2840F332837F380C2290FBF2F3EC
:1044900002FB13007330C0B298F8001005F03CF82E
:1044A000BBF80030032B7FF687AC3868BAF80030D1
:1044B000114AC31A82FB0321DA17C2EB610202EB35
:1044C0004202A3EB820303EB430304EB8304A368E0
:1044D00018447F287FF7C9AC7F380C2290FBF2F399
:1044E00002FB1300733062E4FCF7B6F8FFF784BBFD
:1044F000FCF7B2F804E400BFABAAAA2A802A0100A4
:104500009C9EFF1F209DFF1FB09CFF1FDFF83CA358
:1045100099F80000BAF80030C44AC54CC31A82FBAF
:104520000317D917C1EB670101EB4101A3EB81032D
:1045300003EB430354F8233018447F286ADD7F38A7
:1045400082FB0032C317C3EB620202EB4202A0EB14
:1045500082007330DFF8F8B2C0B205F001F8BBF8A2
:104560000030022B7FF673A999F80000BAF80030EA
:10457000AE4AC31A82FB0321DA17C2EB610202EBD7
:104580004202A3EB820303EB430304EB83035B6868
:1045900018447F2840F3AD827F380C2290FBF2F361
:1045A00002FB13007330C0B204F0DAFFBBF8003036
:1045B000032B7FF64CA999F80000BAF800309B4A0B
:1045C000C31A82FB0321DA17C2EB610202EB42023B
:1045D000A3EB820303EB430304EB8304A3681844B7
:1045E0007F2814DD7F380C2290FBF2F302FB1300CE
:1045F0007330C0B204F0B4FFFFF729B9FCF72CF810
:104600002CE6FCF729F8A3E6FCF726F819E7FCF7F7
:1046100023F8EEE7FCF720F89CE7DFF830A299F8E2
:104620000000BAF80030814A824CC31A82FB031E94
:10463000D917C1EB6E0101EB4101A3EB810303EB41
:10464000430354F8233018447F28DADD7F3882FB97
:104650000032C317C3EB620303EB4303A0EB8300F9
:10466000733075E6DFF8E4A13868BAF800306F4AB5
:10467000704CC31A82FB031ED917C1EB6E0101EB0C
:104680004101A3EB810303EB430354F823301844A7
:104690007F28B3DD7F3882FB0032C317C3EB620390
:1046A00003EB4303A0EB83007330D7E5DFF89CA155
:1046B0005E49BAF800205F4C9A1A81FB020ED017AF
:1046C000C0EB6E0000EB4000A2EB800202EB420266
:1046D00054F8220018447F2896DDA0F17F0381FB67
:1046E0000321DA17C2EB610000EB4000A3EB80006E
:1046F0007330A6E6FBF7B0FF0DE4FBF7ADFF87E4F0
:10470000FBF7AAFF05E5DFF844A199F80000BAF825
:104710000030464A484CC31A82FB0317D917C1EB35
:10472000670101EB4101A3EB810303EB430354F861
:10473000233018447F287FF76DAF7F3882FB00322B
:10474000C317C3EB620303EB4303A0EB8300733097
:1047500000E73A4800903A483A490390FEF76EB8AD
:10476000DFF8E8A03868BAF80030304A364CC31A8F
:1047700082FB0321DA17C2EB610202EB4202A3EBD8
:10478000820303EB430354F8233018447F2840F39B
:10479000A0817F380C2290FBF2F302FB13007330F0
:1047A000DFF8B080DFF8A8B098F80010C0B204F0CD
:1047B000B3FEBBF80030022B1AD93868BAF80030C3
:1047C0000C22C11A91FBF2F302FB131302FB034309
:1047D0005B6818447F2840F352847F3890FBF2F3E3
:1047E00002FB13007330C0B298F8001004F094FE7E
:1047F000BBF80030032B7EF654ADBAF800303868B1
:104800000C22C11A91FBF2F302FB131302FB0344C7
:10481000A36818447F287FF739AB7F3890FBF2F309
:1048200002FB13007330FFF7BBB900BFABAAAA2A83
:104830000428010070240100F0290100F29EFF1FEE
:10484000759CFF1FA09EFF1F042D01009C9EFF1F53
:10485000B09CFF1F209DFF1FDFF860A399F80000A8
:10486000BAF80030CC4ACD4CC31A82FB0321DA17C8
:10487000C2EB610202EB4202A3EB820303EB4303B0
:1048800054F8233018447F2840F32D817F380C22C0
:1048900090FBF2F302FB13007330DFF824B3C0B2D5
:1048A00004F05EFEBBF80030022B19D999F8000025
:1048B000BAF800300C22C11A91FBF2F302FB131379
:1048C00002FB03435B6818447F2840F390837F38E2
:1048D00090FBF2F302FB13007330C0B204F040FE11
:1048E000BBF80030032B7EF699ABBAF8003099F88C
:1048F00000000C22C11A91FBF2F302FB131302FB1E
:104900000344A36818447F287FF7ACAA7F3890FB44
:10491000F2F302FB13007330FFF7C6B9DFF89CA275
:104920009D49BAF800209D4C9A1A81FB0210D117BC
:10493000C1EB600101EB4101A2EB810202EB4202FB
:1049400054F8220018447F2840F3C680A0F17F036A
:104950000C2093FBF0F200FB12307330DFF860B2F2
:1049600098F80010C0B204F0D7FDBBF80030022B5D
:104970001AD93868BAF800300C22C11A91FBF2F348
:1049800002FB131302FB03435B6818447F2840F3C8
:104990002B837F3890FBF2F302FB13007330C0B21D
:1049A00098F8001004F0B8FDBBF80030032B7FF638
:1049B00003AABAF8003038680C22C11A91FBF2F34E
:1049C00002FB131302FB0344A36818447F287FF7FC
:1049D0004CAA7F3890FBF2F302FB13007330FFF711
:1049E000E6B9FBF739FEFFF7AFB8FBF735FEFFF787
:1049F00030B9012B3DF4CBAE0124FFF7F8B9DFF855
:104A0000BCA199F80000BAF80030634A644CC31A9C
:104A100082FB0321DA17C2EB610202EB4202A3EB35
:104A2000820303EB430354F8233018447F2846DD08
:104A30007F380C2290FBF2F302FB13007330DFF897
:104A400080B1C0B204F08CFDBBF80030022B19D944
:104A500099F80000BAF800300C22C11A91FBF2F369
:104A600002FB131302FB03435B6818447F2840F3E7
:104A70008F807F3890FBF2F302FB13007330C0B2DB
:104A800004F06EFDBBF80030032B7EF6E0AEBAF802
:104A9000003099F800000C22C11A91FBF2F302FBDE
:104AA000131302FB0344A36818447F287FF7AFADBC
:104AB0007F3890FBF2F302FB1300733099E5FBF7AC
:104AC000CBFDBCE7FBF7C8FDFFF747B9FBF7C4FD1B
:104AD00067E4FBF7C1FD63E6FBF7BEFD3EE7FBF7CE
:104AE000BBFDFFF7E7BBFBF7B7FDD6E6FBF7B4FD71
:104AF000D1E4FBF7B1FD56E5DFF8C0A03868BAF89D
:104B00000030254A274C32E6DFF8B0A099F80000C3
:104B1000BAF80030204A234CA6E6029B1B78002BF3
:104B20007EF45CAAFEF77FBAFBF796FDFFF720BA8A
:104B3000DFF888A099F80000BAF80030164A1A4C3D
:104B400065E7FBF789FDFFF793BAFBF785FDFFF7F4
:104B50000EBBDFF868A01049BAF80020114CE3E65C
:104B6000124B1B78002B00F0C282114B1B78002BDC
:104B70007DF40DAE0F4B1B78002B3DF408AEB8F85A
:104B800000300D490A33A8F800300A70FDF7FFBD68
:104B9000FBF762FD73E700BFABAAAA2A042D010050
:104BA000802A0100AC2B0100702401003A9FFF1FF6
:104BB0003B9FFF1F3C9FFF1F9C9CFF1F9C9EFF1F56
:104BC000B09CFF1FA44C2288002A00F02183A34937
:104BD000DFF89CB20988BBF800000331884227DD6A
:104BE0009F48A0490088B1F800E0DFF87CC2181A9D
:104BF0000C2190FBF1F901FB19004FF0900909FB22
:104C00000EFE01FB00E06FF00B0E5CF800000344A9
:104C10000EFB02307F2840F3F1847F3890FBF1F3E4
:104C200001FB13007330C0B298F8001004F074FC5C
:104C3000BBF8002023881344022B23DD884B894ACC
:104C400038681B88B2F800C0DFF81CE2C31A0C21D8
:104C500093FBF1F201FB1232902303FB0CF301FBF7
:104C6000023373445B6818447F2840F351857F38D2
:104C700090FBF1F301FB13007330C0B298F8001001
:104C800004F04AFCBBF8002023881344032B23DDE7
:104C9000734B744A38681B88B2F800C0DFF8C8E16B
:104CA000C31A0C2193FBF1F201FB1232902303FB98
:104CB0000CF301FB023373449B6818447F2840F3D4
:104CC0002B857F3890FBF1F301FB13007330C0B2EA
:104CD00098F8001004F020FCBBF80020238813444F
:104CE000042B7FF769A85D4B1B88012B7FF464A818
:104CF0003A68A2F10C007F287FF7B7A88B3A0C2006
:104D000092FBF0F300FB13207330FFF750B8524CC6
:104D10002388002B40F0BC82DFF854B15049514A3F
:104D20000988D7F80080B2F800E04F48C1EB080CC2
:104D30000C229CFBF2F102FB11C14FF0900C0CFB1A
:104D40000EFE02FB01E16FF00B0E405880440EFB9B
:104D500003807F2840F31784A0F17F0393FBF2F0D8
:104D600002FB10307330414BC0B2197804F0D4FB11
:104D7000BBF8002023881344022B23DD384A394B2B
:104D800011883868B3F800C0DFF8DCE0411A0C2263
:104D900091FBF2F302FB1311902303FB0CF302FBD4
:104DA000013373445B6818447F2840F3FD847F38E7
:104DB00090FBF2F302FB130073302C4BC0B2197856
:104DC00004F0AAFBBBF8002023881344032B23DD47
:104DD000234A244B11883868B3F800C0DFF888E014
:104DE000411A0C2291FBF2F302FB1311902303FBF7
:104DF0000CF302FB013373449B6818447F2840F393
:104E000077847F3890FBF2F302FB13007330174B6B
:104E1000C0B2197804F080FBBBF80020238813444B
:104E2000042B7EF73EAA0D4B1B88012B7EF439AA7A
:104E30003A68A2F10C007F2840F356818B3A0C208F
:104E400092FBF0F300FB13207330084BC0B21978CB
:104E500004F062FBFEF725BA289DFF1FCA9CFF1FC6
:104E60009C9EFF1F4C9EFF1F00250100209DFF1FE1
:104E7000B09CFF1FCB4C2388002B40F0CC81DFF887
:104E800054B3C949C94A098899F80000B2F800E04A
:104E9000DFF84483C1EB000C0C229CFBF2F102FB17
:104EA00011C14FF0900C0CFB0EFE02FB01E16FF004
:104EB0000B0E58F8011008440EFB03007F2840F346
:104EC000A183A0F17F0393FBF2F002FB103073305B
:104ED000C0B204F045FBBBF8002023881344022B2A
:104EE00022DDB14AB14B118899F80000B3F800C037
:104EF000DFF8E4E2411A0C2291FBF2F302FB1311FA
:104F0000902303FB0CF302FB013373445B681844EA
:104F10007F2840F3F1837F3890FBF2F302FB13000C
:104F20007330C0B204F01CFBBBF80020238813448C
:104F3000032B22DD9C4A9D4B118899F80000B3F8A1
:104F400000C0DFF894E2411A0C2291FBF2F302FB5D
:104F50001311902303FB0CF302FB013373449B6892
:104F600018447F2840F3CE837F3890FBF2F302FB96
:104F700013007330C0B204F0F3FABBF800202388AA
:104F80001344042B7EF74AA8894B1B88012B7EF41F
:104F900045A899F80020A2F10C007F287EF762AFA7
:104FA0008B3A0C2092FBF0F300FB13207330FEF7DA
:104FB0007BBEDFF8F4A199F80000BAF800307D4C10
:104FC000C11A0C2291FBF2F302FB131302FB03F351
:104FD000E35818447F287FF772AD7F3890FBF2F3D7
:104FE00002FB130073302AE5FBF736FBD7E4FBF72F
:104FF00033FB72E4704B1A88182A13D03B681344B1
:10500000A3F118007F2840F3D3830C20973B93FB38
:10501000F0F200FB123303F17300684BC0B2197851
:1050200004F07AFA664B67491A78022A94BF013273
:1050300000221A701A7831F81200182810D10424AE
:10504000022A02F10100C2B288BF002231F8120028
:10505000182804D1013CF3D11A70FEF722B91A7056
:105060003B680344A3F118007F283DDD0C20973BEB
:1050700093FBF0F200FB123303F17300E5E6FBF75C
:10508000EBFAFFF7B0BB4C4B1B88182B12D099F8EA
:1050900000201344A3F118007F2840F341830C2023
:1050A000973B93FBF0F200FB123303F17300C0B2A5
:1050B00004F056FA424A434B127833F81230182B58
:1050C0003DF4ACAF99F800201344A3F118007F28F9
:1050D0007EF7C8AE0C20973B93FBF0F200FB123337
:1050E00003F17300FEF7E0BDFBF7B6FAADE6364B11
:1050F0001B78002B7DF4FBAF344B1B78002B3DF469
:1051000046ABB8F8003032490133A8F800300A70D5
:10511000FDF73DBB2C4B1B78002B7DF438AB2B4BA4
:105120001B78002B3DF433ABB8F800302849013B25
:10513000A8F800300A70FDF72ABB1F4A1288182A07
:1051400012D01344A3F118007F2840F3DE820C2014
:10515000973B93FBF0F200FB123303F17300C0B2F4
:1051600098F8001004F0D8F9154B16491A78022A5D
:1051700094BF013200221A701A7831F812001828F0
:105180002DD10424022A02F10100C2B288BF0022FC
:1051900031F81200182821D1013CF3D11A703B6874
:1051A000FEF776B9289DFF1F9C9EFF1F4C9EFF1F98
:1051B000CA9CFF1F042D0100B89CFF1F209DFF1FEC
:1051C0008C89FF1FB89EFF1F3B9FFF1F3C9FFF1F47
:1051D0009C9CFF1FB09CFF1F002501001A703B68BC
:1051E0000344A3F118007F287EF73FAE0C20973BC5
:1051F00093FBF0F200FB123303F17300FEF7D7BD0F
:10520000DFF82CA399F80000BAF80030BF4CD7E6BD
:10521000DFF82CB3E4E4BE4ADFF824B31288BBF80D
:105220000010033291427FF756AE2AE6B94A12883F
:10523000182A12D01344A3F118007F2840F3738278
:105240000C20973B93FBF0F200FB123303F1730049
:10525000C0B298F8001004F05FF9AF4BAF491A786C
:10526000022A94BF013200221A701A7831F8120013
:105270001828B4D10424022A02F1010294BFD2B248
:10528000002231F812001828A8D1013CF3D185E79B
:105290009F4ADFF8ACB21288BBF80010033291428B
:1052A0007FF766AD3AE59B4B1A88182A13D03B6806
:1052B0001344A3F118007F2840F30C820C20973B85
:1052C00093FBF0F200FB123303F17300944BC0B276
:1052D000197804F021F9904B90491A78022A94BF6A
:1052E000013200221A701A7831F8120018287FF45F
:1052F000B7AE0424022A02F1010294BFD2B2002206
:1053000031F8120018287FF4AAAE013CF2D11A70CD
:10531000FDF7C7BF7F4B1B88182B12D099F80020D0
:105320001344A3F118007F2840F3E9810C20973B38
:1053300093FBF0F200FB123303F17300C0B204F0F0
:105340000FF9754A754B127833F81230182B7FF429
:10535000B9AEFDF763BE734B01227F2107201A808F
:1053600004F0AAF87F210B2004F0A6F8FDF7EABEAE
:105370006D4B04227F2107201A8004F09DF8002144
:105380000B2004F099F8FDF7D6BE674B02227F216F
:1053900007201A8004F090F87F210B2004F08CF88D
:1053A000FDF7C4BE604B002107201C8004F084F888
:1053B0007F210B2004F080F8FDF7B3BE5B4C2388FF
:1053C000002B40F08A81DFF878B1594999F8000044
:1053D000584A09881788DFF860E1411A0C2291FBCE
:1053E000F2FC02FB1C114FF0900C0CFB07F702FBC8
:1053F00001716FF00B075EF80110014407FB031009
:105400007F2840F3D8817F3890FBF2F302FB130032
:105410007330C0B204F0A4F8BBF800202388134412
:10542000022B21DD424B434A99F800001B88B2F859
:1054300000E0414FC31A0C2193FBF1F201FB123241
:10544000902303FB0EF301FB02333B445B681844DB
:105450007F2840F3C8817F3890FBF1F301FB1300F4
:105460007330C0B204F07CF8BBF8002023881344EA
:10547000032B21DD2E4B2F4A99F800001B88B2F830
:1054800000E02D4FC31A0C2193FBF1F201FB123205
:10549000902303FB0EF301FB02333B449B6818444B
:1054A0007F2840F38B817F3890FBF1F301FB1300E1
:1054B0007330C0B204F054F8BBF8002023881344C2
:1054C000042B7EF7C4A9124B1B88012B7EF4BFA9C5
:1054D00099F80020A2F10C007F287FF798A88B3A5A
:1054E0000C2092FBF0F300FB13207330FFF781B820
:1054F000124B00227F2107201A8003F0DDFF7F215D
:105500000B2003F0D9FFFDF725BE00BFAC2B010037
:10551000CA9CFF1FC29CFF1F8C89FF1F2C9EFF1F70
:10552000209DFF1F3A9DFF1F929EFF1F289DFF1F7A
:105530009C9EFF1F4C9EFF1F00250100949CFF1F97
:10554000B09CFF1FAB4B1B88182B12D099F8002082
:105550001344A3F118007F2840F33C810C20973BB3
:1055600093FBF0F200FB123303F17300C0B203F0BF
:10557000F7FFA14AA14B127833F81230182B7FF4B1
:10558000A1ADFDF74BBDFBF767F8FFF7ECBB994BFF
:105590001A88182A13D03B681344A3F118007F28F7
:1055A00040F31B810C20973B93FBF0F200FB12337E
:1055B00003F17300924BC0B2197803F0ADFF8E4B2C
:1055C0008E491A78022A94BF013200221A701A7882
:1055D00031F8120018287FF443AD0424022A02F1A6
:1055E000010294BFD2B2002231F8120018287FF4D1
:1055F00036AD013CF2D11A70FDF753BEFBF72CF823
:10560000FFF711BBFBF728F862E47A4A1288182AE0
:1056100012D01344A3F118007F2840F3D2800C204D
:10562000973B93FBF0F200FB123303F17300C0B21F
:1056300098F8001003F070FF6F4B70491A78022A37
:1056400094BF013200221A701A7831F8120018281B
:105650007FF4C5AD0424022A02F1010294BFD2B244
:10566000002231F8120018287FF4B8AD013CF2D1C5
:1056700094E5644B1B88182B12D099F80020134432
:10568000A3F118007F2840F3AB800C20973B93FBDD
:10569000F0F200FB123303F17300C0B203F060FFBD
:1056A000554A594B127833F81230182B3EF4CFA8D4
:1056B00099F800201344A3F118007F287EF7A7AFC4
:1056C0000C20973B93FBF0F200FB123303F17300C5
:1056D000FEF78FBFFAF7C0FFF8E54C4ADFF83CB1A0
:1056E0001288BBF80010033291427FF795AE6CE64A
:1056F000FAF7B2FFFFF78BBBFAF7AEFF11E4FAF748
:10570000ABFF1BE6FAF7A8FF34E4FAF7A5FF26E59E
:10571000FAF7A2FFFFF7B1BAFAF79EFFFFF7D7BA81
:10572000FAF79AFFC3E4FAF797FF91E5314B1B882C
:10573000182B11D099F800201344A3F118007F28EA
:1057400042DD0C20973B93FBF0F200FB123303F198
:105750007300C0B203F004FF274A284B127833F8D5
:105760001230182BA4D1FEF772B8294B1B88182BC6
:1057700011D099F800201344A3F118007F2826DDEA
:105780000C20973B93FBF0F200FB123303F1730004
:10579000C0B203F0E5FE184A1E4B127833F81230FF
:1057A000182B85D1FEF753B8FAF756FFFFF705BB64
:1057B000FAF752FF31E4FAF74FFF2AE6FAF74CFF07
:1057C00077E6FAF749FF32E7FAF746FFC1E7FAF75B
:1057D00043FFDDE7FAF740FFC8E6FAF73DFFE9E6E9
:1057E000FAF73AFF59E7FAF737FF3AE60A4B02931E
:1057F000FDF705BFC49CFF1F8C89FF1F349EFF1F50
:10580000209DFF1FB89CFF1FB89EFF1FCA9CFF1F53
:10581000C29CFF1F2C9EFF1F469DFF1FB09CFF1FB9
:1058200038B507F071FE0B4805F0A8FD00234FF0D6
:105830007E5201210848FAF719FE084B084A094927
:10584000802400251C7118461D60BDE838400BF00F
:1058500061BC00BF389DFF1F709EFF1FFC9EFF1F95
:105860001C89FF1FFD05000010B50446A4206368D5
:10587000198803F07BFFE368A6201988BDE8104073
:1058800003F074BF43682A20198803F06FBF00BF7C
:1058900010B5044622206368198803F067FFE368A7
:1058A00024201988BDE8104003F060BF10B50446FD
:1058B0000A206368198803F059FFE3680C201988EF
:1058C000BDE8104003F052BF10B5044606206368DF
:1058D000198803F04BFFE36808201988BDE81040E1
:1058E00003F044BF10B5044602206368198803F032
:1058F0003DFFE36804201988BDE8104003F036BF7F
:1059000070B50E4C84B01225042201230646039084
:10591000029320468DE824001423102106F032FF64
:105920000622092302930396019520460092142330
:10593000102106F027FF04B070BD00BF709FFF1F4D
:1059400070B5AE4CB4F90030032B00F0E880002BAA
:105950004DD0022B6CD0052B00F09880012B00F06D
:10596000C080042B00D070BD00244FF4AF75E1B2AD
:10597000A34805F06BFD01348542A8BF05460C2CF9
:10598000F5D1012008F040FE0446002008F03CFE5E
:10599000323CA0F132039B496FF4957000FB03F396
:1059A00000FB04F081FB034281FB0041DB17C017C1
:1059B000C3EB6223C0EB612003F5AF7200F5AF7358
:1059C0009342A8BF13469D42A8BF1D46A5F11401EE
:1059D000312900F3E28040F26C7332218A488B4A0D
:1059E0000180BDE870402A20136003F0BFBE0E2086
:1059F00007F0EEFC40F6FF71C8308842A8BF0846A9
:105A000020EAE07000F2DC5283B28A42804D814E7F
:105A1000A8BF0A460220194633802A8003F0A6FE5A
:105A20002988042003F0A2FEB4F90030022B92D1A1
:105A3000172008F0E9FD0546162008F0E5FDA8420C
:105A4000B8BF284600F1C801B1F5FA7FC0F2BF80A7
:105A5000B1F57A6FA8BF4FF47A6101F54873B3F5D9
:105A60007A6FA8BF4FF47A639BB289B26A4A6B4DD2
:105A700011800A202B8003F079FE29880C2003F086
:105A800075FEB4F90030052B7FF468AF0F2008F0E5
:105A9000BBFDC0F53F630433B3F5AF6FC0F28F8039
:105AA000B3F5FA6FA8BF4FF4FA6399B25C4BC0F537
:105AB0004360B0F5AF6F19807EDBB0F5FA6FA8BF19
:105AC0004FF4FA6083B2574DA4202B8003F04EFEB2
:105AD0002988A62003F04AFEB4F90030012B7FF498
:105AE00040AF0B2008F090F900283CD0112008F0BE
:105AF0008BFD00F1C801B1F52F7F3CDB41F25C2347
:105B0000994278DC484A00F5487089B2B0F52F7F99
:105B100011806DDB8342A8BF03469BB231E01020A9
:105B200008F072FDC830B0F5FA7F4BDBB0F57A6F44
:105B30000146A8BF4FF47A6101F51673B3F57A6F89
:105B4000A8BF4FF47A639BB289B2384A384D1180AE
:105B500022202B8003F00AFE2988242003F006FE71
:105B6000B4F90030F3E6152007F032FC00F5967129
:105B7000B1F52F7F30DA40F214534FF42F712A4AD7
:105B800011802C4D06202B8003F0F0FD2988082081
:105B900003F0ECFDB4F90030E3E640F23A72A5F50B
:105BA000B975254B02FB05F583FB0523ED17A5EB26
:105BB000631389B2323311E74FF4AF6383E74FF4D5
:105BC000AF6173E740F24C434FF4FA71BDE740F226
:105BD00014534FF4FA7149E741F25C2399420ADC0D
:105BE000114A00F5617089B2B0F52F7F118091DA0A
:105BF0004FF42F73C5E71946C1E700BF489FFF1F49
:105C0000389DFF1F67BBCF46069FFF1F9889FF1F68
:105C10000E9FFF1F449DFF1FA89EFF1FC09CFF1FDC
:105C2000489DFF1FC89EFF1FFE9CFF1F569EFF1F23
:105C3000529EFF1FDC9EFF1FB5814E1B2DE9F041D8
:105C4000224D82B0012602B284B20092284601960B
:105C50007823192106F0DCFC04F10C0212B28DE865
:105C600044002846A7197823192104F1020806F0F8
:105C7000CFFC3FB20FFA88F819233A462846194656
:105C80000196CDF8008006F0C3FC78233A462846FA
:105C90001946CDF80080019604F10A070B3406F08E
:105CA000B7FC3FB224B278233A46284619468DE81D
:105CB000500006F0ADFC192300943A4601962846A0
:105CC000194606F0A5FC02B0BDE8F081709FFF1FE9
:105CD00030B583B000230C4605B2009326225B2327
:105CE0001C210C4806F0E4F9294601232622094824
:105CF00005F0EEFC002C24B205DB21460123262210
:105D0000044805F0E5FC044A044B15801C8003B0F0
:105D100030BD00BF709FFF1FAE89FF1FB089FF1FFE
:105D200070B5A54C237882B01BB1A44B4FF6FF721F
:105D30001A80A34BB3F90030C3B9A24A9F4B106835
:105D4000B3F9002080F30C005B2303FB00F0001389
:105D50001C3082424AD04FF0FF31FFF7B9FF9A481A
:105D600006F00AFA0023237002B070BD012B1BD08D
:105D7000022B5AD0032B3FD0042B00F09A80052B26
:105D8000F0D10F2008F040FCC0F53B600830B0F5C2
:105D9000AF6F48DBB0F5FA6FA8BF4FF4FA60A0F51B
:105DA000AF625B23894835E0894B1B78002B70D0AC
:105DB000152007F00DFB874B1860B0F52F7F32DB05
:105DC00041F25C239842A8BF1846A0F52F735B22CE
:105DD000814802FB03F380FB0320DB17C3EBA02009
:105DE0001C30764BB3F900308342B4D17B4BB3F90E
:105DF00000300133AFD1B5E7794B1B68B3F5FA7FBB
:105E000011DBB3F57A6FA8BF4FF47A637548A3F539
:105E1000FA725B2303FB02F380FB0320DB17C3EB67
:105E200020201C30DDE71C20DBE76F4B1B68B3F53F
:105E3000FA7F36DBB3F57A6FA8BF4FF47A63A3F528
:105E4000FA7268485B2303FB02F380FB0320DB1735
:105E5000C3EB20201C30654B1B68B3F5FA7F1EDBBB
:105E6000B3F57A6FA8BF4FF47A63A3F5FA725D4970
:105E70005B2303FB02F381FB0321DB17C3EB21212F
:105E80001C314E4BB3F9003083420CD0FFF720FF9A
:105E900065E7112008F0B8FB4E4B18608DE71C2118
:105EA000EFE71C20D7E74D4BB3F900308B42EDD123
:105EB00058E7272200258DE8240076231C2142483C
:105EC0004B4E06F0A5FB16E0B0F5AF7FA8BF4FF430
:105ED000AF70323803FB00F386FB0321DB17C3EB03
:105EE00061111C3109B201231D442722364805F0F7
:105EF000EFFB0C2D09D0E9B23E4805F0A7FA312896
:105F00004FF05B03E0DC1C21EDE7012008F07CFB97
:105F10006FF495733238384A03FB00F082FB00239C
:105F2000C017C0EB632303F5AF73312B42DDB3F52C
:105F3000AF7FA8BF4FF4AF735B22323B2C4D02FB07
:105F400003F385FB0325DB17C3EB65151C35002028
:105F500008F05AFB6FF495733238274A03FB00F0C0
:105F600082FB0023C017C0EB632303F5AF73312B13
:105F70001EDDB3F5AF7FA8BF4FF4AF735B22323B9A
:105F80001B4902FB03F381FB0321DB17C3EB611108
:105F90001C310A4BB3F90030AB4201D0284675E7FB
:105FA0000E4BB3F900308B423FF4D9AE28466DE773
:105FB0001C21EEE71C25CAE7429FFF1FAE89FF1F89
:105FC000489FFF1FAC9EFF1F709FFF1F37800B6D08
:105FD000C29EFF1F809CFF1FD3058541B089FF1F14
:105FE000D09CFF1F011FB812E09CFF1FA49CFF1F45
:105FF0004B48371B389DFF1F67BBCF462DE9F0414B
:10600000044682B071482768E56805F0A9FF1120B1
:10601000FFF714FE012619234FF028081946242201
:106020006A480196CDF8008006F0F2FA7823194606
:10603000242266480196CDF8008006F0E9FA314640
:10604000624806F07BFE02221921604806F072FECB
:1060500038460BF035FE394602465C4807F004F836
:106060005A4807F017F814220021584806F062FE3B
:1060700003225749554806F0F7FF544807F00AF83D
:1060800023220021514806F055FE032251494F4872
:1060900006F0EAFF4D4806F0FDFF7DB12F20FFF727
:1060A000CDFD32220021494806F044FE03224A4930
:1060B000464806F0D9FF454806F0ECFF0123474A61
:1060C00018461370FFF71CFC2189638962685B1A0C
:1060D0005C2B128854DD521A02EB4202C2EB4212D0
:1060E000013392FBF3F31B333D4A384813800126FA
:1060F0001A221BB28DE844001946142206F088FAD1
:10610000002D4FD0218A638AE2685B1A5C2B1288CB
:106110003EDC511A5C2202FB01F292FBF3F31B33CB
:10612000304A2A48138001251BB2382219468DE8CF
:106130002400322206F06CFA4023002209218DE867
:1061400006002248194606F031FA29461F4806F093
:10615000F5FD022244211D4806F0ECFD63681B4852
:10616000198806F0E7FF2A461F49184806F07CFF09
:10617000E3681648198802B0BDE8F04106F0DABFBE
:10618000511A5C2202FB01F292FBF3F31B33ABE7E3
:10619000521A02EB4202C2EB4212334492FBF3F377
:1061A0001B33BDE7402309212A460091074801958A
:1061B000194606F0FBF93146044806F0BFFD0222FD
:1061C0006821024806F0B6FD6368D2E7709FFF1FA2
:1061D000DC2D0100E02D0100E42D0100E99FFF1FEF
:1061E000449FFF1F469FFF1FE82D01002DE9F04748
:1061F0001F4682B01446002A4ED0052A0646D0F823
:106200000C8000F0AB800B9B894A00EBC305012C8E
:10621000B5F80AE029896868C1EB0E0382FB03C266
:106220001A444FEAE373C3EBA213028851D0042C43
:1062300000F08D800022402309218DE806007D4872
:10624000194606F0B3F901217A4806F077FD0222DB
:10625000B8F1000F00F0E1804421764806F06AFDB5
:1062600073687448198806F065FF73497148012204
:1062700006F0FAFEF3686F48198806F05BFF6F4B73
:10628000022CB3F9001000F0A680082C00F0C280A8
:10629000012002B0BDE8F087694E6A4A336812688F
:1062A000CB1A93420D4655D9674A3B88117861480D
:1062B000012918BF012414700A9A06321BB212B2C7
:1062C0008DE814001946BDF9282006F0A1F93560C3
:1062D000DEE79BB2D31A994203DC9E457146A8BF04
:1062E00019460A9A0180B7F90030BDF928A0514833
:1062F00002F106094FF0000E0FFA89F919465246CD
:10630000CDF80090CDF804E006F082F929896A8979
:106310006868521A03885C2AA3EB010373DD03EB60
:1063200043030132C3EB431393FBF2F303F11B026C
:1063300013B201203A80194652460190CDF80090E0
:106340003C4806F065F9404B00221A7072E712FAD9
:1063500083F3C0E7204602B0BDE8F08707254FF081
:1063600000095A2323228DE820021A21314806F021
:106370001DF901212F4806F0E1FC01212D4806F00E
:10638000E3FC232235212B4806F0D4FC2A462F4972
:10639000284806F069FE274806F07CFE254805F0EF
:1063A000EBFE4FF4FA6007F065FDFFF7C9FA5A23D8
:1063B00023221A218DE820021E4806F0F7F81D4816
:1063C00005F0DAFE3046FFF719FE214B01221A7064
:1063D000FFF7A6FC2EE74A1C12B21A8091423FF446
:1063E00057AF0A9AB7F9003012480632012412B2A8
:1063F000009219460194BDF9282006F009F92046BB
:1064000002B0BDE8F0875C2101FB03F393FBF2F2DD
:106410001B328DE700221A80E0E76821054806F06C
:1064200089FC73680348198806F084FE27E700BFDB
:10643000C94216B2709FFF1FE82D01004C9FFF1F3D
:10644000D49FFF1FE43D0100E99FFF1FEC2D0100D9
:10645000429FFF1F2DE9F04F5A4E5B4DB6F9007079
:106460004C7855F8277085B08146984604B10C7871
:10647000DFF874A11AB99AF80030002B39D0534DC7
:10648000002338462B808AF80030FFF7B7FD504ACA
:10649000504BB5F90000012111704FF6FF721A80C0
:1064A00060B301285ED00120322322460190009380
:1064B0004946494B3846FFF799FE00240346B5F993
:1064C0000020022A39DD00222A80B6F900203D4949
:1064D000002A3BDB052AC4BF00220A80B8F1000F66
:1064E00039D1002C0CBF18464FF0FF3005B0BDE885
:1064F000F08F364DB5F900000028D2D1DFF8ECB0AE
:10650000364ADBF800301268C3EB0903934227D9FF
:10651000334B1A78012A18BF01201870FFF7F0F9E1
:106520000123CBF80090012C2AD0042C35D0022C6A
:106530003AD0082C3ED00024C1E7C6D1FA68002A20
:10654000C1D0B6F900201F49002AC3DA05220A800B
:10655000B8F1000FC5D00393FFF7E2FB039BC0E740
:106560000346E0E74FF0000E142322468DE8084072
:1065700049461C4B38467446FFF738FE03469EE7F3
:1065800032888AF80040013232807A6982B1002470
:10659000384603939047039B91E732880121013AE3
:1065A00032808AF80010F0E701222A8000248CE76C
:1065B000144684E77A69002129804FF0FF34002ACD
:1065C000E6D182E7489FFF1FB489FF1F4C9FFF1F42
:1065D000429FFF1FAE89FF1F469FFF1FE43D010042
:1065E000E99FFF1F449FFF1F4A9FFF1FD49FFF1F6C
:1065F00001210D2007F002BC00210D2007F0FEBB99
:1066000001460D2007F0FABB08B50D2007F0FCFB92
:10661000B0FA80F149090D20BDE8084007F0EEBB53
:1066200010B5002144080D2007F0E8FB204607F0D4
:1066300021FC0D20012107F0E1FB2046BDE81040C0
:1066400007F018BC214A224B10881B68984210B5ED
:1066500035DA204A1288141A9A42A8BF1A46B4F5AD
:10666000157F22DA121A40F2532303FB02F393FB45
:10667000F4F105310A2007F031FA174B197801B30C
:10668000164B17491B6840F2271283F3070302FBDE
:1066900003F381FB03211944DB17C3EBA11105317F
:1066A0000920BDE8104007F019BA131A4FF415720B
:1066B000611C02FB03F393FBF1F10531DAE70021E2
:1066C000D8E70920BDE8104007F008BA449DFF1F35
:1066D000789CFF1F0E9FFF1F009DFF1FF49EFF1F52
:1066E000090402817F2838B5A8BF7F200F4C4FF4E2
:1066F000167202FB00F284FB02311144D2170546E8
:10670000C2EBA1110A2007F0E9F97F3D4FF496731F
:1067100003FB05F384FB03211944DB17A3EBA11151
:106720000920BDE8384007F0D9B900BF090402814B
:10673000C368B3F9003030B583EAE374A4EBE374C3
:10674000002BA0B218DB012300E0134603EB830209
:1067500052009442F9DA0A4D90FBF3F285FB03E410
:1067600003FB1200DB173032D3EBA40380B201F835
:10677000012BF1D10B7030BD2D230B700131E2E7FD
:106780006766666638B5094D8224204603F008F82E
:1067900035F8021B00B28842204601D002F0E6FF25
:1067A0000234A4B28A2CF0D138BD00BF349EFF1F42
:1067B000024B8020198802F0D9BF00BFC49CFF1F84
:1067C00038B5094D7824204602F0EAFF35F8021B5F
:1067D00000B28842204601D002F0C8FF0234A4B2C1
:1067E000802CF0D138BD00BF2C9EFF1F024B7620BD
:1067F000198802F0BBBF00BFC29CFF1F38B5094D0E
:106800004624204602F0CCFF35F8021B00B2884235
:10681000204601D002F0AAFF0234A4B24E2CF0D1DF
:1068200038BD00BFB89EFF1F024B4420198802F0FC
:106830009DBF00BFB89CFF1F024B4E20198802F07D
:1068400095BF00BFDC9CFF1F024B9A20198802F005
:106850008DBF00BF289DFF1F024B9820198802F0B2
:1068600085BF00BFCA9CFF1F024B8C20198802F015
:106870007DBF00BF4C9EFF1F024B9C20198802F079
:1068800075BF00BFB09CFF1F024BA020198802F00B
:106890006DBF00BFC09EFF1F024B9620198802F0FB
:1068A00065BF00BF9C9EFF1F024B8A20198802F023
:1068B0005DBF00BF5C9EFF1F024B1020198802F0D5
:1068C00055BF00BF5A9EFF1F024B2C20198802F0B3
:1068D0004DBF00BFAE9CFF1F024B1E20198802F067
:1068E00045BF00BFC89CFF1FC3680E20198802F077
:1068F0003DBF00BF024B2820198802F037BF00BF00
:10690000B69EFF1F024B6220198802F02FBF00BF06
:10691000EC9CFF1F024B6420198802F027BF00BFC8
:10692000B09EFF1F024BB420198802F01FBF00BFAA
:10693000049FFF1F024BB620198802F017BF00BF4B
:10694000309FFF1F024B5A20198802F00FBF00BF73
:10695000889CFF1F024B1620198802F007BF00BF5A
:10696000949CFF1F024B2E20198802F0FFBE00BF2F
:10697000309DFF1F024B3020198802F0F7BE00BF88
:106980001C9FFF1F024B9E20198802F0EFBE00BF24
:106990009489FF1F024BAC20198802F0E7BE00BFAC
:1069A000B29EFF1F024BAE20198802F0DFBE00BF6F
:1069B000D49CFF1F024BB020198802F0D7BE00BF45
:1069C000409EFF1F024BB220198802F0CFBE00BFCD
:1069D000F69CFF1F024B1820198802F0C7BE00BFAB
:1069E0004A9DFF1F024BA220198802F0BFBE00BFC4
:1069F000E29EFF1F024B1A20198802F0B7BE00BFAB
:106A0000E49CFF1F024B1C20198802F0AFBE00BFA0
:106A1000DE9CFF1F024B6620198802F0A7BE00BF54
:106A2000F09EFF1F024B7220198802F09FBE00BF2C
:106A3000189FFF1F024B2020198802F097BE00BF4D
:106A4000EE9EFF1F024B3220198802F08FBE00BF5E
:106A5000DE9EFF1F024B6820198802F087BE00BF30
:106A60001C9DFF1F024B6C20198802F07FBE00BFE7
:106A70007C9CFF1F024B5220198802F077BE00BF9A
:106A80002E89FF1F024B5020198802F06FBE00BFF5
:106A90002089FF1F024B5420198802F067BE00BFF7
:106AA000A889FF1F024B5C20198802F05FBE00BF5F
:106AB000AC89FF1F024B5E20198802F057BE00BF51
:106AC0002C89FF1F024B5620198802F04FBE00BFD1
:106AD0001E9DFF1F244B1B880B2B43D8DFE803F0C0
:106AE0000B10151A1F24292E33383D0608460422A0
:106AF0001E490BF0A3B9084604221D490BF09EB9AC
:106B0000084604221B490BF099B9084604221A4989
:106B10000BF094B90846042218490BF08FB90846C7
:106B2000042217490BF08AB90846042215490BF0D4
:106B300085B90846042214490BF080B9084604229E
:106B400012490BF07BB90846042211490BF076B9C3
:106B5000084604220F490BF071B9084604220E4979
:106B60000BF06CB9704700BF9C9EFF1F48360100B8
:106B7000B43301001C32010034370100203201001F
:106B80001C3701002432010028320100DC340100EE
:106B90002C3201005436010030320100064B074A06
:106BA00010B41C88064B0846002C14BF1146194629
:106BB000042210BC0BF042B9FC9CFF1F34320100D0
:106BC00038320100064B074A10B41C88064B0846B1
:106BD000002C14BF11461946042210BC0BF02EB92C
:106BE000329DFF1F3432010038320100064B074A44
:106BF00010B41C88064B0846002C14BF11461946D9
:106C0000042210BC0BF01AB9509EFF1F3432010051
:106C100038320100064B074A10B41C88064B084660
:106C2000002C14BF11461946042210BC0BF006B903
:106C3000649EFF1F3432010038320100064B074AC0
:106C400010B41C88064B0846002C14BF1146194688
:106C5000042210BC0BF0F2B89E9EFF1F34320100DC
:106C600038320100064B074A10B41C88064B084610
:106C7000002C14BF11461946042210BC0BF0DEB8DC
:106C80003A9DFF1F34320100383201001B4B1B8834
:106C90000A2B0AD8DFE803F00A0E12161A1E222663
:106CA0002A2E0600164B186808607047154B1868A6
:106CB00008607047144B186808607047134B1868D9
:106CC00008607047124B186808607047114B1868CD
:106CD00008607047104B1868086070470F4B1868C1
:106CE000086070470E4B1868086070470D4B1868B5
:106CF000086070470C4B1868086070475C9EFF1F67
:106D000060320100383201003C32010040320100A3
:106D100044320100483201004C320100503201007F
:106D200054320100583201005C320100F0B52B4EA4
:106D30002B4FDFF8C4E005460FCE87B06C460FC47A
:106D400096E803003B68274A274F44F8040B40F6B7
:106D5000CC308342C8BF3A46BEF800602180012E85
:106D600011889278ADF80D108DF80F202AD032D30B
:106D700040F6CA02022E18BF00229A4226DAA3F673
:106D800098031A491A4AC3EB031381FB0301194400
:106D9000DB17C3EB6123243382FB0321DA17C2EB39
:106DA000A10202EB8201A3EB4103303330328DF8B4
:106DB00013308DF811206946284616220BF03EF854
:106DC00007B0F0BD40F698029A42D8DB094B18682C
:106DD000CDF81100EFE740F6FC02CEE77432010077
:106DE000A49EFF1F68320100643201003B773B988C
:106DF000676666666C3201003C9EFF1FF8B5174C53
:106E0000174E2278174D33782F888E46003218BFE0
:106E1000012201467046FFF71DFB002398423370A4
:106E2000237015DB14BF012000202B889F420ED059
:106E300040F23A72A3F5AF730B490C4C02FB03F31B
:106E400081FB0312DB17A3EB621332332360F8BD1F
:106E50000749012218460A702270E6E7808AFF1F60
:106E60005D9FFF1F069FFF1FB5814E1B9889FF1F67
:106E7000E89FFF1F014B187802F010BCD09FFF1F46
:106E8000014B187802F024BC8890FF1F134BB3F914
:106E9000003030B583EAE374A4EBE374002BA0B2B6
:106EA00018DB012300E0134603EB830252009442F7
:106EB000F9DA0B4D90FBF3F285FB03E403FB1200C0
:106EC000DB173032D3EBA40380B201F8012BF1D1F0
:106ED0000B7030BD2D230B700131E2E78890FF1F4E
:106EE00067666666144BB3F9003070B583EAE375E4
:106EF000A5EBE375002BACB21ADB012300E00346DF
:106F000003EB830040008542F9DA0C4E94FBF3F06A
:106F100086FB03E503FB1044DB173030D3EBA503FE
:106F2000A4B201F8010BF1D105480B70106070BDDF
:106F30002D230B700131E0E7889CFF1F67666666B2
:106F40008C320100134BB3F9003030B583EAE3749F
:106F5000A4EBE374002BA0B218DB012300E013467E
:106F600003EB830252009442F9DA0B4D90FBF3F2EB
:106F700085FB03E403FB1200DB173032D3EBA403E1
:106F800080B201F8012BF1D10B7030BD2D230B70B5
:106F90000131E2E79489FF1F67666666134BB3F918
:106FA000003030B583EAE374A4EBE374002BA0B2A5
:106FB00018DB012300E0134603EB830252009442E6
:106FC000F9DA0B4D90FBF3F285FB03E403FB1200AF
:106FD000DB173032D3EBA40380B201F8012BF1D1DF
:106FE0000B7030BD2D230B700131E2E7D49CFF1FE5
:106FF00067666666134BB3F9003030B583EAE37415
:10700000A4EBE374002BA0B218DB012300E01346CD
:1070100003EB830252009442F9DA0B4D90FBF3F23A
:1070200085FB03E403FB1200DB173032D3EBA40330
:1070300080B201F8012BF1D10B7030BD2D230B7004
:107040000131E2E7F69CFF1F67666666134BB3F9F2
:10705000003030B583EAE374A4EBE374002BA0B2F4
:1070600018DB012300E0134603EB83025200944235
:10707000F9DA0B4D90FBF3F285FB03E403FB1200FE
:10708000DB173032D3EBA40380B201F8012BF1D12E
:107090000B7030BD2D230B700131E2E7E29EFF1F24
:1070A00067666666134BB3F9003030B583EAE37464
:1070B000A4EBE374002BA0B218DB012300E013461D
:1070C00003EB830252009442F9DA0B4D90FBF3F28A
:1070D00085FB03E403FB1200DB173032D3EBA40380
:1070E00080B201F8012BF1D10B7030BD2D230B7054
:1070F0000131E2E72E89FF1F67666666134BB3F91D
:10710000003030B583EAE374A4EBE374002BA0B243
:1071100018DB012300E0134603EB83025200944284
:10712000F9DA0B4D90FBF3F285FB03E403FB12004D
:10713000DB173032D3EBA40380B201F8012BF1D17D
:107140000B7030BD2D230B700131E2E72089FF1F4A
:1071500067666666134BB3F9003030B583EAE374B3
:10716000A4EBE374002BA0B218DB012300E013466C
:1071700003EB830252009442F9DA0B4D90FBF3F2D9
:1071800085FB03E403FB1200DB173032D3EBA403CF
:1071900080B201F8012BF1D10B7030BD2D230B70A3
:1071A0000131E2E7A889FF1F67666666134BB3F9F2
:1071B000003030B583EAE374A4EBE374002BA0B293
:1071C00018DB012300E0134603EB830252009442D4
:1071D000F9DA0B4D90FBF3F285FB03E403FB12009D
:1071E000DB173032D3EBA40380B201F8012BF1D1CD
:1071F0000B7030BD2D230B700131E2E7AC89FF1F0E
:1072000067666666134BB3F9003030B583EAE37402
:10721000A4EBE374002BA0B218DB012300E01346BB
:1072200003EB830252009442F9DA0B4D90FBF3F228
:1072300085FB03E403FB1200DB173032D3EBA4031E
:1072400080B201F8012BF1D10B7030BD2D230B70F2
:107250000131E2E72C89FF1F6766666608B5B82032
:1072600002F09EFA044B1988884204D0B820BDE889
:10727000084002F07BBA08BD909CFF1F08B5702043
:1072800002F08EFA044B1988884204D07020BDE8C1
:10729000084002F06BBA08BD3C9EFF1F08B5742081
:1072A00002F07EFA044B1988884204D07420BDE8AD
:1072B000084002F05BBA08BDD49EFF1F054B1B8837
:1072C0000846042213B904490AF0B8BD03490AF07C
:1072D000B5BD00BFDC9CFF1F94320100903201005D
:1072E0000E4B1B88032B17D8DFE803F0110C0702A5
:1072F000084604220A490AF0A1BD084604220949A9
:107300000AF09CBD0846042207490AF097BD0846CA
:10731000042206490AF092BD704700BF4C9EFF1F31
:10732000A0320100383301009C3201009832010084
:1073300010B40A4B0A4C0A4693E8030083B0238832
:1073400002AC04E9030004EB8303104653F8081C65
:10735000052203B010BC0AF071BD00BF6C2E010005
:10736000B09EFF1F30B40A4B0A4D0C4693E807004D
:1073700084B02B8804AD05E9070005EB83032046A4
:1073800053F80C1C042204B030BC0AF057BD00BFF7
:10739000742E01003C9EFF1FF0B40C4D0C4F0E46A6
:1073A0000FCD8CB001AC0FC40FCD0FC495E8070012
:1073B0003B8884E807000CAA02EB8303304653F8AD
:1073C0002C1C04220CB0F0BC0AF038BD802E010049
:1073D000929EFF1F30B50A4B0A4D0C460FCB85B06D
:1073E0000DF1100E0EE90F002B880EEB83032046E3
:1073F00053F8101C042205B0BDE830400AF01EBD51
:10740000BC2E0100B29EFF1F30B50A4B0A4D0C4640
:107410000FCB85B00DF1100E0EE90F002B880EEB8F
:107420008303204653F8101C042205B0BDE8304009
:107430000AF004BDBC2E0100409EFF1FF0B40B4DAE
:107440000B4F0E460FCD86B06C460FC495E8030077
:107450003B8884E8030006AA02EB8303304653F816
:10746000181C042206B0F0BC0AF0E8BCCC2E0100C7
:107470004A9DFF1FF0B40A4D0A4F0E460FCD86B04D
:1074800001AC0FC42A683B88226006AA02EB830382
:10749000304653F8141C0C2206B0F0BC0AF0CEBCE7
:1074A000E42E0100DE9CFF1FF0B40B4D0B4F0E4687
:1074B0000FCD86B06C460FC495E803003B8884E886
:1074C000030006AA02EB8303304653F8181C04227B
:1074D00006B0F0BC0AF0B2BCF82E0100D49EFF1F2B
:1074E000164B1B880BB31BB283EAE370A0EBE3706F
:1074F000002B30B584B21DDB012300E0134603EB03
:10750000830252009042F9DA0D4894FBF3F280FBBB
:1075100003E503FB1244DB173032D3EBA503A4B21F
:1075200001F8012BF1D10B7030BD0846042205494A
:107530000AF084BC2D230B700131DDE71C9DFF1F79
:1075400067666666A432010030B50A4B0A4D0C46E8
:107550000FCB85B00DF1100E0EE90F002B880EEB4E
:107560008303204653F8101C042205B0BDE83040C8
:107570000AF064BC102F01007C9CFF1F054B1B8888
:107580001BB9054B18680860704708460422034978
:107590000AF054BC289DFF1F38320100343201002C
:1075A000164B1B880BB31BB230B583EAE374A4EB14
:1075B000E374002BA0B21CDB012300E0134603EBB5
:1075C000830252009442F9DA0D4D90FBF3F285FBF1
:1075D00003E403FB1200DB173032D3EBA40380B2C9
:1075E00001F8012BF1D10B7030BD064B1868086013
:1075F00070472D230B700131DEE700BFC89CFF1FD1
:107600006766666638320100164B1B880BB31BB2E7
:1076100030B583EAE374A4EBE374002BA0B21CDB67
:10762000012300E0134603EB830252009442F9DA8F
:107630000D4D90FBF3F285FB03E403FB1200DB1717
:107640003032D3EBA40380B201F8012BF1D10B70DF
:1076500030BD064B1868086070472D230B70013150
:10766000DEE700BF909CFF1F676666663832010048
:10767000164B1B880BB31BB230B583EAE374A4EB43
:10768000E374002BA0B21CDB012300E0134603EBE4
:10769000830252009442F9DA0D4D90FBF3F285FB20
:1076A00003E403FB1200DB173032D3EBA40380B2F8
:1076B00001F8012BF1D10B7030BD064B1868086042
:1076C00070472D230B700131DEE700BFA29EFF1F24
:1076D0006766666638320100164B1B880BB31BB217
:1076E00030B583EAE374A4EBE374002BA0B21CDB97
:1076F000012300E0134603EB830252009442F9DABF
:107700000D4D90FBF3F285FB03E403FB1200DB1746
:107710003032D3EBA40380B201F8012BF1D10B700E
:1077200030BD064B1868086070472D230B7001317F
:10773000DEE700BF949CFF1F67666666A832010003
:10774000174B1B881BB31BB270B583EAE375A5EB1F
:10775000E375002BACB21EDB012300E0034603EB14
:10776000830040008542F9DA0E4E94FBF3F086FB6D
:1077700003E503FB1044DB173030D3EBA503A4B2C1
:1077800001F8010BF1D108480B70106070BD074B78
:107790001868086070472D230B700131DCE700BFCB
:1077A000309DFF1F67666666AC320100383201000B
:1077B000164B1B880BB31BB230B583EAE374A4EB02
:1077C000E374002BA0B21CDB012300E0134603EBA3
:1077D000830252009442F9DA0D4D90FBF3F285FBDF
:1077E00003E403FB1200DB173032D3EBA40380B2B7
:1077F00001F8012BF1D10B7030BD064B1868086001
:1078000070472D230B700131DEE700BF1C9FFF1F67
:107810006766666638320100164B1B880BB31BB2D5
:1078200030B583EAE374A4EBE374002BA0B21CDB55
:10783000012300E0134603EB830252009442F9DA7D
:107840000D4D90FBF3F285FB03E403FB1200DB1705
:107850003032D3EBA40380B201F8012BF1D10B70CD
:1078600030BD064B1868086070472D230B7001313E
:10787000DEE700BFF09EFF1F6766666638320100D4
:10788000164B1B880BB31BB230B583EAE374A4EB31
:10789000E374002BA0B21CDB012300E0134603EBD2
:1078A000830252009442F9DA0D4D90FBF3F285FB0E
:1078B00003E403FB1200DB173032D3EBA40380B2E6
:1078C00001F8012BF1D10B7030BD064B1868086030
:1078D00070472D230B700131DEE700BF189FFF1F9B
:1078E0006766666638320100174B1B881BB31BB2F4
:1078F00070B583EAE375A5EBE375002BACB21EDB34
:10790000012300E0034603EB830040008542F9DADF
:107910000E4E94FBF3F086FB03E503FB1044DB17EC
:107920003030D3EBA503A4B201F8010BF1D1084824
:107930000B70106070BD074B1868086070472D23EE
:107940000B700131DCE700BFEE9EFF1F67666666C5
:10795000AC32010038320100054B1B881BB1054BCE
:10796000186808607047044B18680860704700BFCB
:107970001E9DFF1FC0320100BC32010070B5FAF736
:107980004DFB164B1B7813B1154C237833B9154BAF
:107990001020198801F0EAFE012070BD124D134E2F
:1079A0002B783288B3FA83F382F008025B09114620
:1079B00042202B70328001F0D9FE23780BB12B7856
:1079C0002BB90021212006F019FA002070BD0121F9
:1079D000212006F013FA002070BD00BF909EFF1F0B
:1079E000429EFF1F5A9EFF1F589EFF1F109FFF1FA2
:1079F000184B1A8852B3184A128830B50A80B3F966
:107A00000030002B83EAE374A4EBE374BCBF2D23A6
:107A10008B70A0B2ACBF02310331012300E01346EA
:107A200003EB830252009442F9DA0C4D90FBF3F21F
:107A300085FB03E403FB1200DB173032D3EBA40316
:107A400080B201F8012BF1D10B7030BD044B1868E6
:107A500008607047E49CFF1FC432010067666666D9
:107A60003832010070B53C4D2B780646002B35D1DD
:107A70001C4673780BB9204670BDFAF7CFFA374A27
:107A8000374B3848127831781B78007802EB430383
:107A90004A1E03EB80030E2AEDD801A050F822F015
:107AA000097B00002B7B0000777A0000097B000037
:107AB000777A0000777A0000777A0000F77A000082
:107AC000777A0000777A0000777A0000777A0000F2
:107AD000777A0000777A0000F37A0000AE2122481E
:107AE00003F0EEFF204804F03BFA00232B70012442
:107AF000BFE706F0A9FEAF211B4803F0E1FF1B4AD8
:107B0000012313702B70B6E783B919480388042941
:107B10004FF6FF7103F1FF320CBF01230B461344F4
:107B200003F07F03013303800FE073B1013B114A7F
:107B300032F813304BB10E4E0F481049104A3380C3
:107B40000123002606700B701370084A02210123DE
:107B500011702B70204670BD808AFF1F3D9FFF1F54
:107B60003E9FFF1FE49EFF1F709FFF1FE89FFF1FA8
:107B7000E09EFF1F1C9EFF1F149DFF1F9C9CFF1F6C
:107B8000EB9FFF1F10B5064B064C1A8820460121BB
:107B900001F0DAFD21884220BDE8104001F0E6BD89
:107BA000FC9CFF1F109FFF1F10B5064B064C1A8848
:107BB0002046022101F0C8FD21884220BDE8104086
:107BC00001F0D4BD329DFF1F109FFF1F10B5064B63
:107BD000064C1A882046042101F0B6FD2188422077
:107BE000BDE8104001F0C2BD509EFF1F109FFF1F57
:107BF00010B5064B064C1A882046062101F0A4FD5C
:107C000021884220BDE8104001F0B0BD649EFF1FF6
:107C1000109FFF1F10B5064B064C1A882046002106
:107C200001F092FD21884220BDE8104001F09EBD88
:107C30009E9EFF1F109FFF1F08B5122001F0B0FD90
:107C4000054B1988884206D0122001F08FFDBDE84F
:107C5000084001F055BC08BD929EFF1F08B5582092
:107C600001F09EFD054B1988884206D0582001F08E
:107C70007DFDBDE8084001F043BC08BDA29EFF1F8A
:107C800008B5142001F08CFD054B1988884206D0F8
:107C9000142001F06BFDBDE8084001F031BC08BDC7
:107CA0003A9DFF1FF0B480EAE075A5EBE07500286F
:107CB000ACB21FDB1DBF2B230B704E1C0E460123E5
:107CC00000E0134603EB830252009542F9DA0B4FB2
:107CD00094FBF3F287FB030503FB1244DB173032FE
:107CE000D3EBA503A4B206F8012BF1D133700846FB
:107CF000F0BC70472D230B704E1CE0E7676666668C
:107D0000174B18880C2813D0192815D01A2817D00B
:107D10001B2819D01C281BD01D281DD01E2803D0BD
:107D20000C3800B2FFF7BEBF0E4A106808607047FB
:107D30000D4A1068086070470C4A10680860704768
:107D40000B4A1068086070470A4A1068086070475C
:107D5000094A106808607047084A10680860704750
:107D6000DE9EFF1FE4320100CC320100D032010060
:107D7000D4320100D8320100DC320100E0320100CF
:107D8000034B1888A0EB8000400000B2FFF78ABFC9
:107D9000D09FFF1F024B1888643800B2FFF782BFE4
:107DA000309FFF1F024B1888643800B2FFF77ABF7C
:107DB000049FFF1F024BB3F90000FFF773BF00BF22
:107DC000EC9CFF1F024B1888033800B2FFF76ABF14
:107DD000B69EFF1F024B18880C3800B2FFF762BF37
:107DE0008E9CFF1F024B1888183800B2FFF75ABF4D
:107DF000C49CFF1F024B1888183800B2FFF752BF0F
:107E0000C29CFF1F024B1888183800B2FFF74ABF08
:107E1000B89CFF1FC3681888183800B2FFF742BF2C
:107E2000054B1B881BB9054B18680860704708464E
:107E3000042203490AF002B8C09EFF1F3832010035
:107E400034320100054B1B881BB9054B18680860CC
:107E5000704708460422034909F0F0BFCA9CFF1F7F
:107E6000383201003432010030B5134C85B00125A1
:107E70002B463C2202212046009503F097FE204627
:107E800004F06EF8002240218023204601910093E7
:107E900011460A4B029504F011FD204604F06CF9DE
:107EA00007480849084A0023036083800B608B80E1
:107EB0001360938005B030BD709FFF1F78390100BB
:107EC000509FFF1F689FFF1FD89FFF1F10B500EB3B
:107ED000C00000F10F02D2B293B284B09C1E981C75
:107EE0003D2303918DE819003921024804F04AFC32
:107EF00004B010BD709FFF1F014B01221A70704724
:107F00005D9FFF1FF0B57A4B7A4C7B4F7B4E7C4DCB
:107F100085B004228DE80C0002932046794B402264
:107F2000802103F04BFC2046774A7849784C09F0D1
:107F3000F1F8784A784B9761784FD761784F9F6115
:107F4000784FDF61784FB761784FF761784FAF6155
:107F5000784FEF61784FA7617848794FE761794FA3
:107F600087617949794FC761794F8F61794A7A4F33
:107F7000CF617A4F97617A4B7A4FD7617A4F9F6181
:107F80007A4E7B4FDF617B4F7B4DB7617B4FF76153
:107F90007B4F7C4CAF617C4FEF617C4F7C48A7618D
:107FA0007C4FE7617C4F7D4987617D4FC7617D4F85
:107FB0007D4A8F617D4FCF617D4F7E4B97617E4FB4
:107FC000D7617E4F7E4E9F617E4FDF617E4FB761EE
:107FD0007E4D7F4FF7617F4FAF617F4C7F4FEF61E9
:107FE0007F4FA7617F48804FE761804F876180495D
:107FF000804FC761804F8F61804A814FCF61814F31
:108000009761814B814FD761814F9F61814E824F34
:10801000DF61824FB761824D824FF761824FAF615E
:10802000824C834FEF61834FA7618348834FE761A1
:10803000834F84498761844FC761844F844A8F612D
:10804000844FCF61844F854B9761854FD761854FB2
:10805000854E9F61854FDF61854F864DB761864FA5
:10806000F761864F864CAF61864FEF61864F874838
:10807000A761874FE761874F87618749874FC7614E
:10808000874F8F61874A884FCF61884F9761884BB0
:10809000884FD761884F9F61884E894FDF61894F34
:1080A000894DB761894FF761894F8A4CAF618A4F1B
:1080B0008A488B49EF618B4F8B4DA761E5618B4FF0
:1080C0008B4D8C4CDFF850E28B4A8C4B8761C5613D
:1080D0008C618B4E8B4F8C4D8C4CC1F81CE08C48C6
:1080E0008C499761D5619C61D861B16005B0F0BDE4
:1080F00040420F00709FFF1FD57D00006C8EFF1F58
:10810000F88FFF1F5C91FF1F1C89FF1F15B800002F
:10811000448FFF1FF089FF1F208FFF1FE9680000B9
:10812000C57D0000F56800009D6B0000857B0000A8
:10813000C56B0000A97B0000ED6B0000148AFF1FD7
:10814000CD7B0000B57D0000748CFF1F0569000029
:10815000156C0000288DFF1FF17B000031730000BB
:10816000508CFF1F156900003D6C00004C8DFF1FF7
:10817000157C0000A57D0000F090FF1F2569000020
:10818000957D0000CC90FF1F356900000976000046
:10819000048DFF1F5D720000817D0000E08CFF1FD9
:1081A000756E00008D6E0000FC8EFF1F816E00005A
:1081B000657300009C8BFF1F7D72000099730000A7
:1081C000B08FFF1F397C0000717600002C8CFF1FE0
:1081D0005D7C0000E56E00005C8BFF1F45690000C0
:1081E000656C00006490FF1F817C0000D976000060
:1081F000088CFF1F5569000041770000948DFF1F18
:1082000065690000B1770000E48BFF1F756900000D
:10821000456F0000148BFF1F85690000D5730000B7
:108220001C90FF1F956900009D6F0000B48EFF1F1A
:10823000A569000009740000F08AFF1FB5690000FD
:10824000F56F0000708DFF1FC56900003D740000D0
:10825000388AFF1FD56900004D700000988CFF1F01
:10826000E5690000F1790000D88EFF1FF569000074
:10827000757400002091FF1F056A00001978000046
:10828000488EFF1F156A000081780000CC8AFF1F0E
:10829000256A0000A9740000D48FFF1F9D720000A2
:1082A000E9780000908EFF1F356A0000017D000014
:1082B000A88AFF1F456A0000E1740000848AFF1F3E
:1082C000556A000049750000BC8CFF1F656A0000FC
:1082D000A5700000C08BFF1F756A00005C8AFF1F3D
:1082E000388BFF1FFD700000856A0000557100008B
:1082F000956A0000AD710000688FFF1FCC89FF1FD9
:108300001491FF1F05720000B56A00005979000042
:10831000C56A0000DD880000A56A0000F0B5461CB3
:1083200083B00D460127032336B22AB204463146F4
:108330008DE888002348ADB204F0BAF90C23AA1CDA
:1083400012B200930197052321B21E4804F0B0F940
:108350001D4A1E4B12881B68BA422AD023D3022A18
:1083600010D11B4CA3F6CA0384FB03241C44DB1767
:10837000C3EB24140A2CA8BF0A2424EAE474A2B292
:1083800023B202E000231A461C460D35AA1A01202A
:108390000093019012B2314603230A4804F006F913
:1083A000204603B0F0BD0B4CA3F6FC0384FB032472
:1083B000DDE7094CA3F6980384FB0324DB17C3EB2A
:1083C000A404D7E7709FFF1F3C9EFF1FA49EFF1FC2
:1083D00009CB3D8D1F85EB51398EE3382DE9F043F4
:1083E0008FB283B0DFF84C80BD1D461D2DB204B2A4
:1083F00036B24FF001090AB2234631464046009595
:10840000CDF8049004F004F92A463346214640464C
:108410008DE8200204F0FCF807F10C0200953346C9
:1084200012B22146CDF80490404604F0F1F803B0B2
:10843000BDE8F083709FFF1F2DE9F043804685B0B3
:10844000002956D10121304804F078FC2F4998F8D2
:10845000062098F8083011F80290994522DA4FEA80
:1084600089064D460C24D8F80C3027489B595F6884
:1084700022B2002104F05EFC384609F021FC3946A6
:108480000246214804F0F0FD1F4804F003FE98F86E
:10849000083001350934AB42A4B206F1040601DD0F
:1084A000422CE0D1B9F1000F13D109F10609994529
:1084B0000CDA3C2301213B220391029300930192A9
:1084C00039233F223A21104804F05CF905B0BDE899
:1084D000F0830F2301213B22039102930093019229
:1084E00039230C223A21084804F04CF998F8083056
:1084F000DBE700213423009301913F230C22024843
:1085000004F054F89EE700BF709FFF1F689FFF1F95
:1085100010B5104C0121204604F016FC2046012124
:1085200004F00CFC20463422552104F003FC2046C4
:108530000222094904F098FD20460522074904F06B
:1085400093FD204604F0A6FD2046BDE8104003F050
:1085500013BE00BF709FFF1F303301003433010092
:1085600070B50D46064609F0ABFB00EB40008400F9
:10857000002D36D0284609F0A3FB00EB4000400058
:1085800023185B1003F16001091A282209B2174869
:10859000C3F1600404F0CEFB0121144804F0CEFBCB
:1085A000284609F08DFB29460246104804F05CFD80
:1085B0000E4804F06FFD02210C4804F0BFFB21B20D
:1085C00021220A4804F0B6FB304609F079FB314617
:1085D0000246064804F048FD0448BDE8704004F037
:1085E00059BD6410C4F16004E5E700BF709FFF1F30
:1085F00010B50D4B1B5C51F82340237884B013B1A8
:10860000012004B010BD04AA01A942F8103D204683
:10861000A3699847A38A9B07F2D401A80099FFF7A2
:108620009FFF012004B010BD509FFF1F2DE9F04FA8
:108630002F4DDFF8CCB0DFF8C4A0DFF8C8900FCD25
:1086400091B003AC0FC40FCD0FC40FCD0FC42B6876
:1086500023600025A8462F462E4600E09846BAF82B
:10866000003024495BF8232028461123F8F7A4F8AA
:1086700000EBC00400EB840089FB00340444C01705
:10868000C0EB6434C4F13C00C6F13C0207F1410187
:10869000012600B208F1410300901BB2019612B20C
:1086A00009B2154803F0B4FF08EB060305F21115F3
:1086B0003C2B2646ADB24746D0D134226B210E4822
:1086C00004F038FB00210C4804F038FB0B4B1B88EE
:1086D00010AA02EB830353F8344C204609F0F0FA59
:1086E00002460548214611B0BDE8F04F04F0BCBC7D
:1086F000202F0100DC280100709FFF1FAE9CFF1F90
:108700004027010009000280234B70B5B3F9003007
:1087100083EAE374A4EBE374002B82B0A1B234DBF0
:1087200068466D46012300E0134603EB83025200C6
:108730009442F9DA194E91FBF3F286FB03E403FB52
:108740001211DB173032D3EBA40389B205F8012BE9
:10875000F1D119462B70FFF703FF114B1B7813B1B2
:10876000104B1B780BB902B070BD01210E4804F00C
:10877000E5FA332264210C4804F0DCFA04220B49A8
:10878000094804F071FC02B070BD2D238DF8003053
:108790000DF101056846C5E75A9EFF1F67666666CC
:1087A000429EFF1F589EFF1F709FFF1F3C3301001A
:1087B00010B5424C424882B003F0D2FB2378C3B9D3
:1087C00006213F4804F0BAFA2378012B37D90A2250
:1087D000022B11463A486BD004F0ACFA3949032217
:1087E000374804F041FC364802B0BDE8104004F0C0
:1087F00051BC354B1A7801210523002A35D101914E
:10880000009311462E4803F053FF304B1A78002A8C
:1088100036D0052301220192009300220A21284824
:1088200003F0C4FE2A4B1A78002A35D10121052312
:10883000019100931421224803F03AFFC0E7254C30
:108840002388092B32D9632B8CBF0A211F210A22CE
:108850001B4804F06FFA2188194804F06BFC184893
:1088600002B0BDE8104004F015BC00220191009355
:108870001146134803F09AFE144B1A78002AC8D107
:1088800005230121019100930A210D4803F010FFF7
:108890000F4B1A78002AC9D00122052301920093B8
:1088A00000221421064803F081FE89E73021CEE73B
:1088B00004F040FA0322084992E700BFEB9FFF1F34
:1088C000709FFF1F483301003D9FFF1F3E9FFF1F0A
:1088D000E49EFF1FE09EFF1F44330100F8B56D4D7D
:1088E000287840B96C4B1B6899425CD36B4A0123D2
:1088F00013702B70F8BD0C4600266948664F03F0D4
:108900002FFB04F6AC53324665483B6031212E7094
:1089100004F010FA01216248624D04F015FA314664
:108920005F4804F00BFA05225F495D4804F09CFBA8
:108930005B4804F0AFFB0C221021594804F0FAF90F
:108940000B225A49564804F08FFB052258495448D7
:1089500004F08AFB524804F09DFB564B50481C68BB
:10896000A4F69803C3EB031385FB03251D441021D4
:10897000DB172022C3EB652504F0DCF940F6CC338D
:108980009C4205F124054FF022014FF004000BDC5E
:10899000FFF7C4FC484B1C88064674B3012C46D034
:1089A000022C41D00120F8BDFFF718FD09224349F0
:1089B0003B4804F059FB2A221021394804F0BAF947
:1089C0003F4C374884FB0534EB17C3EBA404214626
:1089D00004F0B0FB01223B49314804F045FB04EBB5
:1089E0008401A5EB41012E4804F0A4FB0122364985
:1089F0002B4804F039FB0120F8BD344910222848E7
:108A000004F032FB264804F045FB2A2210212448BA
:108A100004F090F93146224804F08CFB07222C49DF
:108A20001F4804F021FBCBE70C222A49E7E70C2280
:108A300029491B4804F018FB194804F02BFB2A2293
:108A40001021174804F076F9314615481C4E04F001
:108A500071FB07221E49124804F006FB86FB05360F
:108A6000EB17C3EBA60631460D4804F063FB224624
:108A700014490B4804F0F8FA06EB8601A5EB410116
:108A8000074804F057FB22460F49054804F0ECFA6A
:108A90002046F8BD808AFF1F649FFF1FE89FFF1FCD
:108AA000709FFF1F3B773B984C330100543301000C
:108AB00034330100A49EFF1F3C9EFF1F6033010062
:108AC00067666666603F0100D83E01006C330100B6
:108AD0008033010098330100883301002DE9F04113
:108AE000754C2278002A05460F4614BF4FF0010846
:108AF0004FF000084ED1714E3368CB1AB3F5FA6FC0
:108B000004D86B78A3B94046BDE8F0816C4B6D4842
:108B10006D49DFF8D0E11A700123037009882370D2
:108B200026208EF8002000F021FE6B78002BEAD082
:108B30003760F9F773FA654A654B66491278287809
:108B40001B78097802EB4303421E03EB81030E2AD4
:108B5000D9D801A151F822F0498C0000158C0000F1
:108B6000078B0000498C0000078B0000078B00007A
:108B7000078B0000FD8B0000078B0000AF8B00000F
:108B8000078B0000078B0000078B0000078B00009D
:108B9000AB8B0000AF215048484E02F091FFFFF729
:108BA00007FE002337602370ABE705F04DFE4A480F
:108BB00003F0D6F90221484804F0C0F80F2223211F
:108BC000454804F0B7F805224449434804F04CFAFC
:108BD000414804F05FFA1E2223213F4804F0AAF81E
:108BE00005223F493C4804F03FFA3B4804F052FA62
:108BF000394803F0C1FA00F0D3FC84E7394D2B78F3
:108C0000012B50D9304B2620198800F0AFFD0023EE
:108C10002B7078E7002B3FF476AF013B324A32F8F5
:108C20001330002B3FF46FAF274C304825492D4AB5
:108C300023804FF001080023037081F8008082F840
:108C40000080FFF7B5FD5EE793B1013B264A32F89D
:108C5000131019B31C4B254D1A4C224A19800026BB
:108C6000012326202E702370137000F07FFD15E085
:108C7000154C1E4922880B7004284FF6FF7002F134
:108C8000FF310CBF012202460A440E4E154D02F080
:108C90007F0201320121228031702B70FFF788FDA5
:108CA0004FF001082FE70649064A0123002008700B
:108CB00013702370A6E700BF808AFF1FE49FFF1F89
:108CC000E89FFF1F9C9CFF1FE09EFF1F3D9FFF1F13
:108CD0003E9FFF1FE49EFF1F709FFF1FA8330100F0
:108CE000B0330100EB9FFF1F1C9EFF1F149DFF1F51
:108CF0002DE9F04F05468BB00F46AD4801211646D1
:108D000004F022F8AA8812F0010440F0B080DFF8E5
:108D1000CC8298F80030002B7DD1AB79A54AD15C8C
:108D2000A1B9DFF8BCA279781AF8039041B3397879
:108D30000139072900F2B780DFE811F0F100540192
:108D4000B5006C01B500B500B500E9007C78002CD9
:108D500000F0CA800139EC68387854F82170FC685A
:108D6000411EB4F80080072900F2A780DFE811F067
:108D700074015901A5006C01A500A500A5009F0084
:108D8000DFF854A2DAF80020B21AB2F5967F75D94E
:108D9000894A107801281ABF012010701170874A83
:108DA00018BF0146D05CC0EB0900C0B2FFF78EF8D7
:108DB0000124CAF80060AB889B0770D57B78002B34
:108DC0006DD0F9F72BF97E4B7E4A7F481B781278DD
:108DD00039780078022515FB02330A2903EB80035A
:108DE00000F04E810C295AD1002B58D003F1190004
:108DF000764E774A013B0021400080B226F81310DE
:108E00000123157088F8003000F0B0FC714B03228C
:108E100020461A702FE0664803F0A2F8012164484A
:108E200003F08CFF62482246214603F083FFAB88A3
:108E3000580725D42C68204608F042FF21460246F8
:108E40005B4804F011F95A4804F024F9092201237F
:108E50008DE80C0000217F23554803F0D9FB002149
:108E60002846FFF7E9FA002388F8003055E7AB6899
:108E70003146384698470BB0BDE8F08F0846FAE710
:108E80002B6804A8984704A808F01AFF04A9024612
:108E9000474804F0E9F8464804F0FCF8D6E72046D5
:108EA0000BB0BDE8F08F00240AF8039083E700219F
:108EB000D1543846FB699847FC68A4F80080002725
:108EC00025223C238DE8840041211822384803F0F4
:108ED0006DFBE968A879FFF78BFB374A3E4B1770AB
:108EE0001E600BB0BDE8F08F3B490A68B21AB2F5BC
:108EF000967FD4D9304F0E603E78012E00F0B480BA
:108F0000E968184601233B70FFF772FBB3E7304A6C
:108F1000E9791170012288F800200024C4E72A7A38
:108F2000013A4A45BFDD09F10104E4B2A145BAD0D6
:108F3000224E16F803B0CBEB0900C0B20021FEF7B9
:108F4000C5FF2B7A052BD9461BD9CBEB0402042A8B
:108F500040F3AE80A4F1040BBBF1000FC0F2B0806F
:108F6000063B5B45A8BF5B465FFA83F9AA791348C5
:108F7000B15C994205D000F8029001212846FFF724
:108F80005BFAC9EB0400C0B201210B4EFEF79EFF55
:108F900000213423019100930548317040230B22B6
:108FA0003F21A14603F002FB0124AB797CE700BF1F
:108FB000709FFF1FD89FFF1FE99FFF1F689FFF1F24
:108FC0003D9FFF1F3E9FFF1FE49EFF1F1C9EFF1F34
:108FD000E89FFF1FEB9FFF1FD49FFF1F808AFF1F8B
:108FE000509FFF1F0FFA89F1E868604C50F821602C
:108FF0002168049134785E4904980860002C71D08F
:10900000012C7FF450AF5B4A317A88F80040117030
:10901000002449E7B9F1000F50D009F1FF34E4B260
:1090200084E7B98A01F0040189B200293FF440AF16
:109030003B6A03929847039A00283FF43DAFAB790F
:10904000FC680021D15438E77B8A43453CD908F1BC
:1090500001081FFA88F830E73B8A43453BD208F104
:10906000FF381FFA88F828E725238DE818004248C2
:109070003C703C231822412103F098FA3046FAE66E
:10908000002B3FF40CAF3D4A3D4E1188394A03F1A5
:109090001900013B400080B226F81310012388F824
:1090A0000030157000F062FB364B20461D70E2E682
:1090B000002A3FF755AF04F1FF3B4DE74C46F3E67E
:1090C0004FF000094B4651E7BB8ADA077FF5F5AE52
:1090D000B7F81080F1E6BB8AD9077FF5EEAEB7F896
:1090E0001280EAE62849C85CC0EB090009F1010ECC
:1090F000C0B201214FF0340B02F803E0FEF7E6FEA8
:10910000B6681D48019440230B223F210124CDF86D
:1091100000B003F04BFA40230B223F211648CDF854
:1091200000B0019403F0C4FA2146134803F006FE90
:10913000304608F0C5FDA0EB800000F15F0109B2E8
:109140000F220D4803F0F6FD304608F0B9FD314618
:109150000246094803F088FF074803F09BFFE968CF
:10916000A879FFF745FAAB799EE600BF28A0FF1F5C
:10917000D49FFF1FE89FFF1F709FFF1FE09EFF1FF0
:109180001C9EFF1FEB9FFF1F689FFF1F2DE9F047ED
:10919000DFF808926D4B99F800601B68DFF800A2B9
:1091A00082B0003601934FF0030018BF0126019FE3
:1091B0009AF8008004F028FE0546042004F024FEFE
:1091C0000446052004F020FE800040EA4404062006
:1091D00004F01AFE2C4364B25D4944EAC0000A78E8
:1091E00080F00F03DBB29A425A4A3CD0176000224B
:1091F00059480B7003788DF800808DF8012053B327
:10920000564A12684EF66021BA1A8A4219D8022BC1
:1092100059D0012B5FD0062B48D0032B63D0042BF1
:1092200069D0052B77D0072B7DD0082B00F08380E9
:10923000092B68D016B14A4802F09EFF02B0BDE883
:10924000F087484A484C00230121237003701360C3
:10925000938089F800103A4669464448FFF748FD74
:109260003043C6B2E6E71268BA1A1E2A6BD99AF8DA
:109270000020934222D0394C3D488AF80030012B1F
:10928000276082EA030207609846B1D0042BAFD171
:1092900037480068381AB0F5C87FA9D9354C20681E
:1092A000381A3228A4D927601A46A1E73A466946F7
:1092B0003148FFF71DFD3043C6B2BBE7012B4FF02D
:1092C0000002E3D1E4E73A4669462C48FFF710FD77
:1092D0003043C6B2AEE73A4669462948FFF708FD73
:1092E0003043C6B2A6E73A4669462648FFF700FD76
:1092F0003043C6B29EE73A4669462348FFF7F8FC7A
:109300003043C6B296E73A4669462048FFF7F0FC7C
:109310003043C6B28EE73A4669461D48FFF7E8FC7F
:109320003043C6B286E73A4669461A48FFF7E0FC82
:109330003043C6B27EE73A4669461748FFF7D8FC85
:109340003043C6B276E7002252E700BF28A0FF1FD5
:10935000EC9FFF1F589FFF1FE89FFF1FE09FFF1F0D
:10936000709FFF1FD89FFF1FEA9FFF1F70310100F2
:10937000F09FFF1F609FFF1FA0310100C830010058
:10938000DC2F01001C3E01000C3E0100CC2F01002F
:1093900034300100583E01001491FF1F808AFF1FE6
:1093A0005C9FFF1F28B11028044BA8BF1020186035
:1093B0007047024B01201860704700BFF49FFF1FE9
:1093C00008B5002006F02AF90028FAD108BD00BF30
:1093D00010B504464FF4406005F034F805F08CF801
:1093E0000A4B1B7833B96CB1102C094BA8BF102461
:1093F0001C6010BD4FF4C05004F0FAFD04F02EFFC5
:10940000002CF1D1024B01241C6010BD429EFF1FB5
:10941000F49FFF1F70B50D461446064605F062F82E
:10942000284605F05FF8204605F05CF8084B1B78ED
:1094300013B1084B1B7803B970BD304604F0B6FE7B
:10944000284604F0B3FE2046BDE8704004F0AEBEEE
:10945000429EFF1F589EFF1F38B5164D2B780446BD
:1094600041F6FF72A0F50050824203F1FF33A8BF1E
:1094700002461B0202F5005203F47063100443F429
:10948000604343F00E0300F4FE005204184302F060
:10949000FE42104305F0F8FF2868013860F01F0015
:1094A000C4F3C61204F07F01C0B2BDE83840FFF734
:1094B000B1BF00BFF49FFF1F70B5104E3378013B62
:1094C0001B0203F47063044643F43043080622048D
:1094D00000F0FE4043F00B03034302F4FE00184388
:1094E0000D4605F0D1FF3068013860F04F002A4684
:1094F0002146C0B2BDE87040FFF78CBFF49FFF1F4C
:1095000008B564210720FFF7D7FF7F210B20BDE8B6
:109510000840FFF7D1BF00BF70B5104E3378013B54
:109520001B0203F47063044643F41043080622044C
:1095300000F0FE4043F00903034302F4FE00184329
:109540000D4605F0A1FF3068013860F06F002A4633
:109550002146C0B2BDE87040FFF75CBFF49FFF1F1B
:1095600038B50E4D2B78013B1B0203F470630446A3
:1095700043F41043000443F0090300F4FE001843D1
:1095800005F082FF2868013860F06F002146C0B204
:109590000022BDE83840FFF73DBF00BFF49FFF1F2A
:1095A00010B500217B20FFF787FF0024E0B2FFF712
:1095B000D7FF0134022004F05DFC802CF6D110BDF1
:1095C00038B50C46054604F08DFF204604F08AFFAE
:1095D000074B1B7813B1074B1B7803B938BD2846DE
:1095E00004F0E4FD2046BDE8384004F0DFBD00BFD4
:1095F000429EFF1F589EFF1F38B50D4D2B78013B33
:109600001B0203F47063044643F45043000443F028
:109610000D0300F4FE00184305F036FF28680138FA
:1096200060F02F002146C0B2BDE83840FFF7C8BF48
:10963000F49FFF1F38B50E4D2B78013B01381B02FC
:10964000C4B203F47063200443F4404343F00C03BA
:1096500000F4FE00184305F017FF2868013860F099
:109660003F002146C0B2BDE83840FFF7A9BF00BFA8
:10967000F49FFF1F38B504460D46F02004F032FF7A
:1096800035B1254414F8010B04F02CFFAC42F9D19C
:10969000F720BDE8384004F025BF00BF00B50B4BF4
:1096A00083B00246998818680090032AADF8041028
:1096B00002D903B05DF804FB684606218DF8052049
:1096C000FFF7D8FF03B05DF804FB00BF983E010030
:1096D00000B50B4B024683B0186899880090131FA1
:1096E0004C2BADF8041002D903B05DF804FB6846BA
:1096F00006218DF80520FFF7BDFF03B05DF804FBE0
:10970000A03E0100030203F4FE43C0F3C610184359
:10971000704700BF03784078DB0103F47E5300F00C
:109720007F001843704700BF82B002AA114642F87A
:10973000040D002012F8013B03F07F03914243EA3D
:109740000020F7D102B07047003210B403884FF008
:10975000010404FA01F418BF012202FA01F123EA1C
:1097600004020A43028010BC704700BF70B5CEB23D
:109770000C46054603F010FF864203D031462846CA
:1097800003F024FF0135284603F006FF240A844233
:1097900005D021462846BDE8704003F017BF70BDD4
:1097A00038B5054603F0F8FE4FF0000460F30704F7
:1097B000681C03F0F1FE60F30F24A0B238BD00BFB7
:1097C000F8B504460020FFF7EBFF002C00F0838182
:1097D0004FF4AF610220FFF7C9FF04204FF47A6114
:1097E000FFF7C4FF0B2004F00FFB002840F079873F
:1097F0004FF496610620FFF7B9FF4FF4FA61082095
:10980000FFF7B4FF4FF4FA610A20FFF7AFFF40F60D
:10981000B8310C20FFF7AAFF4FF42F612220FFF789
:10982000A5FF40F6AC512420FFF7A0FF7D212A20A0
:10983000FFF79CFF0C210E20FFF798FF012110205D
:10984000FFF794FF02211220FFF790FF0021142060
:10985000FFF78CFF00211620FFF788FF0221182058
:10986000FFF784FF01211A20FFF780FF01211C2050
:10987000FFF77CFF04211E20FFF778FF1421202032
:10988000FFF774FF01212620FFF770FF0321282036
:10989000FFF76CFF04212C20FFF768FF14212E2016
:1098A000FFF764FF00213020FFF760FF0C2132201A
:1098B000FFF75CFF00213420FFF758FF002136201E
:1098C000FFF754FF00213820FFF750FF00213A2016
:1098D000FFF74CFF00213C20FFF748FF00213E200E
:1098E000FFF744FF00214020FFF740FF0021422006
:1098F000FFF73CFF1F214420FFF738FF13214620CC
:10990000FFF734FF0E214820FFF730FF11214A20D6
:10991000FFF72CFF0A214C20FFF728FF00214E20E3
:10992000FFF724FF06215020FFF720FF02215220DD
:10993000FFF71CFF0C215420FFF718FF00215620D1
:10994000FFF714FF00215820FFF710FF01215A20D4
:10995000FFF70CFF08215C20FFF708FF0A215E20BB
:10996000FFF704FF00216020FFF700FF04216220C1
:10997000FFF7FCFE01216420FFF7F8FE00216620BE
:10998000FFF7F4FE0B216820FFF7F0FE7F216A202D
:10999000FFF7ECFE00216C20FFF7E8FE00216E20AF
:1099A000FFF7E4FE00217020FFF7E0FE00217220A7
:1099B000FFF7DCFE00217420FFF7D8FE1F21762080
:1099C000FFF7D4FE13217820FFF7D0FE0E217A2076
:1099D000FFF7CCFE11217C20FFF7C8FE0A217E2074
:1099E000FFF7C4FE1F218020FFF7C0FE1321822055
:1099F000FFF7BCFE0E218420FFF7B8FE1121862060
:109A0000FFF7B4FE0A218820FFF7B0FE00218A206C
:109A1000FFF7ACFE00218C20FFF7A8FE0021962066
:109A2000FFF7A4FE00219820FFF7A0FE00219A2056
:109A3000FFF79CFE05219C20FFF798FE06219E2043
:109A4000FFF794FE0021A020FFF790FE7F21A220C7
:109A5000FFF78CFE40F2A461A420FFF787FE4FF4CD
:109A6000E161A620FFF782FE0021A820FFF77EFE1D
:109A70000021AA20FFF77AFE0221AC20FFF776FE34
:109A80000121AE20FFF772FE0121B020FFF76EFE2C
:109A90000B21B220FFF76AFE6421B420FFF766FEB7
:109AA0006421B620FFF762FE0321B820FFF75EFEB7
:109AB0002C210020FFF75AFE0220FFF771FEB0F5BF
:109AC000805F034616D34FF4AF610220FFF74EFECE
:109AD0004FF4AF630EE04FF6FF7398423FF478AE59
:109AE0002C2840F00A860220FFF75AFEB0F5805F6E
:109AF0000346E8D2D24A04201380FFF751FEB0F5A6
:109B0000805F034680F05684CE4A06201380FFF71C
:109B100047FEA0F52F739BB2B3F57A6F024606D9C4
:109B200040F628210620FFF721FE40F62822C64BEA
:109B300008201A80FFF734FEA0F52F739BB2B3F50F
:109B40007A6F024606D940F6E4410820FFF70EFE80
:109B500040F6E442BD4B0A201A80FFF721FEA0F533
:109B6000FA739BB240F6AC518B42024606D94FF4D1
:109B7000FA610A20FFF7FAFD4FF4FA62B44B0C20A9
:109B80001A80FFF70DFEA0F5FA739BB240F6AC51B8
:109B90008B42024606D940F6B8310C20FFF7E6FDAD
:109BA00040F6B832AB4B0E201A80FFF7F9FD1828AB
:109BB000034600F2C584A84A10201380FFF7F0FD89
:109BC000431E9BB20F2B024604D901211020FFF740
:109BD000CDFD0122A14B12201A80FFF7E1FD0A28DA
:109BE000034600F2A6849E4A14201380FFF7D8FD96
:109BF0000128034604D900211420FFF7B7FD0023F4
:109C0000984A16201380FFF7CBFD7F28034600F209
:109C10008984954A18201380FFF7C2FD0528034662
:109C200000F27984914A1A201380FFF7B9FD0C28BD
:109C3000034600F2BD848E4A1C201380FFF7B0FD5E
:109C40000428034600F2AD848A4A1E201380FFF7E1
:109C5000A7FD0928034600F29D84874A202013802F
:109C6000FFF79EFD4628034600F28D84834A22209A
:109C70001380FFF795FDA0F5FA739BB240F6AC5147
:109C80008B42024606D94FF42F612220FFF76EFD6A
:109C90004FF42F627A4B24201A80FFF781FDA0F544
:109CA000FA739BB240F6AC54A342024604D9214653
:109CB0002420FFF75BFD2246724B26201A80FFF717
:109CC0006FFD7F28034600F257846F4A28201380D7
:109CD000FFF766FD0628034600F247846B4A2A20F8
:109CE0001380FFF75DFDA0F132039BB2B3F5967FC1
:109CF000024604D97D212A20FFF738FD7D22644BDE
:109D00002C201A80FFF74CFD0C28034600F2268415
:109D1000604A2E201380FFF743FD1E28034600F201
:109D200016845D4A30201380FFF73AFD0928034668
:109D300000F2D084594A32201380FFF731FD1E28EB
:109D4000034600F2C084564A34201380FFF728FDF2
:109D50007F28034600F2B084524C36202380FFF760
:109D60001FFD7F28034600F2A08438206380FFF7A0
:109D700017FD7F28034600F291843A20A380FFF765
:109D80000FFD7F28034600F282843C20E380FFF72A
:109D900007FD7F28034600F273843E202381FFF7EE
:109DA000FFFC7F28034600F2648440206381FFF7B4
:109DB000F7FC7F28034600F255844220A381FFF779
:109DC000EFFC394D28804420FFF7EAFC3028034699
:109DD00000F24184354A46201380FFF7E1FC302829
:109DE000034600F23184324C48202380FFF7D8FC30
:109DF0003028034600F221844A206380FFF7D0FC1C
:109E00003028034600F212844C20A380FFF7C8FCE0
:109E10003028034600F2DF834E20E380FFF7C0FCCA
:109E20000128034604D900214E20FFF79FFC0023A0
:109E3000204A50201380FFF7B3FC431E3CE000BFD4
:109E4000449DFF1F0E9FFF1FFE9CFF1FDC9EFF1FF8
:109E5000A89EFF1FC09CFF1F8E9CFF1F5A9EFF1FC6
:109E6000929EFF1F3A9DFF1F949CFF1F4A9DFF1F5C
:109E7000E49CFF1FDE9CFF1FC89CFF1FEE9EFF1F80
:109E8000569EFF1F529EFF1FE09EFF1FB69EFF1FA4
:109E9000069FFF1FAE9CFF1F309DFF1F1C9FFF1FD3
:109EA000DE9EFF1F1C9EFF1F109FFF1FB89CFF1F01
:109EB000B89EFF1FDC9CFF1F9BB20B2B024604D9F0
:109EC00006215020FFF752FC0622CF4B52201A8069
:109ED000FFF766FC0428034600F27783CB4A542040
:109EE0001380FFF75DFC431E9BB21D2B024604D975
:109EF0000C215420FFF73AFC0C22C54B56201A8047
:109F0000FFF74EFC0128034604D900215620FFF735
:109F10002DFC0023BF4A58201380FFF741FC7F2807
:109F2000034600F24C83BC4A5A201380FFF738FCEA
:109F3000431E9BB2092B024604D901215A20FFF788
:109F400015FC0122B54B5C201A80FFF729FC431E4B
:109F50009BB2102B024604D908215C20FFF706FCB7
:109F60000822AF4B5E201A80FFF71AFC431E9BB2FB
:109F70001D2B024604D90A215E20FFF7F7FB0A22B7
:109F8000A84B60201A80FFF70BFC0228034600F262
:109F9000A482A54A64201380FFF702FC012803462F
:109FA00004D901216420FFF7E1FB01239F4A6220CD
:109FB0001380FFF7F5FBC31E9BB2012B024604D9A9
:109FC00004216220FFF7D2FB0422994B66201A80FD
:109FD000FFF7E6FB7F28034600F27982954A682066
:109FE0001380FFF7DDFB7F28034600F26A82924A66
:109FF0006A201380FFF7D4FB7F28034600F25B82C0
:10A000008E4A6C201380FFF7CBFB0328034600F237
:10A010004C828B4A6E201380FFF7C2FB192803463F
:10A0200000F23D82874A70201380FFF7B9FB0228B7
:10A03000034600F22E82844A72201380FFF7B0FBA1
:10A040000628034600F21F82804A74201380FFF71F
:10A05000A7FB0528034600F210827D4A8A20138060
:10A06000FFF79EFB0A28034600F20182794A8C2002
:10A070001380FFF795FB0428034600F2F281764A2D
:10A0800098201380FFF78CFB0128034604D9002198
:10A090009820FFF76BFB0023704A9A201380FFF78C
:10A0A0007FFB0128034604D900219A20FFF75EFBBD
:10A0B00000236B4A96201380FFF772FB0B280346A0
:10A0C00000F2C981674A9C201380FFF769FB831E59
:10A0D0009BB2032B024604D905219C20FFF746FBC7
:10A0E0000522614B76201A80FFF75AFB3028034681
:10A0F00000F2AB815D4A78201380FFF751FB3028D6
:10A10000034600F29C815A4C7A202380FFF748FBDB
:10A110003028034600F28D817C206380FFF740FBEE
:10A120003028034600F27F817E20A380FFF738FBB2
:10A130003028034600F271818020E380FFF730FB76
:10A140003028034600F263814A4A82201380FFF7D9
:10A1500027FB3028034600F25481474C842023809B
:10A16000FFF71EFB3028034600F2458186206380FE
:10A17000FFF716FB3028034600F237818820A380C2
:10A18000FFF70EFB3028034600F22981A020E38070
:10A19000FFF706FB0128034604D90021A020FFF7A2
:10A1A000E5FA0023354A9E201380FFF7F9FAC31E13
:10A1B0009BB20C2B024604D906219E20FFF7D6FA4B
:10A1C00006222F4BA2201A80FFF7EAFA431E9BB209
:10A1D0007E2B024604D97F21A220FFF7C7FA7F22F7
:10A1E000284BA4201A80FFF7DBFAA0F5AF639BB2DF
:10A1F000B3F5167F024647D940F2A461A420FFF7C9
:10A20000B5FA40F2A4623FE02089FF1F2E89FF1FAC
:10A21000A889FF1F1E9DFF1FA29EFF1F889CFF1F76
:10A22000AC89FF1F2C89FF1F4E9EFF1FB09EFF1F92
:10A23000EC9CFF1FF09EFF1F1C9DFF1FCC9CFF1F6F
:10A240007C9CFF1F409FFF1F3C9EFF1F189FFF1F0E
:10A25000D49EFF1F5C9EFF1F4C9EFF1FCA9CFF1FCA
:10A26000289DFF1F9C9EFF1FB09CFF1FC29CFF1FCD
:10A270002C9EFF1FC49CFF1F349EFF1FC09EFF1F0C
:10A280009489FF1FE29EFF1FD64BA6201A80FFF77E
:10A2900087FAA0F5AF639BB2B3F5167F024606D9E5
:10A2A0004FF4E161A620FFF761FA4FF4E162CE4B73
:10A2B000A8201A80FFF774FA0628034600F2898066
:10A2C000CA4AAA201380FFF76BFA032803467AD8FC
:10A2D000C74AAC201380FFF763FA0328034600F255
:10A2E0001481C44AB0201380FFF75AFA03280346AA
:10A2F00000F20581C04AAE201380FFF751FA7F2893
:10A30000034600F2F680BD4AB2201380FFF748FAF8
:10A310007F28034600F2E780B94AB4201380FFF794
:10A320003FFA431E9BB2C62B024604D96421B420D7
:10A33000FFF71CFA6422B34BB6201A80FFF730FAFD
:10A34000431E9BB2C62B024604D96421B620FFF7F8
:10A350000DFA6422AC4BB8201A80FFF721FA0828C6
:10A3600022D82B88DFF8C0E2A84FA94AA94DAA4EEF
:10A37000AA4CAB4903F0010CAEF800C0C3F3400E89
:10A38000A7F800E0C3F380071780C3F3C007A54A0E
:10A390002F70C3F30017C3F34015C3F38013378046
:10A3A00025800B801080F8BDB8200321FFF7DEF96F
:10A3B0000320D6E74FF47A610420FFF7D7F94FF472
:10A3C0007A63FFF7A1BB0021AA20FFF7CFF9002392
:10A3D0007EE70021A820FFF7C9F9002370E70A21D2
:10A3E0008820FFF7C3F90A23D0E611218620FFF762
:10A3F000BDF91123C2E60E218420FFF7B7F90E2321
:10A40000B4E613218220FFF7B1F91323A5E61F213B
:10A410008020FFF7ABF91F2396E60A217E20FFF785
:10A42000A5F90A2388E611217C20FFF79FF9112363
:10A430007AE60E217A20FFF799F90E236CE61321B4
:10A440007820FFF793F913235DE61F217620FFF7AD
:10A450008DF91F234EE600219620FFF787F9002390
:10A4600030E600218C20FFF781F9002307E6002168
:10A470008A20FFF77BF90023F8E500217420FFF71D
:10A4800075F90023E9E500217220FFF76FF9002339
:10A49000DAE500217020FFF769F90023CBE5002100
:10A4A0006E20FFF763F90023BCE500216C20FFF765
:10A4B0005DF90023ADE57F216A20FFF757F97F237F
:10A4C0009EE50B216820FFF751F90B238FE5002152
:10A4D0006620FFF74BF9002380E500216020FFF79D
:10A4E00045F9002355E50B21B220FFF73FF90B2377
:10A4F00012E70121AE20FFF739F9012303E701211B
:10A50000B020FFF733F90123F4E60221AC20FFF776
:10A510002DF90223E5E602211820FFF727F902238F
:10A52000FFF780BB00211620FFF720F90023FFF77B
:10A5300070BB02211220FFF719F90223FFF753BB6A
:10A540000C210E20FFF712F90C23FFF734BB142166
:10A550002E20FFF70BF91423FFF7E3BB04212C2077
:10A56000FFF704F90423FFF7D3BB03212820FFF7EB
:10A57000FDF80323FFF7B2BB01212620FFF7F6F811
:10A580000123FFF7A2BB14212020FFF7EFF81423CB
:10A59000FFF76CBB04211E20FFF7E8F80423FFF748
:10A5A0005CBB01211C20FFF7E1F80123FFF74CBB46
:10A5B00001211A20FFF7DAF80123FFF73CBB002145
:10A5C0005820FFF7D3F80023ADE402215220FFF713
:10A5D000CDF8022382E40A214C20FFF7C7F80A23B2
:10A5E0001AE400BF489DFF1FC89EFF1F8A9CFF1FE3
:10A5F000029DFF1FB29EFF1F409EFF1FD49CFF1FA6
:10A60000F69CFF1F049FFF1F309FFF1FFC9CFF1F36
:10A61000329DFF1F589EFF1F509EFF1FB49EFF1FBD
:10A62000649EFF1F909CFF1F9E9EFF1F11214A20CA
:10A63000FFF79CF81123FFF7E7BB0E214820FFF737
:10A6400095F80E23FFF7D8BB13214620FFF78EF8AD
:10A650001323FFF7C8BB1F214420FFF787F81F23F0
:10A66000FFF7B8BB00214020FFF780F80023FFF779
:10A67000A4BB00213E20FFF779F80023FFF795BB2C
:10A6800000213C20FFF772F80023FFF786BB002172
:10A690003A20FFF76BF80023FFF777BB0021382043
:10A6A000FFF764F80023FFF768BB00213620FFF7AF
:10A6B0005DF80023FFF759BB00213420FFF756F85F
:10A6C0000023FFF749BB0C213220FFF74FF80C2382
:10A6D000FFF739BB00213020FFF748F80023FFF7D0
:10A6E00029BB40F628210620FFF740F840F6E44158
:10A6F0000820FFF73BF8FFF785B817287FF668A812
:10A7000019287FF6D7A81B287FF6F4A81C283FF449
:10A7100009A91E287FF60EA91F283FF413A9202897
:10A720003FF42CA921283FF435A922283FF43AA967
:10A7300023283FF443A924283FF474A925283FF493
:10A7400079A926283FF47AA927283FF47FA9282849
:10A750003FF48AA929283FF48FA92A283FF49CA90D
:10A760002B287FF4A5A9FFF79FB900BFF8B5CB2030
:10A7700006F00AFD204B214A054603CB1368C5F8B5
:10A7800003001A0CBA20C5F807102B80AA70FEF738
:10A79000B9FF2E46002426F80B0FA0B2FFF700F8F1
:10A7A000FEF7B0FF0234BA2C26F8020FF5D16C1E6A
:10A7B00005F1C6064FF0FF3014F8013F0827584056
:10A7C0000F4B40F300017A1E0B4012F0FF0783EAA3
:10A7D0005000F5D1B442EFD1C043FEF7A5FF3A4691
:10A7E000C5F8C700CB21284604F09CFE2846BDE8EA
:10A7F000F84006F0D1BC00BFAC3E0100A83E01000D
:10A800002083B8EDF0B50E4B0E4C054693E80700DB
:10A8100085B024682E88AD7801AB83E80700270C4B
:10A82000184600220B21ADF804408DF80670ADF8F3
:10A830000C608DF80E5004F075FE05B0F0BD00BF41
:10A84000B83E0100A83E0100F0B5124B124D1E6843
:10A85000124F0FCD87B06C460FC495E8030044F843
:10A86000040B38683B79CDF80D00320C2C20218088
:10A870008DF802208DF81130ADF80060FEF742FF30
:10A880000022ADF80B001221684604F04BFE07B021
:10A89000F0BD00BFA83E0100C43E010034330100FA
:10A8A000002004F0BBBE00BF02F02EBE70B5124CFB
:10A8B00082B0002540230646294620460093019594
:10A8C0008023202201F072FE20222946204602F039
:10A8D00031FA2046012102F037FA304607F0F0F94C
:10A8E00031460246204602F0BFFB204602B0BDE8DA
:10A8F000704001F041BC00BF709FFF1FF0B5CA2936
:10A9000083B075D90546441E00F1C6064FF0FF30EE
:10A9100014F8012F08275040404A40F300017B1EE5
:10A920000A4013F0FF0782EA5000F5D1B442EFD19C
:10A93000C043FEF7F9FE0146D5F8C7000190019A21
:10A94000914202D0B2F17F2F0BD105F10B00FEF73F
:10A95000E1FEBA280BD03248FFF7A8FF002003B071
:10A96000F0BD3048FFF7A2FF384603B0F0BD05F157
:10A970000D00FEF7CFFE2C2840D1002440F6AC5647
:10A9800013E004281AD0062821D008281FD00A284E
:10A9900028D00C2822D1A1F5FA7292B2B24201D885
:10A9A000FEF7E4FE0234BA2C0ED004F10D00284468
:10A9B000FEF7B0FE022C0146A0B2E2D1B1F5805FF5
:10A9C000EED30234BA2CF0D1012003B0F0BDA1F5D2
:10A9D0002F7292B2B2F57A6FE4D8E1E7222801D063
:10A9E000242811D1A1F5FA7292B2B242DAD8D7E78F
:10A9F0000D48FFF75BFF002003B0F0BD0B48FFF7E9
:10AA000055FF002003B0F0BD2A28C9D1A1F13202C0
:10AA100092B2B2F5967FC5D8C2E700BF2083B8EDE9
:10AA2000083F0100F43E0100DC3E01001C3F010034
:10AA300003290CD970B5461C82B005460C46304639
:10AA400003222A4907F0AAF910B102B070BD70477D
:10AA50000B2C05D905222649281D07F09FF940B186
:10AA60002448FFF723FF244802B0BDE87040FFF7F9
:10AA7000C9BE05F10901032201A807F0DFF901A809
:10AA800003221E4907F08AF9D8B103221C4901A804
:10AA900007F084F908B301A803221A4907F07EF9E8
:10AAA000B0B91948FFF702FFA11E89B23046FFF77F
:10AAB00025FF0028C9D0154802B0BDE87040FFF757
:10AAC000F5BE1348FFF7F2FEFFF750FE1148F3E71B
:10AAD0001148FFF7EBFE1148C6E71148FFF7E6FE05
:10AAE00002B0BDE87040FFF7AFBE00BFA83E010056
:10AAF0004C330100343F0100483F01004C3F01004E
:10AB0000743F01008C3F0100903F0100A43F010011
:10AB1000503F0100643F0100B83F0100CC3F0100FD
:10AB2000783F01002DE9F043174D2B6883B0814633
:10AB30000F469046F3B1154E34880A1992B2184662
:10AB40001146328006F09EFE28603A46494620446F
:10AB500002F06CFDB8F1000F09D031882868FFF7CA
:10AB600067FF286806F018FB00232B60338003B0D2
:10AB7000BDE8F083054E01930846318006F004FBE2
:10AB8000019B28601C46E0E7FC9FFF1FF89FFF1F0A
:10AB900010B51F4C4FF4FA70FBF742FD204601F050
:10ABA000DFF900221146204602F0C4F820460121B8
:10ABB00002F0CAF82046002102F0C0F80B22154925
:10ABC000204602F051FA204602F064FA0F221249A0
:10ABD000204602F049FA204602F05CFA0F490722AB
:10ABE000204602F041FA204602F054FA204601F0D5
:10ABF000C3FA0B4B0B4A1A604FF4FA70FBF710FDC7
:10AC0000FFF722FE0848BDE81040FFF74FBE00BF27
:10AC1000709FFF1FD03F0100DC3F0100EC3F0100AF
:10AC200030A2FF1F25AB0000F43F01000020704759
:10AC300090F8392090F83800101A704790F83830A2
:10AC400090F839209A4205D95A1C034480F83820DC
:10AC5000187E70474FF0FF30704700BF90F83830D3
:10AC600090F839209A4286BF1B18187E4FF0FF30AB
:10AC7000704700BF704700BF38B50546B0F85E00AA
:10AC800090B195F85D301446C3F1210294420CD87E
:10AC900005F13B001844224602F0C8FC95F85D30EF
:10ACA000234485F85D30204638BD012014462871C4
:10ACB000EEE700BFB0F85E306BB190F85D30202B4E
:10ACC00007D8C218013380F85D30012082F83B10AC
:10ACD0007047012303710020704700BF00234269C1
:10ACE00080F8383080F8393080F85C3080F85D309A
:10ACF00080F85E3080F85F3006CA30B40D680469B1
:10AD000043662A4383660A60A370426990F8613003
:10AD10001649146813441D7A5B7B01EBC5051B02C1
:10AD20006D6803F4E06343F064032B6090F86230D5
:10AD300013449D7CDB7D01EBC5011B02496803F4D4
:10AD4000E06343F064030B6021685368194205D047
:10AD5000036927225A70036904229A710369202229
:10AD60005A71036980229A7030BC7047284B0100E9
:10AD700043690CCB12681A420CD0094B99420AD98C
:10AD8000084B9942036994BF1A220D225A70036935
:10AD900004229A717047036927225A70F7E700BFAF
:10ADA0007F1A06003F420F0010B50269D378DBB26C
:10ADB000D90604463DD510215806D17038D503F088
:10ADC000040303F0FF02002B51D03D49626E0023C3
:10ADD0000B7084F85D30002A5BD0904794F85D30AA
:10ADE000002B56D02369D0229A70236994F83B2017
:10ADF0001A712369012284F85C200222DA7010BDE6
:10AE0000304B84F860009C424AD02F4B9C4252D079
:10AE100094F8391013791F29DBB207D82848007835
:10AE200020B16018013184F8391003760223D37001
:10AE300010BD5906C3D4917801F0100101F0FF0054
:10AE40000029DDD013F001031ED194F85C1094F8B2
:10AE50005D00884281BF4B1C091984F85C3091F871
:10AE60003B3013712369D0229A702269DEE723698F
:10AE700084F83920C0229A702369114A1979012176
:10AE800011700222DA7010BDC02393702269137909
:10AE9000CCE70122002384F85D2084F83B30A1E751
:10AEA000626994F86130094913440322187A02F068
:10AEB00043FD2269ACE7626994F861300449F3E725
:10AEC00000A0FF1F5C91FF1FC891FF1F31AF000062
:10AED0003DAF00000369DB7803F0200373B190F805
:10AEE00060300133DBB2012B80F860301AD942693F
:10AEF00090F861301344187A02F09ABD70B5426937
:10AF000003F0FF0590F8613013440446187A02F00C
:10AF10008FFDA36E5BB184F8385094F83900BDE81A
:10AF20007040184790F85F30002BE0D0704770BD3C
:10AF30000148FFF7CFBF00BF5C91FF1F0148FFF73B
:10AF4000C9BF00BFC891FF1F2DE9F047374FDFF899
:10AF5000E0903B68026982B006460093DDF800800D
:10AF60000021A025D3789B065BD53B680193019B0C
:10AF7000C8EB03030F2BF5D949B1102BF2D00020F9
:10AF80009070336980229A7002B0BDE8F0877269D0
:10AF900096F8613013440521187A02F043FF726974
:10AFA00096F861301344012193F812A0504602F044
:10AFB00039FF09240021504602F020FF2B46013BB7
:10AFC000FDD10121504602F019FF2B46013BFDD176
:10AFD000013CEFD1706996F8611001444FF4A07202
:10AFE0000C7A4B7B09EBC4011B02496803F4E06354
:10AFF00043F064030B6096F862300344997CDB7D78
:10B0000009EBC1011B02496803F4E06343F06403E8
:10B010000B60013AFDD13269D3789B064FF00101F4
:10B02000A3D4012002B0BDE8F08700BF28A0FF1F15
:10B03000284B0100F0B503691222DA700269937897
:10B0400003F0200385B004460D46002B5ED0B423E8
:10B0500093703C4922690B680093009E05E00B68E1
:10B060000193019B9B1B042B42D8D37803F0200350
:10B0700003F0FF00002BF2D094F85D30002B31D0AC
:10B080004FF0000E4FF0020C04EB0E0393F83B3030
:10B0900013710B680393039F206907E09B060DD58E
:10B0A0000B680293029BDB1B052B28D8C378DBB20D
:10B0B00003F0020202F0FF06002AEFD080F803C07E
:10B0C0002669F378DBB2DF0632462DD49F062BD5F6
:10B0D000DB0731D40EF1010E94F85D305FFA8EFE7D
:10B0E0007345D1D800201DBB002384F85E3004E0F6
:10B0F0009070236980229A70042005B0F0BD86709C
:10B100002369802204209A7005B0F0BD03F0FF0689
:10B11000FFF71AFF10B9042005B0F0BD236984F8C9
:10B120005F60B0229A7094E78023B3700420DAE75E
:10B1300026698023B370D7E7BEF1000F0CBF022051
:10B140000320F6E728A0FF1F2DE9F041066900253E
:10B15000122780F8385080F83950F770D0F810C0B6
:10B160009CF802E00EF0200E88B004468846154692
:10B170001E46BEF1000F49D0B4238CF80230784B44
:10B1800021691A680092DDF800E006E01A68019271
:10B190000198CEEB0000042830D8C87800F02000D9
:10B1A00000F0FF070028F1D04FEA480242F0010208
:10B1B000D2B20A711A680292DDF808E0206906E04E
:10B1C0001A6803920399CEEB010105292AD8C178A8
:10B1D00001F0020101F0FF070029F1D04FF0020C4D
:10B1E00080F803C02269D17811F0110722D12DBB5C
:10B1F000002E0CBFA0238023937003E08F7023697F
:10B2000080229A70384608B0BDE8F0810EF0FF0742
:10B21000FFF79AFE0028F5D0236984F85F70B0220A
:10B220009A70ACE787702369802238469A7008B01C
:10B23000BDE8F081802393700027E3E7012D75D0EE
:10B24000A021917021690A79BE4667464FF0A80C8B
:10B250001A680492049805E01A680592059A121A71
:10B26000052A4AD8CA7802F0020202F0FF08002A32
:10B27000F2D0CF702169CA78D2B212F0100F08460E
:10B280005AD1920658D5013DEDB2012D49D0BEF1FB
:10B290001F0F3BD90A79012DDAD11A680692069D53
:10B2A00005E01A680792079A521B052A46D8C27809
:10B2B00002F0020202F0FF01002AF2D00223C37062
:10B2C0002269D378DBB2D9063AD49B0634D5B023B1
:10B2D000BEF11F0F93703FD8226904EB0E03127961
:10B2E0001A760EF1010E5FFA8EFE16B123698022E6
:10B2F0009A7084F839E0774684E781F80280236900
:10B3000080229A70774684F839E07BE704EB0E02DE
:10B3100091F8048082F818800EF1010E5FFA8EFE1B
:10B32000B9E781F802C021690846B0E7A821917009
:10B330002069BE460279B0E7774663E78170DEE7B1
:10B340001021A023D170013BFDD12269937803F035
:10B35000F7037746937055E723691B79C5E700BF6C
:10B3600028A0FF1F0148FFF71FBD00BF5C91FF1F12
:10B370000148FFF719BD00BFC891FF1F704700BF0C
:10B3800038B5144C037801225B000546204684F84A
:10B390003B3084F85E2084F85D20FFF78BFC20466C
:10B3A0000021FFF747FE0B4C2978012320461A465F
:10B3B000FFF7CAFE0128F6D194F8383094F8392006
:10B3C0009A4205D9E218013384F83830107E38BD2E
:10B3D000FF2038BD5C91FF1F38B51B4C037801225C
:10B3E0005B000546204684F83B3084F85E2084F8F4
:10B3F0005D20FFF75FFC20460021FFF71BFE124C8B
:10B400002978204601230222FFF79EFE0228F6D16A
:10B4100094F8382094F839108A420FD2531CDBB2CA
:10B42000A018994284F83830007E0AD923440232A9
:10B430001B7E84F8382040EA032038BD4FF6FF70A9
:10B4400038BD40F47F4038BD5C91FF1F0C2901D905
:10B45000002070470231490001F0FE01FFF7BCBF38
:10B4600070B50C4C0378164601255B00204684F825
:10B470003B3084F85E5084F85D50FFF71BFC31468A
:10B480002046FFF717FC29462046BDE87040FFF72D
:10B49000D1BD00BF5C91FF1FF8B505460F461646AB
:10B4A000412421463A462846FFF7DAFF611C023460
:10B4B000C9B232462846E4B2FFF7D2FF592CF0D188
:10B4C000F8BD00BF38B504460D463548FFF706FC09
:10B4D0006322802120462570FFF7C2FF012002F081
:10B4E000C9FC204600225E21FFF7BAFF20465D21FD
:10B4F000FFF746FF242801D0002038BD2046062251
:10B500000C21FFF7C9FF204601222B21FFF7A8FFDE
:10B51000204601222C21FFF7A3FF20460E222D21D9
:10B52000FFF79EFF204600222E21FFF799FF2046BD
:10B5300001222F21FFF794FF204605223021FFF73B
:10B540008FFF204601223121FFF78AFF204600228B
:10B550003221FFF785FF204600223321FFF780FFCD
:10B56000204600223421FFF77BFF204600223521B0
:10B57000FFF776FF204600225B21FFF771FF204690
:10B5800010225C21FFF76CFF204620225D21FFF78F
:10B5900067FF20468F225E21FFF762FF012038BD42
:10B5A0005C91FF1F10B4047F4160022CC26002D086
:10B5B00010BC01F0D7BB836810BC184790E80C00A2
:10B5C000F0B41C6859682568164F174E294321604E
:10B5D000164D17491760D66015611160417A154AFA
:10B5E0005C180A3194F8244053F8215002EBC4014E
:10B5F00049680D60017A5C1803EB8101247ECD69F6
:10B6000002EBC40149680D60817A581803EB81038D
:10B6100090F83000596B02EBC002F0BC536819601F
:10B62000704700BF01401F00011000380110007872
:10B6300000001F80284B0100704700BFF0B50C1EB2
:10B64000BDF8146034DBB0F906701919B942C4BFF3
:10B650003B1B1BB2002BA6461CDD002A1146B8BFBF
:10B66000D11D02F00705CC10826A012007FB04E11E
:10B67000A840012E0A44C0B21ED00CD3022E09D11C
:10B68000013B12FA83F3013A12F8011F41409A423A
:10B690001170F9D1F0BDC043013B12FA83F3C0B27F
:10B6A000013A12F8011F014093421170F9D1F0BD27
:10B6B00023441BB20024C6E7013B12FA83F3013A8C
:10B6C00012F8011F01439A421170F9D1F0BD00BF79
:10B6D000F8B50D1E0EDB14461F46064601F03AFB78
:10B6E000A84207DD002C05DB304601F037FBA04205
:10B6F00001DCF8BDF8BD304601F02AFB022853D02A
:10B7000003284BD0012806D16540F3886C40654082
:10B71000013B5D1B2DB2012F03D02AD3022F14D081
:10B72000F8BD002C2246B6F90630B06AB8BFE21D5B
:10B7300042F3CF0202FB035504F00704435D0121ED
:10B7400001FA04F41C434455F8BD002C2246B6F916
:10B750000630B06AB8BFE21D42F3CF0202FB0355C8
:10B7600004F00704435D012101FA04F45C404455F0
:10B77000F8BD002C2246B6F90630B06AB8BFE21D0B
:10B7800042F3CF0202FB035504F00704435D01219D
:10B7900001FA04F423EA04044455F8BD3389013B5B
:10B7A000591B25460CB2B6E7F18832890139013AB6
:10B7B0004D1B141B2DB224B2ADE700BF2DE9F041A3
:10B7C000079E9DF91880089D04461F4600F0C0FFA3
:10B7D0000D4B0E480E4984F83380FF22002F08BF1E
:10B7E0001F4684F82F20002384F8302084F831206D
:10B7F00084F832202060A665E56567626165236292
:10B80000A3622046BDE8F0815C91FF1F80400100EB
:10B810000110013810B50446806A034B236008B15B
:10B8200005F0BAFC204610BD80400100F8B5436A1F
:10B83000DBB190F82C200125AA4083F83B2083F847
:10B840005E5083F85D500446406A03680E461B68EC
:10B8500000219847606A036831461B68984729466B
:10B86000606ABDE8F840FFF7E5BBC26BC56C1368C2
:10B87000046A23EA050313604CB122684FF00043C9
:10B88000D3625163D36A002BFCDA936BF8BD836BF0
:10B89000466B0825802410E03768426C3A433260DA
:10B8A0001F68826C3A431A601A68876C013D22EA6D
:10B8B00007024FEA54041A6007D02142ECD13268E3
:10B8C000476C22EA07023260EAE7F8BD70B5044629
:10B8D000406A0D4600282BD0A16DFFF749FA002DD4
:10B8E00020460CBFA621A721FFF7A0FF606A20B168
:10B8F000E16DBDE87040FFF73BBA216C226D08682E
:10B90000236A02430A6093B1DA7A82B1D00703D581
:10B91000224A99691160DA7A910703D5204AD969D8
:10B920001160DA7A520702D51E4A1B6A136070BD95
:10B93000236A002B2BD0D97A626DE1B172B6D97A25
:10B94000CE0706D51848D96806683140996101606C
:10B95000D97A880706D51548196906683140D96132
:10B960000160D97A4E0705D51148596906683140FA
:10B970001962016062B61B68D968914207D00D4810
:10B9800018600D49DA6042F0804018611960226C3D
:10B99000216D136823EA01031360A0E700E100E0D2
:10B9A00004E100E008E100E080E100E084E100E083
:10B9B00088E100E001403F0000003F80436A2DE93C
:10B9C000F04105460E469046002B3ED090F82C10D4
:10B9D0000124A14083F83B1083F85E4083F85D406A
:10B9E000406A036800211B6808F1FF379847FFB2DF
:10B9F000B8F1000F23D03744A046013E686A16F81C
:10BA0000011F03681B6898470134B742E4B216D09F
:10BA1000202CF3D10121686AFFF70CFB95F82C204C
:10BA20006B6A520083F83B2083F85E8083F85D8068
:10BA3000686A036800211B6898470124DEE7686A8A
:10BA40000121BDE8F041FFF7F5BAC26BC16C136884
:10BA500023EA010306EB080413604FF00048A642F6
:10BA60000ED02B6A16F801EB63B11A68C2F82C806D
:10BA7000C2F834E0D36A002BFCDAA642936BF0D113
:10BA8000BDE8F081AB6BD5F834C008208021DCF82C
:10BA900000206F6C1EEA010F14BF3A43BA43CCF882
:10BAA00000201A68AF6C3A431A601A68AF6C01380C
:10BAB00022EA07024FEA51011A60E8D1CFE700BF3E
:10BAC00070B50446406A0D46002828D0A16DFFF7E6
:10BAD0004FF920462946FFF7A9FE606A20B1E16DC3
:10BAE000BDE87040FFF744B9216C226D0868236AF5
:10BAF00002430A6093B1DA7A82B1D00703D5234AB0
:10BB000099691160DA7A910703D5214AD9691160E0
:10BB1000DA7A520702D51F4A1B6A136070BD236A86
:10BB2000002B2BD0D97A626DE1B172B6D97ACE07EB
:10BB300006D51948D9680668314099610160D97AFB
:10BB4000880706D51548196906683140D961016032
:10BB5000D97A4E0705D512485969066831401962ED
:10BB6000016062B61B68D968914207D00D48186021
:10BB70000D49DA6042F0804018611960226C216D35
:10BB8000136823EA01031360A3E700BF00E100E0AC
:10BB900004E100E008E100E080E100E084E100E091
:10BBA00088E100E001403F0000003F802DE9F041C6
:10BBB000044686B0806A9DF830801E460F461546C2
:10BBC000B4F90830002800F04281DA1D48BF03F1C3
:10BBD0000E02B4F90630D21003FB02F2002105F088
:10BBE000FFFDB4F90820202A00F39280B4F9061072
:10BBF000A34B0120203A733902EBD27201EBD171D1
:10BC00004FF0200E029073208DE8014042F34F0266
:10BC100041F34F01204600F051FE606A84F82D7018
:10BC2000002800F04D81002D40F08A80B4F90830E2
:10BC3000202B14BF3D253C2584F82C50B8F1000F73
:10BC400040F0858006B394F93300002818DBC0B2B9
:10BC5000012102F0E7F8012194F8330002F0CEF858
:10BC6000012002F007F9002194F8330002F0C6F831
:10BC70000A2002F0FFF8012194F8330002F0BEF828
:10BC8000606A002800F08280A16DFFF771F804223D
:10BC90007C492046FFF792FE217A0139C9B220463D
:10BCA000FFF7C4FD784904222046FFF787FE94F988
:10BCB0002D30012B14BF142110212046FFF7B6FDB3
:10BCC000042272492046FFF779FEB4F90630802B32
:10BCD00000F09280602B00F0A680D9212046FFF76B
:10BCE000A5FD94F92D30012B14BFF121222120460E
:10BCF000FFF79CFD204606226549FFF75FFE606A5C
:10BD000050B3E16DFFF734F8012006B0BDE8F081D3
:10BD1000B4F906105F4B0120403A52394FF0400E03
:10BD2000029002EBD272522001EBD1718DE80140FA
:10BD300042F34F0241F34F01204600F0BFFD6CE794
:10BD40006DB284F82C50B8F1000F3FF47BAFFEF7D2
:10BD5000C5FF002E94D076E7216C226D0868236A17
:10BD600002430A6073B1DA7A62B1D00703D54A4A56
:10BD700099691160DA7A91077CD4520702D5474A53
:10BD80001B6A1360012006B0BDE8F081236A002B16
:10BD90002BD0D97A626DE1B172B6D97ACF0706D5C8
:10BDA0003F48D9680568294099610160D97A8E07B2
:10BDB00006D53C48196905682940D9610160D97ADE
:10BDC0004D0705D538485969056829401962016051
:10BDD00062B61B68D968914207D03448186034496C
:10BDE000DA6042F0804018611960226C216D13689E
:10BDF00023EA010313604AE7B4F90830202B00F06E
:10BE00008680402B7FF469AF2A4920460322FFF742
:10BE1000D5FD94F92D30012B14BFCF219F21204651
:10BE2000FFF704FD59E7B4F90830102B7FF455AF44
:10BE3000214920460322FFF7C1FD94F92D30012B43
:10BE400014BFAF2110212046FFF7F0FC45E7DA1DB3
:10BE500048BF03F10E02B4F90630D21003FB02F220
:10BE60001046059205F090F9A06200283FF44DAF0E
:10BE7000059AB3E6114AD9691160DA7A7DE700BF05
:10BE8000D8400100B8420100BC420100C04201009C
:10BE9000C4420100CC42010000E100E008E100E002
:10BEA00080E100E084E100E088E100E001403F0043
:10BEB00000003F80D44001008C45010004E100E017
:10BEC000012194F83100244F01F0ACFF94F83200C6
:10BED000012101F0A7FF94F9312094F9323057F88D
:10BEE0003220E26357F83330206A23640125E56489
:10BEF00025651A682A431A6078B1B8F1000F3FF43B
:10BF000028AFFFF75BFB002E3FF4BAAE9BE604229E
:10BF100012492046FFF752FDDFE6294694F82F002C
:10BF200001F080FF294694F8300001F07BFF94F97E
:10BF30002F2094F9303057F83220626357F83330AD
:10BF40006564A5641A68A36322F001021A60002EDA
:10BF50003FF496AE77E600BF284B0100D0400100C9
:10BF6000B0F90820D31D48BF02F10E03B0F9062036
:10BF7000806ADB1002FB03F2002105F031BC00BF38
:10BF8000F0B50029BDF814502EDBB0F90660B142BF
:10BF90002ADA002A59DBB0F9087014461C44BC4266
:10BFA000C4BFBB1A1BB2002B1EDDD2B2D408D0F81E
:10BFB00028E016FB041112F00702DBB20EEB0104BD
:10BFC00021D0C2F10807FAB2374F9342BF5C0CD2BE
:10BFD000C3EB020CFF2646FA0CF6012D07EA060712
:10BFE0003FD005D3022D36D0F0BD012D39D030D24F
:10BFF0001EF8016026EA07070EF801709342F3D39A
:10C00000B0F906100C449A1AD2B2072A10D9022DA0
:10C0100036D0002D14BFFF26002613462670083B9D
:10C02000B0F90610DBB2072B0C44F7D802F0070278
:10C03000002AD9D01D4B012D9B5C1DD017D3022D9A
:10C04000D2D1227853402370F0BD13441BB200229A
:10C05000A1E7022D25D11EF8016077400EF801708E
:10C06000CCE71EF8016037430EF80170C6E722786E
:10C0700022EA03032370F0BD227813432370F0BD3E
:10C0800011462378DB4323700839B0F90630C9B272
:10C0900007291C44F5D812F00702A5D0034B9B5C7E
:10C0A000CFE73444AFE700BF7040010060400100BB
:10C0B00070B4C47DBDF80C50022C18D0032C1FD0D6
:10C0C000012C0BD0002A03DBB0F90840944201DCBC
:10C0D00070BC7047039570BCFFF7B0BAC488039575
:10C0E000013CA41A0A4621B270BCFFF749BF068979
:10C0F000C488013E641AB21AE41A12B221B2E1E70E
:10C1000004890395E41A641A114622B270BCFFF741
:10C1100037BF00BF70B4C57DBDF80C60022D1AD0CA
:10C12000032D12D0012D03D0039670BCFFF728BF5A
:10C13000C488E41AA41A0A4621B2002A03DBB0F923
:10C140000840944213DC70BC70470489013C641AB7
:10C15000114622B2F1E7C48805890396013CAD1A65
:10C16000ED1A621A11B22AB270BCFFF709BF03962A
:10C1700070BCFFF763BA00BF2DE9F8430446406A7C
:10C18000002863D0A16DFEF7F3FD05227449204617
:10C19000FFF714FCA1790139C9B22046FFF746FB2D
:10C1A000B4F90820E588A66AD31D48BF02F10E0342
:10C1B000DB10626A15FB03F51FFA85F8002A7BD0B5
:10C1C00094F82C300125AB4082F83B3082F85E5069
:10C1D00082F85D50606A036840211B6808F1FF37F0
:10C1E0009847BFB2B8F1000F23D03744A846013EAC
:10C1F000606A16F8011F03681B6898470135B7424B
:10C20000EDB216D0202DF3D10121606AFEF712FFA6
:10C2100094F82C20636A520083F83B2083F85E80F8
:10C2200083F85D80606A036840211B689847012598
:10C23000DEE70121606AFEF7FDFE606A002800F07B
:10C240008D80E16DBDE8F843FEF792BD236A002BB7
:10C250002BD0D97A626DE1B172B6D97ACE0706D504
:10C260004048D9680568294099610160D97A8D07ED
:10C2700006D53D48196905682940D9610160D97A18
:10C28000480705D539485969056829401962016090
:10C2900062B61B68D968914207D0354818603549A5
:10C2A000DA6042F0804018611960226C216D1368D9
:10C2B00023EA0103136068E7E26BE36C1168276A05
:10C2C0000B4306EB080913604FF0004E4E450DD0AE
:10C2D00016F801CB2FB33A68C2F82CE0C2F834C08C
:10C2E000D36A002BFCDA4E45936BF1D1226C236D9F
:10C2F00011680B43136097B1FB7A83B1D90703D55B
:10C300001D4BBA691A60FB7A9A0703D51B4BFA6971
:10C310001A60FB7A5B0702D5194B3A6A1A60BDE8CE
:10C32000F883A36BD4F8348008208021D8F800204B
:10C33000656C1CEA010F14BF2A43AA43C8F8002009
:10C340001A68A56C2A431A601A68A56C013822EA9B
:10C3500005024FEA51011A60E8D1B7E7276AC5E73D
:10C360006840010080E100E084E100E088E100E055
:10C3700001403F0000003F8000E100E004E100E0F8
:10C3800008E100E02DE9F04F85B09946BDF938701D
:10C39000BDF83CA0BB1AC1EB090B002BB8BF5B4238
:10C3A000BBF1000FB8BFCBF1000B5B450D46164645
:10C3B0000093804648DC4D453A4633464CDC1946EE
:10C3C00013460A46C5EB09019B1A89B2002B0CB231
:10C3D000B8BF5B4204EBD474BE42ACBF4FF0FF3237
:10C3E00001224D45039102924FEA640429DC9BB27D
:10C3F00001930DE0D8F80070BF69B847019BE41ABB
:10C40000A3B21CB20135002C2DB211DBA94518DBFB
:10C41000009B5B452A46534631464046EADCD8F845
:10C42000002053469769294632464046B847E5E71B
:10C43000029A1644039AA94502EB030436B224B2C9
:10C44000E6DA05B0BDE8F08F4A462B46B9463546D8
:10C450004D4517461E46B2DD304629463E464D46FE
:10C4600007468946AEE700BF10B404682469A446B5
:10C4700010BC604730B40468BDF808500295A46B46
:10C48000A44630BC604700BF30B40468BDF8085013
:10C490000295E46BA44630BC604700BF70B40468EA
:10C4A000BDF90C60BDF8105003960495246CA446A9
:10C4B00070BC6047704700BF10B582B0B0F90C2067
:10C4C00001910168009200220C6CB0F90A3011460B
:10C4D000A04702B010BD00BF704700BF01F00301CC
:10C4E0000129C17506D0032904D0C288038942817D
:10C4F000838170470289C38842818381704700BF6E
:10C500002DE9F0410568134E6F6986B0B7420446C5
:10C51000BDF8308010D1013B13441BB20093CDF81D
:10C5200004800B46AD6A2046A8472368DB6AB34205
:10C530000AD106B0BDE8F081059304920391B84793
:10C5400003A925680EC9E6E7204606B0BDE8F0411C
:10C55000184700BFB5C400002DE9F0410568124E30
:10C560006F6986B0B7420446BDF830800FD1013BF9
:10C57000CDF804800B4400921BB2AD6A2046A84758
:10C580002368DB6AB3420AD106B0BDE8F0810593A7
:10C5900004920391B84703A925680EC9E7E720462E
:10C5A00006B0BDE8F0411847B5C400002DE9F04FD2
:10C5B0000568DFF858B06F6985B05F450646BDF97C
:10C5C0003890BDF83CA00C46904615D11F19BC42CE
:10C5D0000CDACDF800A0214601342D6A4B464246C4
:10C5E000304624B2A847BC423568F2DBEB6A5B45B3
:10C5F00007D105B0BDE8F08F0393B8473568039BBA
:10C60000E4E7304605B0BDE8F04F1847B5C4000078
:10C610002DE9F04387B099420546BDF93840BDF891
:10C620003C6025D0A24212D00768DFF88080D7F89E
:10C630001490C14532D18DE850002846BC6AA0470D
:10C640002B68DB6A434524D107B0BDE8F0839942EB
:10C6500002DD08461946034628680E96C46B01336E
:10C660005B1A1BB22846A44607B0BDE8F0436047FA
:10C67000A24202DD134622461C4628680E96631C21
:10C68000846B9B1A1BB22846A44607B0BDE8F04352
:10C690006047284607B0BDE8F04318470593049269
:10C6A0000391C84703A92F680EC9C4E7B5C40000A9
:10C6B0002DE9F04FD0F800E0DFF89090DEF814B0EC
:10C6C00083B0CB450446BDF93080BDF834A00D469B
:10C6D00017461E4631D1CDF800A0DEF824B0294619
:10C6E00033463A462046D8472368CDF800A008F1E3
:10C6F000FF323A44D3F824B0294612B233462046DA
:10C70000D8472368CDF800A02946D3F820B03A4690
:10C7100043462046D8472068CDF800A0711E294422
:10C720004346056A09B23A462046A8472368DB6AB1
:10C730004B4506D103B0BDE8F08FD847D4F800E0F0
:10C74000C9E7204603B0BDE8F04F1847B5C4000064
:10C75000F0B4002401264FF6FF75094F07600471FD
:10C76000C475C48104824476C46186750676858268
:10C770004582C180028141818281F0BC704700BF47
:10C78000984501002DE9F04F85B00668BDF844508A
:10C79000BDF93880CDF8008004460195D6F848B040
:10C7A0000392BDF93C60BDF9407089469A46D8476E
:10C7B00023680195009742465146D3F848802046A9
:10C7C0003346C0472068039B0E930F95856C4B46FC
:10C7D0003A4631462046AC4605B0BDE8F04F6047CA
:10C7E0002DE9F04F87B01746BDF94040009125462E
:10C7F000E91D059344BF2B4603F10E010268BDF805
:10C80000486053690294C91003912B49BDF9444013
:10C8100001968B42824645D1002C3CDD029B3C4474
:10C820005E1EB6B24FF0000923B2049301364D46A6
:10C83000029B002B28DD059B002403EB090806E082
:10C84000EDB22B0604F1010411D4A6421CD0A1B212
:10C8500011F0070F23B24FEA4505F1D1002BB8BF05
:10C860000733DB10013418F803502B06EDD5009B7D
:10C87000D2F818B019443A4609B2019B5046D8473D
:10C88000A642DAF80020E2D1039B01379944049BC9
:10C890003FB2BB42CCD1D36A074A934206D107B01C
:10C8A000BDE8F08F9847DAF80020B5E7504607B0AA
:10C8B000BDE8F04F184700BFB5C4000070B4BDF923
:10C8C0000C60BDF91050BDF8144003960495059412
:10C8D00070BCFFF785BF00BF2DE9F04F93B09046C5
:10C8E0000591C1691090BDF870000790BDF8749073
:10C8F0009DF878A00493002900F0CD800A7A0AC937
:10C90000894604998A1AD2B203EBC203BAF1010F25
:10C91000DA780B9293F905201E8893F802B00F92F3
:10C9200093F9064079D913B2099323B20C93109B63
:10C930001A68A94B1193194653698B4240F0A6809F
:10C940000B9B002B55D01FFA88F300210D93C8468E
:10C950002344DDF8409006910E930F460C46BBF140
:10C96000000F3FD0BDF818100C9B03971FFA8AF0F8
:10C97000CB1813FB00F304900E9801440D98034468
:10C9800009B21BB20A910893002505E00135EBB20C
:10C9900064009B45E4B222D9039B2B44590703D181
:10C9A000731C18F806409EB22306EFD5099BBDF80C
:10C9B0001000E91811FB00F10598BAF1010F0FFA08
:10C9C0008AF301441CD0079801900093D26909B200
:10C9D00017464846089AB847D9F80020D6E7039F7B
:10C9E0005F44FFB2069B0B9901330693DBB2994279
:10C9F000B5D8D36A119A934243D113B0BDE8F08FF2
:10CA00000F9B191893690A9A29441F4609B2079B7C
:10CA10004846B847D9F80020B8E700230C9309939B
:10CA200085E70A9A0D9B0132013B52B213F0FF03D6
:10CA30000A920D936FD1DDF81890079BDDF83C80CA
:10CA4000DDF820A04B4517D0BAF1010F00F0C880E7
:10CA50000B9A109DCDF804900BEB8B014FEACB03A2
:10CA60000A4400931146DEF81C405346424609B280
:10CA70002846A047D5F800E0DEF82C30119A934202
:10CA8000BBD0109813B0BDE8F04F1847109D284652
:10CA900098472A6854E7109A0598B2F90A308342F9
:10CAA000ABDDB2F90C304345A7DD062313FB0A03C7
:10CAB000002BA2DD08EBCA03002B9EDD537E2BB9B1
:10CAC000049BAF2B02D90133DBB20493109BD3F844
:10CAD00000E0414B11931A46DEF81430934240F0C7
:10CAE0008E801FFA88F30E9308339BB2BDF8142092
:10CAF000059305230D9300230A93CDF83C800FFA8C
:10CB00008AF3DDF84080CDF818900B921FFA8AFB6B
:10CB1000CDF820A099460A9ABDF810000B9C0E9DF6
:10CB20000523194611FB00232C481146C75C0397C7
:10CB300002FB0B4214FA81F312B21BB209920C935E
:10CB40002C462E461CE0089B0999012B2AB24B4625
:10CB500040462DD0079F0197CDF80090DEF81CA02D
:10CB6000D047D8F800E0039B5B0801340393059B92
:10CB7000A4B25D445E44A342ADB2B6B23FF451AF3D
:10CB8000039BD807DFD4079B069A9342EBD0089B00
:10CB9000012B16D0069B0193CDF80090DEF81CA067
:10CBA00009994B4632B24046D047D8F800E0DAE760
:10CBB000DEF818A0079B0C9922B2D047D8F800E005
:10CBC000D1E7DEF818A00C991346404622B2D047B0
:10CBD000D8F800E0C7E700BFB5C40000E845010091
:10CBE0000B99109DCDF800900531DEF8204009B278
:10CBF000424608232846A047D5F800E03CE7109CB1
:10CC000020469847D4F800E06BE700BFF0B5C36951
:10CC100085B004462BB30A2968D00D294AD01A7A68
:10CC2000914247D3587A884244D35D688A1A05EB0B
:10CC3000C205AA78002A50D0E87800284DD0207E7E
:10CC400000283AD095F905E0B4F90E00A67DB4F9B4
:10CC50000A70724406FB0202BA4262DCB4F9102088
:10CC600030E00A2956D00D2924D0027E002A4BD06C
:10CC7000B0F90E00A57DB4F90A60062212FB050288
:10CC8000B2423EDD228AE38102EBC50212B21846AF
:10CC90002282A78A668A02950B468DE8C00001466B
:10CCA0002046FFF719FEA37DE28903EB430302EB65
:10CCB0004303E381012005B0F0BDA67DB4F90E0069
:10CCC000B4F91020B4F814E0678A02960B468DE898
:10CCD000804001462046FFF7FFFD2979E389A27DC8
:10CCE000012001FB0233E38105B0F0BD0022C281C7
:10CCF0009A7A817D038A01FB02330382012005B009
:10CD0000F0BDB4F91020C4E7857DB4F91020B0F966
:10CD10000E00BEE7028A817DC38102EBC10303825C
:10CD2000C8E70020E0819B7A228A03FB062212B228
:10CD30002282C7E7C1810282704700BF002908BF75
:10CD400001218175704700BF81824182704700BF19
:10CD5000C07D7047B0F90A00704700BFB0F90C0001
:10CD6000704700BF10B4EFF3108272B6437F33B93F
:10CD7000017F012907D003290FD00123437702B98E
:10CD800062B610BC7047124C2168A1B111494361D1
:10CD90000B68836108605861EFE70F4C216881B12F
:10CDA0000E4943610B688361086058610C4B4FF07A
:10CDB00080511960E1E7074B416181612060186093
:10CDC000DBE7064B4161816120601860EEE700BF40
:10CDD00014A0FF1F10A0FF1F04A0FF1F08A0FF1F2B
:10CDE00004ED00E070B5EFF3108272B60C4C2068D1
:10CDF00080B10C4E00254369236073B19D6102B977
:10CE000062B6457783689847EFF3108272B6206860
:10CE10000028F0D102B962B670BD3360EFE700BF01
:10CE200004A0FF1F08A0FF1FFFF7DCBF184A30B4A3
:10CE30001468002C27D0036821688B420ED2CB1ACD
:10CE400000218460C1602360E060106002230375EC
:10CE500030BC704711688B42144608D3A2685B1A35
:10CE60000360002AF6D18260C460A060EEE7D26859
:10CE7000C2608460E060C568CB1A0222A8602360AB
:10CE8000027530BC70478460C4601060DEE700BF8C
:10CE90000CA0FF1FF8B5224E34682CB32368002B7A
:10CEA0003AD1204F1D4604E03468ECB12368002BD2
:10CEB00032D1A36803B1DD60206933600368257552
:10CEC0001B68BB4221D1037F4560022BC46020D088
:10CED000FFF748FF6368002BE6D023602046FFF78A
:10CEE000A5FF3468002CE1D1EFF3108372B60E4A2F
:10CEF00000211068116003B962B628B18468FFF799
:10CF000095FF20460028F9D1F8BD22460021984718
:10CF1000E0E783689847DDE7013B2360E4E700BF73
:10CF20000CA0FF1FA5B500001CA0FF1F024A13683C
:10CF300001331360FFF7AEBF28A0FF1F704700BF8B
:10CF40000368F0B4FBB1002501249D60DC601B4C3C
:10CF50001A601C44241104F144056A11032692004E
:10CF60009E60174F0679174B47F8241002F1604274
:10CF700002F5614205F01F05012000FA05F5E654AF
:10CF80001560F0BC7047104C236843F40003236025
:10CF900000BF0E4B0E4DA4F58734A4F59E740126F8
:10CFA0001E60234604609C68002CD0D01033AB4236
:10CFB0000360F8D1002303601846E2E7008FFCBF4E
:10CFC0003492FF1F44E400E03C80044000700340C2
:10CFD000407103400168A9B10B4BF0B40B441B1125
:10CFE0000A4E0B4F0B4D46F8237003F1440202F03A
:10CFF0001F0401235211A340002445F822308C6005
:10D000000460F0BC704700BF008FFCBF3492FF1F6C
:10D010003DCF000080E100E0024A034B0121116096
:10D020001B6818470C7103403492FF1F024A034BE0
:10D03000012111605B6818471C7103403492FF1F87
:10D04000024A034B012111609B6818472C71034071
:10D050003492FF1F024A034B01211160DB6818471D
:10D060003C7103403492FF1FF8B50E4671B17AB19E
:10D070000746144600253B6816F8011B1B68384616
:10D080009847013C0544F6D12846F8BD0846F8BD4E
:10D090001046F8BD00B5064A036812885B6883B085
:10D0A00001A9ADF804200222984703B05DF804FB03
:10D0B000E84A0100F0B507468BB0002A33D0012AB8
:10D0C00008BF0A2251B3212400E0F4B2B1FBF2F50B
:10D0D00002FB1511C8B2092900F1300198BFC8B28E
:10D0E0000AA988BF3730214488BFC0B201F8240C98
:10D0F000661E2946002DE8D133B1013CE4B20AABEB
:10D1000023442D2203F8242C3B6801AA11195B68E3
:10D110003846C4F1220298470BB0F0BD30228DF89A
:10D1200025202124E8E70368C9B21B6898470BB0A3
:10D13000F0BD00BF0029BABF49422D2300230A22B7
:10D14000FFF7B8BF374A384913681B06FCD40B6891
:10D1500013F08003F8D172B634490A78002A5FD000
:10D16000334A3448F0B4344C176806682568D468EC
:10D170000C303E44143200681268304F35442C4461
:10D1800020440244C2F34E022D4E2E482E4D2F4C09
:10D1900042F400423A60376806682D682C4A2468D9
:10D1A0000C303E44006812682A4F35442C44204419
:10D1B0000244C2F34E02284E2848294D294C42F41D
:10D1C00000423A60376806682D68274A24680C30A8
:10D1D0003E4400681268254F35442C4420440244E4
:10D1E000C2F34E02224E2348234D244C42F4004207
:10D1F0003A60376806682D68214A24680C303E443E
:10D200000068126835442C4420440244C2F34E02A4
:10D210001C4842F4004202600B7062B6F0BC7047DA
:10D2200062B6704724B0034024B00B4021A0FF1F1A
:10D2300038B003403CB0034040B003402CB0034042
:10D2400058B003405CB0034060B0034064B003409A
:10D250006CB0034030B0034038B00B403CB00B40E2
:10D2600040B00B4044B00B404CB00B402CB00B40D6
:10D2700058B00B405CB00B4060B00B4064B00B404A
:10D280006CB00B4030B00B4030B42948294A2A4BCF
:10D290002A4D6024E121047011701B78284C082B62
:10D2A00030D00A2B2748284937D00C2B0CBF352209
:10D2B0003D2212232A60236002600B60234B244925
:10D2C0001B78244ABBB101230B601360224B234916
:10D2D0001B78234A012B26D9042B0FD9082B1ED9E2
:10D2E000102B94BF862387230B6013601D4B0122F4
:10D2F0001A7030BC70470B601360E7E784230B6043
:10D300001360F3E700F58E200F4908300122132344
:10D310002A60236002600B60D0E73922F7E785239B
:10D320000B601360E2E780230B601360DEE700BF51
:10D3300000400740014007404492FF1F08B00340EF
:10D340000CB0034008B00B400CB00B4024A0FF1FF2
:10D3500020B0034020B00B404592FF1F24B0034093
:10D3600024B00B4021A0FF1F0C2830B417D9102384
:10D37000984228BF18461C46104A114D1178181AB9
:10D380008C42287018D00F4913700B7823B10E49C6
:10D390000E4A00230B60136030BCFFF775BF0A28EC
:10D3A00002D90C231C46E7E7082802D90A231C46A9
:10D3B000E2E708231C46DFE730BC70474492FF1FBA
:10D3C00020A0FF1F21A0FF1F24B0034024B00B406A
:10D3D00028282FD8334B2DE9F0411E5CFF2E2BD08F
:10D3E000314B1B78002B2AD132062CD472B62F4D2C
:10D3F0002F4C2F46012326602B7062B672B623682D
:10D400001B060CD43B781BB9F4E72B78002BF1D02A
:10D4100062B602F073FB72B623681806F5D5254B89
:10D420001B6800222A7062B6234A107843FA00F083
:10D43000BDE8F081002070470020BDE8F081FFF7D3
:10D4400081FE3206D2D572B61C4DDFF87C801C4CB2
:10D4500006F04007FFB206F03F06D8F80030DFB113
:10D4600023F01003C8F8003001232660134A2B7004
:10D4700062B672B6236819060CD413781BB9ECE7B0
:10D480002B78002BE9D062B602F038FB72B6236825
:10D490001B06F5D50B4BC3E743F01003C8F800306B
:10D4A000E2E700BFEC4A010021A0FF1F23A0FF1FFD
:10D4B00000B0034010B0034020A0FF1F22A0FF1FB8
:10D4C00000B00B4010B00B400CB00B400A4A0B49A7
:10D4D000136843F4805313600B7843B9084BC022A0
:10D4E0001A70084B80F30C0000B218807047044B90
:10D4F00080221A70F5E700BF2C80044024A0FF1F93
:10D5000021C00C4000C00C40F0B51B4B1B4E5968AD
:10D5100018689A68DB6885B06C460FC43378990741
:10D520001DD5174A174C1378174913F0700318BF0D
:10D530001370164A164B80271770002633200322DB
:10D5400026706D4608701A7072B6043C45F00105ED
:10D550002046A84762B6237813F0700309D10D4B1B
:10D56000064901E0013B02D00A78D207FAD505B09E
:10D57000F0BD237005B0F0BD184B01000100024062
:10D5800000000240040002400B000240070002407D
:10D590000A000240410D0300B0F5006F0AD210B539
:10D5A000094B1B78DB07044606D504F1A050007830
:10D5B000C0B210BD00207047FFF7A6FF04F1A050D5
:10D5C0000078C0B210BD00BF01000240B0F5006F8E
:10D5D00017D238B50F4B1B78DA070D46044611D524
:10D5E00004F1A0500378AB420AD00B4A137813F031
:10D5F000700318BF1370074A05701378DB07FCD55A
:10D6000038BD7047FFF780FF04F1A0500378AB42AC
:10D61000EBD1F5E7010002400000024008B5F4F745
:10D6200011FBF4F779FF02F069FAFAE7844641EA60
:10D63000000313F003036DD1403A41D351F8043B8A
:10D6400040F8043B51F8043B40F8043B51F8043BDC
:10D6500040F8043B51F8043B40F8043B51F8043BCC
:10D6600040F8043B51F8043B40F8043B51F8043BBC
:10D6700040F8043B51F8043B40F8043B51F8043BAC
:10D6800040F8043B51F8043B40F8043B51F8043B9C
:10D6900040F8043B51F8043B40F8043B51F8043B8C
:10D6A00040F8043B51F8043B40F8043B51F8043B7C
:10D6B00040F8043B51F8043B40F8043B403ABDD2EB
:10D6C000303211D351F8043B40F8043B51F8043B8D
:10D6D00040F8043B51F8043B40F8043B51F8043B4C
:10D6E00040F8043B103AEDD20C3205D351F8043B1C
:10D6F00040F8043B043AF9D2043208D0D2071CBFE8
:10D7000011F8013B00F8013B01D30B880380604610
:10D71000704700BF082A13D38B078DD010F0030386
:10D720008AD0C3F10403D21ADB071CBF11F8013BF6
:10D7300000F8013B80D331F8023B20F8023B7BE745
:10D74000043AD9D3013A11F8013B00F8013BF9D270
:10D750000B7803704B7843708B788370604670470A
:10D7600008B5104C08E0236859050DD423681A0544
:10D770000FD42368DB0411D423685803F3D501F0D8
:10D7800065F823685905F1D502F01CFA23681A05DB
:10D79000EFD500F07FFD2368DB04EDD500F0C8FE77
:10D7A000EAE700BF3480044008B5FFF7D9FF00BFA7
:10D7B000014B10221A80704700200540704700BFBF
:10D7C000094908B50B6830B16A461844A2F5805281
:10D7D000904202D20860184608BD03F0A7FC0C2353
:10D7E00003604FF0FF3008BD4892FF1FFEE700BF07
:10D7F000EFF3138070B9EFF310836BB9EFF3058289
:10D800005AB94FF48070EFF311832BB1984228BFBF
:10D81000184670474FF0FF3070470F2A01D818465E
:10D82000F1E7014BD05CEEE7F0E300E0F0B44D1E11
:10D830002E46002400E00134B0FBF2F302FB13009B
:10D84000092800F130078ABF3730F8B2C0B206F8B5
:10D85000010F1846002BEED10A1953704CB1107805
:10D8600015F8016F28700133E01A834202F801694C
:10D87000F5DB0846F0BC7047704700BF10B40F4B93
:10D8800053F8302092F880422CB1012369B182F81C
:10D89000803010BC704703EBC0035B681A6841B965
:10D8A00022F002021A6010BC704782F8003110BCEE
:10D8B000704742F003021A6010BC7047284B010009
:10D8C0001C4A02EBC00301295B6811D004291BD05C
:10D8D00052F83000002280F8802229B1022920D09D
:10D8E000032922D01A6070474FF480721A60704783
:10D8F00052F830004FF4A27280F880121A601A6851
:10D9000022F020021A60704752F830104FF4A272D1
:10D91000012081F880021A601A6842F020021A6021
:10D92000704740F203121A6070474FF481721A6018
:10D93000704700BF284B0100212848D8F8B5042AB9
:10D9400044D8DFE802F0484B4E0345004FF4102660
:10D950002B4B03EBC0030D465C68216811F4E061BA
:10D9600048D0284B284A2949C3F89C2104F1404259
:10D970002748C3F8A411A2F59221264FC3F8A001AD
:10D980007C292548C3F8A871C3F8AC012CD9A2F5AD
:10D9900094237C2B2AD9A2F596237C2B28D9A2F597
:10D9A00098237C2B29D9A2F59A227C2A27D81B48B8
:10D9B00072B6236823F4702343F08072C4F38401A9
:10D9C0001643236040F82150266062B6F8BD7047C8
:10D9D0004FF43026BCE74FF40026B9E74FF4402659
:10D9E000B6E74FF42026B3E70D48E1E70D48DFE73F
:10D9F0000D48DDE7FFF764FFB3E70C48D8E7F8BD53
:10DA0000284B01000082FF1FF188FF1F9988FF1F2C
:10DA1000C588FF1F6D88FF1F4188FF1F2493FF1FCC
:10DA20004C92FF1F8492FF1FD492FF1F0493FF1F8D
:10DA30001A4B03EBC00010B4426802F14043A3F557
:10DA400092217C2923D9A3F594217C290DD9A3F512
:10DA500096217C291FD9A3F598217C2919D9A3F5F2
:10DA60009A237C2B11D80E4C00E00E4C72B6136832
:10DA70000D4823F08773C2F3840123F4803343F00D
:10DA80008073136044F8210062B610BC7047074CE5
:10DA9000ECE7074CEAE7074CE8E700BF284B01003A
:10DAA0002493FF1F8492FF1F79D800004C92FF1F20
:10DAB0000493FF1FD492FF1F30B4054B054D064C55
:10DAC000002210211A602A602060196030BC704763
:10DAD00014D0034004D0034000D00340282838B5B8
:10DAE0002ED0002904464FDD5F4B1B78012505FA37
:10DAF00003F28A4202D8212837D938BD0338C2B28E
:10DB0000012A3AD9202C4AD0192C48D0574A1268F9
:10DB100002FB011222FA03F31D2800F29B80DFE8CA
:10DB200000F0928B847D9999766F9999999999993A
:10DB300099999968615A53994C99999999999945E4
:10DB4000494B1B780B2B08D90C2B1CBF0C3B1941E4
:10DB50000846BDE83840FFF7B9BCC3F10C03994053
:10DB60000846BDE83840FFF7B1BC2946FFF786FEFE
:10DB70002946BDE83840FFF7A3BE3D4A126802FBC4
:10DB8000011222FA03F3C7E72128B6D80021FFF7D4
:10DB900075FE20460121BDE83840FFF791BE354AA9
:10DBA000126802FB011222FA03F3B5E73249334A45
:10DBB0000B604FF45173136038BD3149314A0B602B
:10DBC0004FF45173136038BD2F49304A0B6040F257
:10DBD0004443136038BD2E492E4A0B6040F2444343
:10DBE000136038BD2C492D4A0B6040F2444313604A
:10DBF00038BD2B492B4A0B6040F24443136038BDBB
:10DC000029492A4A0B6040F24443136038BD284931
:10DC1000284A0B6040F24443136038BD2649274A26
:10DC20000B6040F24443136038BD2549254A0B6020
:10DC300040F24443136038BD2349244A0B604FF43B
:10DC40005173136038BD2249224A0B604FF451735F
:10DC5000136038BD212C3FF650AF7F29D4BF00217F
:10DC60000121204693E700BF2C93FF1F088003404B
:10DC70000890034008800B4010800B4048A00440EF
:10DC800018800B404CA004401880034008B00440AA
:10DC90001080034004B004404080034018C004409A
:10DCA0003880034014C004402880034010B0044072
:10DCB000208003400CB004403080034010C004407A
:10DCC000488003401CC00440189003403490044036
:10DCD000109003403090044038B1102828BF102025
:10DCE000044AC3B2107813707047024A01231078B7
:10DCF000137070472C93FF1F2DE9F8430E468046A2
:10DD00003249334D304603F097F947F61223002885
:10DD10001ABF1D464FF002094FF00109002425FAF1
:10DD200004F002F093FF4FF05E51074602F0E6FF69
:10DD30000146304603F094F930B90134072CEED196
:10DD4000E80902F083FF07463146384603F08AF8B7
:10DD50004FF07C5102F0C8FE03F0BCF94FF6FF72A1
:10DD60009042A8F1030328BF1046012B29D9B8F12E
:10DD7000170F17D8174B23FA08F303F0010383F0AA
:10DD8000010223B9B8F1190F0FD0BDE8F883124B87
:10DD9000124D13491A6044EAC9042A6008601C60E5
:10DDA000BDE8F883B8F1200FECD10E4B0E4D0F49B2
:10DDB000002244EAC9041A602A6008601C60BDE8B9
:10DDC000F8830B4B0B4D0C49F2E700BF001BB7402B
:10DDD000006CDC026006F000008003400480034019
:10DDE0000880034000800B4004800B4008800B40FB
:10DDF000009003400490034008900340212801D87C
:10DE0000FFF73CBD704700BF212806D8044B53F8EC
:10DE1000303093F80002C0B270470020704700BF56
:10DE2000284B0100212801D8FFF74ABD704700BFE9
:10DE300072B60C490C4B0D4A1B680868126862B632
:10DE4000520102D5322B88BF01300949C3F5BB33DB
:10DE50004FF47A72FF33A1FB031302FB00F000EBD7
:10DE60009310704728A0FF1F18E000E004ED00E0C9
:10DE7000ABAAAAAA2DE9F843054672B6204F214B5A
:10DE8000214A1B683C68126862B6520102D5322BE7
:10DE900088BF013495B3C3F5BB331C4EDFF86490E3
:10DEA000DFF86480FF334FF47A72A6FB031302FBA2
:10DEB00004F404EB931472B6D9F800103A68D8F859
:10DEC00000E062B6C1F5BB33FF33A6FB03031EF0CF
:10DED000806FC4EB93134FF47A7002D0322988BF5D
:10DEE000013200FB0233B3F57A7F04D3013D05D044
:10DEF00004F57A74DFE701F001FEDCE7BDE8F883A2
:10DF000028A0FF1F18E000E004ED00E0ABAAAAAAD9
:10DF1000F8B52D4B2D49DFF8D0E0DFF8D0C02C4EFE
:10DF20002C4D2D4C2D4A2E4F4FF4000018604FF011
:10DF3000807018604FF0007018604FF080601860BB
:10DF40004FF0006018600020086028234BF6FF7136
:10DF5000CCF80010CEF80030336013602B602360E3
:10DF60003B60B3629362092245F8242CC4F8D80FB1
:10DF700005F57F65C7F8D41F07F5FF2707F5FA6792
:10DF8000C6F8F83F2B6006F5FF26C4F8D42F05F538
:10DF9000FD2504F5FF24386006F2F476114831605F
:10DFA00005F5FF6504F5FD642B6023600260FFF753
:10DFB0006BF91920FFF75EFF01F08EF940F21310A4
:10DFC000BDE8F840FFF756BF08E100E004800340D9
:10DFD00014800340248003402C8003401C800340B5
:10DFE0003480034000800B400C80034008800340D5
:10DFF0002B4A2C491368F0B543F4006313600A7888
:10E00000294F2A4E2A4D2B4C2B490023092A3B70BD
:10E0100033702B7023700B703DD01A2A21D0274B00
:10E020001B780A2B25D01F2B30D01F2827D8002083
:10E0300002460125224B234C1A7023495D700422AD
:10E040004FF0020E88273C26402598729A704FF4B4
:10E05000004083F813E05A751F74DE702570086065
:10E06000F0BD1A4B40F213321A60144B1B780A2B86
:10E07000D9D1174B4FF451721F281A60D7D9C0F36A
:10E080004432C0F3471500F01F00D3E7114B4FF4A3
:10E0900051721A60C9E7104B40F213321A60BEE7A2
:10E0A000348004402D93FF1F9CA0FF1F31A0FF1F51
:10E0B000A4A0FF1F9DA0FF1F30A0FF1F2E93FF1FD6
:10E0C00000B006402FE400E004E100E004D004408A
:10E0D00010B0044000D004400CB0044009B140F03E
:10E0E0008000174A1378984216D010B4154C246853
:10E0F00024050FD503F07F030A2B1CD01F2B11D052
:10E10000002900F07F0114BF602344230A290DD0A9
:10E110001F2902D0107010BC70470B4943F44073A4
:10E120000B60F7E7084B00241C60E9E7074943F45C
:10E1300040730B60EEE7054B00241C60E0E700BF76
:10E140002E93FF1F3480044000D0044010B00440E0
:10E15000124B1A7882420CD011490968090507D57B
:10E16000092A16D01A2A0AD009280DD01A2801D057
:10E17000187070470B4A40F213311160F8E7094AF2
:10E18000002109281160F1D1074A40F213311160D2
:10E19000EEE7054A00211160E6E700BF2D93FF1F5F
:10E1A0003480044004D004400CB004402DE9F84F02
:10E1B000234B1B681A053BD5224B1B680BB1012270
:10E1C0001A70DFF89090204D99F80040DFF88880B1
:10E1D0001E4E0134272C8ABF4FF0000A5FFA84FAE2
:10E1E00054460746AB462B789C4216D1FFF700FBFE
:10E1F00040281FDC33791B06F5D59BF8003001332E
:10E20000272B86BF00221346DAB218F80330DBB2A0
:10E21000F3712A702B789C42E8D00D490B4BFFB26A
:10E220000120BC2208F80470087089F800A0DA7098
:10E23000BDE8F88FFF28D6DD01F060FCD3E700BF12
:10E2400034800440A0A0FF1F9DA0FF1F00B0064027
:10E2500030A0FF1FA4A0FF1F34A0FF1F10B5044C67
:10E26000237823B101F04AFC2378002BFAD110BDAA
:10E2700030A0FF1F054A064B10781B78C0B2DBB2F6
:10E28000984238BF4030C01A704700BF9CA0FF1FA3
:10E2900031A0FF1FF0B4384B1A7912F0300F2CD098
:10E2A00072B6997D01F0FF0200293DD062B6334F6E
:10E2B000334938780D78334E1C46C0B2EDB2431C5A
:10E2C000402BE17928BF0023AB4202F1FF32C9B2F3
:10E2D0001CBFF154184612F0FF02F0D12A4B1B6804
:10E2E000C2B23A704BB1A84236BFC5F14005401BDF
:10E2F00040192728C4BF01221A701F49CA78D2B218
:10E30000150616D452060DD51B4B1B795B0609D595
:10E310001E4B1F491B6800220A7003B11A70164B6E
:10E320003C22DA70F0BC70474022D9795A7462B648
:10E33000E3E70B791C06E5D5164B174E1C783378AE
:10E34000E4B2DBB29C420ED0144D01E0A3420AD0ED
:10E350000133282B28BF00230879E85CC0B2C871BC
:10E36000087D0728F2D9DBB2034933700B79180610
:10E3700044BF7C23CB70C5E700B006409CA0FF1FC4
:10E3800031A0FF1F5CA0FF1F2CA0FF1FA0A0FF1F3C
:10E3900030A0FF1FA4A0FF1F9DA0FF1F34A0FF1FE0
:10E3A0002DE9F84F214B1B6807460BB101221A706B
:10E3B000DFF888901E4D99F80040DFF884801D4EEC
:10E3C0000134272C8ABF4FF0000A5FFA84FA5446C2
:10E3D000AB462B78A34216D1FFF70AFA40281FDC80
:10E3E00033791B06F5D59BF800300133272B86BF08
:10E3F00000221346DAB218F80330DBB2F3712A7048
:10E400002B78A342E8D00C490A4BFFB208F80470FD
:10E410000120AC22087089F800A0DA70BDE8F88FFE
:10E42000FF28D6DD01F06AFBD3E700BF1CA1FF1F68
:10E4300019A1FF1F00C0064018A1FF1F20A1FF1F48
:10E44000B0A0FF1F1C4BDFF894C01A681B49F0B541
:10E4500042F480521A4D1A60DFF884E0194F1A4EC8
:10E460001A4C00238CF800304FF451722B701F2887
:10E4700040F213358EF800303B70337025600A602F
:10E4800012D819460124124A124D117012485470C4
:10E4900000212C27402693724FF4003491701174A0
:10E4A000D7702E700460F0BDC0F34431C0F3471440
:10E4B00000F01F03E7E700BF348004400CC00440B5
:10E4C000ADA0FF1F19A1FF1F18A1FF1F08C0044026
:10E4D00000C0064031E400E004E100E0ACA0FF1F12
:10E4E00020A1FF1F034B1B68DB0401D5FFF758BFBA
:10E4F000704700BF3480044010B5044C237823B12A
:10E5000001F0FCFA2378002BFAD110BD18A1FF1FEF
:10E51000054A064B10781B78C0B2DBB2984238BF70
:10E520004030C01A704700BFACA0FF1FADA0FF1F56
:10E5300030B42B4B1A7994061FD52A48DA79037820
:10E54000294901333F2B0978C8BF00238B42D2B23F
:10E5500003D0264CD9B2E2540170254A116861B14A
:10E56000244A1278D2B2934236BFC2F140029B1ABB
:10E570009B18272BC4BF01230B70194AD378DBB239
:10E58000180611D45A060DD5154B1B795B0609D513
:10E59000194B1A491B6800220A7003B11A70104BFC
:10E5A0002C22DA7030BC704711790906EAD514497B
:10E5B00010480C780178C9B28C420DD04A1C272A29
:10E5C00084BF00210A460F4D054C98BFD1B2AA5C0A
:10E5D000D2B2E2710170D5E76C21D170D2E700BFF1
:10E5E00000C00640ACA0FF1FADA0FF1FD8A0FF1FBA
:10E5F000A8A0FF1F19A1FF1F1CA1FF1F18A1FF1F2B
:10E6000020A1FF1FB0A0FF1F21282FD8184B195C95
:10E61000FF292BD0174B184ADFF870C003EBC0005E
:10E62000F0B54368DFF868E0144F154D154E00242F
:10E630001C60DEF80030012043F020038840CEF853
:10E64000003014604FF4A07338602E60C2F800C030
:10E65000013BFDD113689B05FCD42023013BFDD178
:10E66000094B09B233F8110080B2F0BD00207047A9
:10E67000384C0100284B0100005004400850044071
:10E6800004500440000002030051044080014A008D
:10E6900038800440431E032B14D872B60A4951F83F
:10E6A000230068B170B4094C058834F8132046681B
:10E6B00041F82360521B24F8132062B670BC7047E7
:10E6C00062B67047002070477CA1FF1F44A3FF1F64
:10E6D000013803280BD872B6074B53F8203043B1EA
:10E6E00000205B680130002BFBD162B67047002030
:10E6F00070471846F9E700BFD0A1FF1F30B472B6CB
:10E700002B4A13781D0706D52A4B196A002936D0E3
:10E71000996A002941D053781C0706D5254B196CFE
:10E7200000293ED0996C002939D09378190705D576
:10E73000204B196E002936D0996E89B1D3781B070A
:10E7400007D51C4BD3F880207AB3D3F88820112149
:10E750003AB162B6184B00221A7030BC00F04ABEC3
:10E760000D21154C154D227843F8315003EBC103B0
:10E770000830013A5860227062B630BC70470422FB
:10E780000D4C0F4D217843F8325003EBC203083093
:10E790004A1E5860227062B6EFE70521E1E70921C1
:10E7A000DFE70822ECE70C22EAE71022E8E700BFE7
:10E7B0005C4C01000080FF1FF9A1FF1FC800400052
:10E7C00088004000431E032B1DD81B4A400140F027
:10E7D000100030B4104472B6184CE25C032A1BD807
:10E7E000DFE802F00212151703220D88E25410F040
:10E7F000080F14BFC823882343EA05430831036088
:10E80000416062B630BC704708300222EDE7052255
:10E81000EBE708300422E8E7094A52F8230038B150
:10E82000084A52F82300416042F8231062B6E9E733
:10E8300042F82310034AF7E70080FF1F08A2FF1FDA
:10E84000D0A1FF1FE0A1FF1F00BE70472DE9F04FD0
:10E85000DFF818B3DFF818A387B044E0AD4F4FEAF4
:10E86000930807EBC809013ED9F8042003F0080318
:10E87000F6B2A2F1080003F0FF04002B40F0018182
:10E8800057F838301B0C99B222F8081C002B00F006
:10E89000EF80A14B22F8064C42F8044C53F8262096
:10E8A000002A00F0CF819D4D55F8263058609C4CD1
:10E8B00045F8260034F81630194424F8161000F0F4
:10E8C00079FD002800F0C281964A974B19F0080F95
:10E8D00000F1080018BF1346C9F8040047F83830A3
:10E8E00008238BF800309BF80040E4B265071CD584
:10E8F0008E4B1B78B3B18E490A7802F0FF0322B128
:10E90000013BDBB20B7003B900BE8A490A7802F002
:10E91000FF032AB1013BDBB20B70002B00F06881D2
:10E9200000F066FE04238BF8003004F0080303F0C7
:10E93000FF02002B00F0C9809AF80030DBB21E09FC
:10E940008CD19A08DFF8CC9159F8321009EBC2004B
:10E95000C1F38301013940680C2900F28580DFE8AA
:10E9600001F07A7A838383838383468383830700DA
:10E970000168714D4068714F714E6860296088B2BE
:10E9800040F281610024674B49F832304FF0010EAC
:10E9900088423C60C9F81040C9F8184086F800E089
:10E9A0005C4A00F2E780B0F5D06F80F01B82B0F5D2
:10E9B000817F00F0D98100F26981802800F02A82ED
:10E9C000822840F0D781A98801F07F01042900F254
:10E9D000D1815C485C4A8900084414705470017805
:10E9E0008C0740F1608382F800E0022173E1534F0D
:10E9F0003A682AB3554B524E5548198834780578F1
:10EA000040298E4645F0020828BF4FF0400E002CEA
:10EA100084F001043470CEEB01010CBF8824C824BB
:10EA200009EBC80689B285F0010544EA0E4472601C
:10EA3000198049F8384072440570002965D03A6061
:10EA40003D4B1A88B2F5A06F0ED100219A7859700B
:10EA5000404B1A7008E038493F4C0D68A54200F061
:10EA60009880304949F832103C4A0123137037E747
:10EA70002C4A2D4B19F0080F18BF134647F83830B1
:10EA80002EE700F0B7FC364A364952F82630002B04
:10EA900000F0E38058688C5D42F8260003F108021C
:10EAA000C9F80420032C05D8DFE804F02C0229263D
:10EAB00002228A551A8819F0080F0CBF8823C82330
:10EAC00043EA024347F838300AE7E00700F1938051
:10EAD000210600F1D180A20706D5234A23491378E5
:10EAE0000220DBB213700870E30602D51F4B102220
:10EAF0001A7007B0BDE8F08F04228A55DAE70522C4
:10EB00008A55D7E703228A55D4E7BEF1400F18BFD4
:10EB1000002294E70080FF1F7CA1FF1F28A1FF1F98
:10EB200044A3FF1FC80040008800400004A2FF1F4C
:10EB30008DA1FF1F78A2FF1FF0A1FF1F24A1FF1FBF
:10EB40008CA1FF1FC0200740FCA1FF1F38A1FF1FA1
:10EB5000F8A1FF1F982007402109000394200740D7
:10EB6000D0A1FF1F08A2FF1F882007408020074078
:10EB700090200740B0F5106F00F07C8140F2A38038
:10EB800040F62112904240F07B82A54A0123137087
:10EB90006AE74C68A3498C427FF463AF0178A929E6
:10EBA0007FF45FAF417845297FF45BAF8178C2295C
:10EBB0007FF457AFC1786B297FF453AF9A489B4ECF
:10EBC0000178347881F00105002C41F002010570D4
:10EBD0000CBF8820C82084F0010449F8310009EBFB
:10EBE000C10193483470002505244D60047038E756
:10EBF00000F064FF94E68F4B89488B491A614FF00F
:10EC0000020E80F800E08C4F0A708C491960996000
:10EC10008B4E8C4D8C4C9A610D213970FF213170D7
:10EC2000DFF84CE229702270884D894A8EF8001076
:10EC30009F27012406F8047C5D600470DA6007B049
:10EC4000BDE8F08F43F82600824D30E6824A47F84F
:10EC5000380013780133137042E68B5D032B00F20A
:10EC6000BA8001A252F823F0E1E80000E1E80000D8
:10EC7000C1EC0000BBEC00006F49724B80220D20FC
:10EC800008701A70A2077FF52FAF26E740F2023214
:10EC9000904240F0ED81AA8802F07F02042A69D8F0
:10ECA0006D88002D66D16449CDF804E092001144CE
:10ECB0000A7842F002020A70C1E101238B550FE687
:10ECC00000238B550CE6B0F5086F53D16349644AB5
:10ECD000097811707146ED888D4280F0E8825248C3
:10ECE0000478402DAE4644F0020C28BF4FF0400E91
:10ECF00002EB0E0309EBCC01029301234A604FEAB9
:10ED00000E48CEEB050101930025C82242EA080314
:10ED100084F0010249F83C3035700270DFF814C10C
:10ED2000424BDFF8048149BBBEF1400F7FF42DAFA9
:10ED300042F0020C09EBCC03029ADFF8F8E05A60CB
:10ED40008DBB0D0445F088059DF804304EF83C500D
:10ED50000A4433700470134640297FF416AF002133
:10ED6000404A3B60118010E7AA8802F07F02042A23
:10ED700040F28B81304A0F23137006E74029D7D920
:10ED800042F002020CEBC200029E4660BDB19DF84B
:10ED9000045035481D703346403988F800404033F0
:10EDA0004CF83200DCE79DF8043033700D04029B10
:10EDB000047045F0C8050B444EF83C50CCE79DF874
:10EDC00004501D70029B1D4888F8004040394033B4
:10EDD0004CF83200C4E719F0080F0CBF02230323DC
:10EDE0008B557DE521494A68002AC3D06C88B5F867
:10EDF00004E003E00C314A68002ABBD00B88A34230
:10EE0000F8D14B887345F5D1240A032C0CBF117837
:10EE1000098960E7124A0221147054705BE700BF51
:10EE20009420074001000400F8A1FF1F8CA1FF1FE0
:10EE30008DA1FF1F0080FF1FC020074088004000F9
:10EE40008820074080200740982007403CA1FF1FF2
:10EE500090A1FF1F28A1FF1FF9A1FF1F04A2FF1F00
:10EE6000FCA1FF1F38A1FF1FC8004000604C01003B
:10EE70008C200740B248116AAC7804700C0600F18F
:10EE80009881D9F82820AF49100600F1DB81D9F824
:10EE90003020AC49120600F1D081D9F83820A949B8
:10EEA000130600F1C581D9F84020A649150600F1E6
:10EEB000BA81D9F84820A349140600F1AF81D9F8E6
:10EEC0005020A049100600F1A481D9F858209D498E
:10EED000120600F19981D9F860209A49130600F1D1
:10EEE0008E81D9F868209749150600F18381D9F8F9
:10EEF00070209449140600F17881D9F8782091495E
:10EF0000100600F16D81D9F880208E49120600F1BB
:10EF10006181D9F888208B49130600F15581D9F811
:10EF200090208849150600F14981D9F89820854933
:10EF3000140600F1FF808448844A85490190854881
:10EF4000854D864C049700230596029580460F4612
:10EF500016461D460394306828B1446800F04AFA0A
:10EF60002046002CF9D100233360029B38681A46F2
:10EF7000002342F8253028B1446800F03BFA2046CF
:10EF8000002CF9D100223A60019A98F8003011461D
:10EF9000002241F8042B039A0191023B4FF000013B
:10EFA00022F81510032B07D8DFE803F05D025D029D
:10EFB0004FF0010388F800300135042D06F10406F6
:10EFC00007F1040708F10108C5D1654C654D2278A9
:10EFD000654B049F059E0021100729701A7000F1EF
:10EFE0009280624962780A700021C9F83010C9F82D
:10EFF00038101107DFF84C816ED4A2785C49DFF835
:10F0000044810A7000211207C9F85010C9F858103D
:10F010004BD4E27857494B4C0A7013074FF000016C
:10F02000C9F87010C9F8781000F1AE8033780193F8
:10F03000002283F00105C9F89020C9F8982000212A
:10F04000029188468E460A464B48047844F0020CEA
:10F0500009EBCC030393019B002B039B5A600CBF6D
:10F060008822C82252E64FF0000388F80030A3E758
:10F07000B0F5A06F7FF47EAE012300250193DEE79B
:10F0800040F621229042F7D074E66D88002D7FF47F
:10F0900071AE3A49CDF804E0920011440A7822F0AA
:10F0A00002020A70CBE7022115E600F083F900287E
:10F0B00000F0EB800830324AC8F86400C8F86020DD
:10F0C00000F078F9002800F0DA8008302D4AC9F8FD
:10F0D0006C00C9F868209CE700F06CF9002800F08B
:10F0E000E0800830264AC8F84400C8F8402000F004
:10F0F00061F9002800F0CF800830224AC9F84C009E
:10F10000C9F8482079E700F055F9002800F0A580FB
:10F1100008301B4AC9F82400C9F8202000F04AF939
:10F12000002800F094800830164AC9F82C00C9F86D
:10F13000282056E7D1F89C00083800F05BF9FAE681
:10F1400004A2FF1F0080FF1FE0A1FF1F7CA1FF1F83
:10F15000D0A1FF1F08A2FF1F28A1FF1F44A3FF1F6C
:10F160005C4C0100F9A1FF1FC4200740C8200740E4
:10F17000CC200740D0200740F8A1FF1FC020074047
:10F1800088004000C800400000F014F9002870D04A
:10F1900008304F4AC4F88400C4F8802000F00AF90F
:10F1A000002860D008304B4AC9F88C00C9F8882084
:10F1B0003CE7506A083800F01DF962E6D1F8940087
:10F1C000083800F017F9B0E6D1F88C00083800F0E4
:10F1D00011F9A4E6D1F88400083800F00BF998E69C
:10F1E000C86F083800F006F98DE6486F083800F05F
:10F1F00001F982E6C86E083800F0FCF877E6486E40
:10F20000083800F0F7F86CE6C86D083800F0F2F83E
:10F2100061E6486D083800F0EDF856E6C86C08382D
:10F2200000F0E8F84BE6486C083800F0E3F840E6F8
:10F23000C86B083800F0DEF835E6486B083800F097
:10F24000D9F82AE6C86A083800F0D4F81FE62A7808
:10F25000C9F8280001322A70C3E62A78C9F82000CC
:10F2600001322A705AE72A78C9F8880001322A70D8
:10F27000DCE62A78C4F8800001322A708EE72A780A
:10F28000C9F8680001322A70C3E62A78C8F860001D
:10F2900001322A7014E72A78C9F8480001322A702E
:10F2A000ABE62A78C8F8400001322A701FE74029EF
:10F2B0008E4628BF4FF0400E02EB0E03029301234F
:10F2C000CEEB01014FEA0E4800250193BCE600BFDA
:10F2D00088004000C8004000F8B500F0F9FC294B58
:10F2E00029482A4C2A4F2B4DDFF8BCC0DFF8BCE080
:10F2F000294E00221A605A609A60DA601A615A61D7
:10F300009A61DA611A625A629A62DA621A635A631D
:10F310009A63DA631A645A649A64DA641A655A65FD
:10F320009A65DA651A665A669A66DA661A675A67DD
:10F330009A67DA67C3F880200168C3F8842041F433
:10F3400080210160C3F307212170C3F307401349F3
:10F3500038701B0E2B70FF238CF80030104D8EF888
:10F36000003010480B700123337084F8642070263D
:10F370004FF40074102207F82C3C2E70046081F8C2
:10F38000F820F8BD0080FF1F348004409C20074017
:10F39000B0200740B42007409420074010200740C9
:10F3A00049E400E008E100E08020074088200740B1
:10F3B000704700BF72B60D480268B2FA82F30F2B95
:10F3C00010DC4FF00041D94022EA0102026062B62F
:10F3D000074803EBC303DB00C2180021C1501046ED
:10F3E0005160704762B60020704700BF3093FF1F26
:10F3F000BC83FF1F0D4B0E4AC31AA2FB03231B093C
:10F400000F2B0CD80B4A127852B972B60A484FF03B
:10F410000041026821FA03F31A43026062B67047A2
:10F42000064A1278002AF0D0FFF768B9BC83FF1FA4
:10F43000398EE338F9A1FF1F3093FF1F04A2FF1F8D
:10F4400038B50E4B0E4C1B68218805468BB1B1F5C3
:10F45000917F05D20B4A4B1C55549BB2238038BD7B
:10F460000022084898470021064A5554012323806A
:10F4700038BDB1F5917FEDD338BD00BF30A2FF1F7D
:10F480004EA3FF1F54A3FF1F2DE9F843214E224F27
:10F490003168012380463B70B1B1204D4B8801EBB0
:10F4A0008302013300240F2BC2F808802C7004D88B
:10F4B0004B8000233B70BDE8F88340230B80032082
:10F4C000FFF780F93460F4E7DFF8549099F80030E2
:10F4D000002BF0D0114D45F6215408E0013C12D02C
:10F4E0002B7883B900F00AFB99F800307BB1032038
:10F4F000FFF7EEF80528F1D8FFF75CFF0146306012
:10F500000028EBD0CAE701232B70BDE8F883BDE8E3
:10F51000F88300BF4CA2FF1F20A2FF1F50A2FF1FB5
:10F5200004A2FF1F1201F8B5D5B2A1B3012943D03F
:10F530004378044600781B0643EA004040F47040DC
:10F5400045F004068F1E3043FFF79EFF022F04F1A3
:10F55000020314D9053414F8023C14F8032C14F8EF
:10F56000010C1B0443EA0223334343EA0060033FD8
:10F57000FFF78AFF022F234604F10304EBD8022F82
:10F5800023D0012F0DD045F4774040F00500BDE8B1
:10F59000F840FFF779BF14482843BDE8F840FFF76B
:10F5A00073BF187845F4770545F0060545EA002055
:10F5B000BDE8F840FFF768BF03780C4845EA03450B
:10F5C0002843BDE8F840FFF75FBF1A78587845F048
:10F5D000774545F0070545EA022545EA0040BDE8C4
:10F5E000F840FFF751BF00BF06F0F70007F000F743
:10F5F00038B5084B1C7824B9074D296809B14B88E8
:10F6000003B938BD9B000B800320FFF7DBF82C60AB
:10F6100038BD00BF20A2FF1F4CA2FF1F2DE9F04103
:10F62000AD4E33680746002B00F092801D885A8843
:10F63000910803EB81010432AA428C6842D25A80BD
:10F6400004F00F064FEA1428A449A6F1080208F0B6
:10F650000F00C4F30313062A00F101050B701AD939
:10F66000B31E012B5FFA88F04ED9052E48D0042E28
:10F6700000F0A481731F022B7FD90F2E0ED1F72823
:10F6800042D8F02802D0964B1B883BB1FFF7D8FE3A
:10F690000020BDE8F08127B1BD4202D00020BDE8C6
:10F6A000F081082EC4F3033300F08780092E11D0B7
:10F6B0000A2E40F094800A2BF0D18A4B8A4A1B68AC
:10F6C000A02181E01846FFF795FE0420FEF7E2FF37
:10F6D0003060B5E7092BE1D1270E00F07B81834B29
:10F6E000814A1B689021C4F307461170EDB2FCB249
:10F6F000002B00F09D80224631462846984797E02F
:10F70000F02843D9F72841D0F1380E28C6D801A3F4
:10F7100053F820F0CBF80000AFF800009DF800008F
:10F720009DF600009DF600008FF800009DF6000099
:10F730006FF900009DF6000039F9000053F9000050
:10F7400077F800009DF600005FF8000043F8000025
:10F75000674B1B78002BA1D00420FEF79BFF0346CC
:10F76000306000289AD00588002D7FF460AFFFF745
:10F7700041FE35602846BDE8F081FFF761FEC4F325
:10F780000740FFF75DFE072E02D1200EFFF758FE5F
:10F79000534B584A198858481468584D524A0170BA
:10F7A00000270E0AF0201F802E7010700CB301226B
:10F7B0005348A0470120BDE8F081082B7FF46EAFCD
:10F7C000504B494A1B688021C4F307461170EDB2C3
:10F7D000240E6BB3284622463146984728E00B2E6C
:10F7E00011D10B2B7FF45AAF474B3F4A1B68B02116
:10F7F000EAE7464B1B68002B00F0FB804048984727
:10F800000120BDE8F0810C2E40F000810C2B7FF42C
:10F8100045AF3F4B344A1B68C0211170EDB2C4F3B1
:10F820000746002B00F0C88028463146240E984732
:10F830003849314A314B0D7016701C700120BDE8FB
:10F84000F081354B1B68002B00F0D6809847C4F33D
:10F850000746254BEDB2240E83F80080E8E72F4BD6
:10F860001B68002BF2D12E4B1B68A3B1FE209847DA
:10F87000C4F30746EDE72B4B1B68002BE6D1284B62
:10F880001B6843B1FC209847C4F30746E1E7264BC9
:10F890001B68002BDAD1C4F30746DAE7234B1B6859
:10F8A000C4F30746002BD4D030469847D1E7204B0D
:10F8B0001A68002AEFD0260C630C06F07F0003F4D0
:10F8C0007E531843F6B29047C3E71A4B1B68C4F344
:10F8D0000746002BE8D1BCE758A2FF1F52A3FF1F29
:10F8E0004EA3FF1F34A2FF1F4CA3FF1F68A2FF1FE0
:10F8F00004A2FF1F30A2FF1F50A3FF1F51A3FF1F31
:10F9000054A3FF1F60A2FF1F64A2FF1F48A2FF1F96
:10F9100024A2FF1F53A3FF1F10A2FF1F14A2FF1F4B
:10F9200018A2FF1F54A2FF1F44A2FF1F5CA2FF1FCB
:10F930002CA2FF1F40A2FF1F3F4B1B68002B85D14D
:10F940003E4B1B68002BA6D0FA209847C4F307460D
:10F950007FE73B4B1B68002B7FF478AF374B1B686E
:10F96000002B98D0FB209847C4F3074671E7354B2E
:10F970001B68002B7FF46AAF304B1B68002B8AD0CA
:10F98000F8209847C4F3074663E70E2B7FF486AE52
:10F990002D4A2E4B1268E0211970002A47D0260C00
:10F9A000610C06F07F0301F47E511943EDB2A1F51D
:10F9B000005128469047F6B2240E39E7FFF740FD84
:10F9C000C4F30740FFF73CFD200EFFF739FD002090
:10F9D000BDE8F0811E4B1D4A1B6880211170EDB2FD
:10F9E000C4F3074683B1314628463A4698473C4619
:10F9F0001EE70120BDE8F081104B1B68002B3FF48F
:10FA00004AAFFF20984746E71C4611E70D2EBCD1B0
:10FA10000D2B7FF443AE0F4B0C4A1B68D0211170A5
:10FA2000EDB2C4F30746002B7FF4FEAEC4E7C4F387
:10FA30000746EDB2240EFBE63CA2FF1F18A2FF1FF3
:10FA40001CA2FF1F0CA2FF1F28A2FF1F4CA3FF1F19
:10FA500060A2FF1F38A2FF1F38B5164D2868E0B11D
:10FA600001884488A14213DD03191B7A83B104F194
:10FA70000803C2180C1B002302E012F8011F21B179
:10FA80000133A342F9D1204638BD1C46204638BD7B
:10FA9000FFF7B0FC0020286038BD074B1B780BB97E
:10FAA000002038BD0220FEF7F5FD28600028D7D1E0
:10FAB000F6E700BF74A2FF1F04A2FF1F0D4B1B78C7
:10FAC000BBB910B50C4C216803F0FF024B883F2BEB
:10FAD00007DC07330B4401F1470003F8012F834291
:10FAE000FBD140230B800120FEF76CFE0023236036
:10FAF00010BD70476CA2FF1F70A2FF1F38B5224CCB
:10FB0000237803B138BD01232370FFF7A5FF70BB35
:10FB100000F048F840BBFEF7ADFB10BBFEF7F8FC69
:10FB2000E0B900232370EFF30583002BEAD1EFF354
:10FB3000108172B6154B1868E0B1154C2278CAB91D
:10FB400045691D6001232370C5B1AA6101B962B680
:10FB500000254577836898472570D3E700F020F8A3
:10FB6000DFE700F01BF8D9E700F016F8D3E7FFF75E
:10FB70001FFCCDE70029C5D162B638BD054B1D601D
:10FB80000029E5D1E3E700BF79A2FF1F14A0FF1F02
:10FB900018A0FF1F10A0FF1F704700BF704700BFD5
:10FBA000704700BF054A064B10781B78C0B2DBB225
:10FBB000984238BF4030C01A704700BF80A2FF1F74
:10FBC00081A2FF1FF0B4384B1A7912F0300F2CD0FD
:10FBD00072B6997D01F0FF0200293DD062B6334F25
:10FBE000334938780D78334E1C46C0B2EDB2431C11
:10FBF000402BE17928BF0023AB4202F1FF32C9B2AA
:10FC00001CBFF154184612F0FF02F0D12A4B1B68BA
:10FC1000C2B23A704BB1A84236BFC5F14005401B95
:10FC200040192728C4BF01221A701F49CA78D2B2CE
:10FC3000150616D452060DD51B4B1B795B0609D54C
:10FC40001E4B1F491B6800220A7003B11A70164B25
:10FC50003C22DA70F0BC70474022D9795A7462B6FF
:10FC6000E3E70B791C06E5D5164B174E1C78337865
:10FC7000E4B2DBB29C420ED0144D01E0A3420AD0A4
:10FC80000133402B28BF00230879E85CC0B2C8715B
:10FC9000087D0728F2D9DBB2034933700B791806C7
:10FCA00044BF7C23CB70C5E700A0064080A2FF1FA5
:10FCB00081A2FF1FC4A2FF1F7CA2FF1F08A3FF1F7A
:10FCC00004A3FF1F0CA3FF1F05A3FF1F84A2FF1F98
:10FCD00070B584B072B6194B194D1A48702241267E
:10FCE0000F2480211A702E701A4604701970137830
:10FCF0001B06FCD5144B186862B6144B144C984282
:10FD000098BF00EB800001A998BF40000A22FDF7D0
:10FD10008DFD01A92046002311F8012B01333AB1D2
:10FD20000A2B20F8022FF7D11623237004B070BDE0
:10FD30005B00DBB2237004B070BD00BF0000024066
:10FD40000700024006000240080002407F9698002B
:10FD5000FC93FF1FFFFFFFFF2DE9F043DFF8EC806E
:10FD60008BB006460F4600F073F898F90030013367
:10FD700004460D4637D03046394600F0DFF90028FA
:10FD800031D02BA3D3E900233046394600F026FEBC
:10FD9000814668BB28A3D3E900233046394600F0EA
:10FDA000FFFD00B398F90030254ACDF820900424D7
:10FDB00000200021022BCDE90467CDE90267009401
:10FDC0000192CDE906012CD0684600F0BDF940B3A0
:10FDD000089B1BB101F0AAF9089B0360DDE906014D
:10FDE0000BB0BDE8F083204629460BB0BDE8F08398
:10FDF000134A98F90030019203210022CDE90467EB
:10FE0000CDE90267009108922BB90E4B4FF060428A
:10FE1000CDE90623D8E70C490020022BCDE90601E5
:10FE2000D2D101F083F922230360D1E7AFF3008040
:10FE3000EF39FAFE422E864051302DD5104987C049
:10FE4000CC4C0100FFFFEF470000F07F1294FF1F32
:10FE50002DE9F04FB04F21F00042BA4283B00C467A
:10FE60004FEAD17605460DD9AC4FBA4225D9C1F338
:10FE70001303034340F0EF800EB10020014603B0AE
:10FE8000BDE8F08FA64B9A4200F2CC80A54B9A4277
:10FE900000F2DE808AA3D3E9002300F05DF900229E
:10FEA000A14B00F09BFD002800F00581284621466B
:10FEB00000229D4B00F050F9E1E783A3D3E9002332
:10FEC00000F08CFD002840F0CB802846214680A31E
:10FED000D3E9002300F064FD0028CED1934B2846DF
:10FEE00003EBC60821467CA3D3E9002300F0E6FA21
:10FEF000D8E9002300F030F900F07AFD804600F0E8
:10FF000077FA77A3D3E9002306460F4600F0D6FA26
:10FF100002460B462846214600F01CF972A3D3E99D
:10FF20000023CDE900013046394600F0C7FA824689
:10FF30008B4652465B46DDE9000100F00BF90546B1
:10FF40000C462A4623462846214600F0B7FA68A305
:10FF5000D3E9002306460F4600F0B0FA66A3D3E9C2
:10FF6000002300F0F7F832463B4600F0A7FA64A3FE
:10FF7000D3E9002300F0F0F832463B4600F09EFA49
:10FF800061A3D3E9002300F0E5F832463B4600F0D8
:10FF900095FA5FA3D3E9002300F0DEF832463B4632
:10FFA00000F08CFA02460B462846214600F0D2F8B3
:10FFB00006460F462846214632463B46B8F1000F1A
:10FFC00056D000F07BFA324604460D463B460020F0
:10FFD0004FF0804100F0BEF802460B46204629460D
:10FFE00000F096FB02460B465046594600F0B2F828
:10FFF000DDE9002300F0AEF80B4602464A49002036
:020000021000EC
:1000000000F0A8F86FF47F7398454FDA08F57A7816
:1000100001EB085100224FF0B87300F04FFA03B023
:10002000BDE8F08F424B9A423FF658AF414BF40087
:100030002344D3E9002300F08DF83F4BC6F10108BB
:100040001C44CDE90001D4E900ABC6EB080870E719
:100050004FF0000875E702460B4600F07DF80EE70A
:1000600017A3D3E900231046194600F027FA06E744
:1000700000F024FA0022804689464FF08043304643
:10008000394600F067F802460B464046494600F004
:100090003FFB2A46234600F05DF802460B4600204F
:1000A000214900F057F803B0BDE8F08F01EB08518B
:1000B00003B0BDE8F08F804643E700BFAFF3008098
:1000C0009C7500883CE4377EEF39FAFE422E86406C
:1000D00051302DD5104987C0FE822B654715F73F5B
:1000E0000000E0FE422EE63F763C7935EF39EA3DEE
:1000F000D0A4BE726937663EF16BD2C541BDBB3E2E
:100100002CDE25AF6A56113F93BDBE166CC1663F0B
:100110003E5555555555C53F412E8640FFFFEF7F53
:10012000422ED63FFFFF2F3E0000F03FD04C010093
:10013000B1A2F03FF04C0100E04C010041F0004161
:1001400001F58010C00F70470020704781F000411A
:1001500002E000BF83F0004330B54FEA41044FEAAC
:10016000430594EA050F08BF90EA020F1FBF54EA47
:10017000000C55EA020C7FEA645C7FEA655C00F0E3
:10018000E2804FEA5454D4EB5555B8BF6D420CDDB4
:100190002C4480EA020281EA030382EA000083EA37
:1001A000010180EA020281EA0303362D88BF30BDD7
:1001B00011F0004F4FEA01314FF4801C4CEA11312D
:1001C00002D0404261EB410113F0004F4FEA03338C
:1001D0004CEA133302D0524263EB430394EA050F17
:1001E00000F0A780A4F10104D5F1200E0DDB02FA86
:1001F0000EFC22FA05F2801841F1000103FA0EF21A
:10020000801843FA05F359410EE0A5F120050EF1DF
:10021000200E012A03FA0EFC28BF4CF0020C43FA10
:1002200005F3C01851EBE37101F0004507D54FF01D
:10023000000EDCF1000C7EEB00006EEB0101B1F56D
:10024000801F1BD3B1F5001F0CD349085FEA3000B3
:100250004FEA3C0C04F101044FEA445212F5800FBE
:1002600080F09A80BCF1004F08BF5FEA500C50F15B
:10027000000041EB045141EA050130BD5FEA4C0C3E
:10028000404141EB010111F4801FA4F10104E9D1C7
:1002900091F0000F04BF01460020B1FA81F308BFBE
:1002A0002033A3F10B03B3F120020CDA0C3208DD8A
:1002B00002F1140CC2F10C0201FA0CF021FA02F165
:1002C0000CE002F11402D8BFC2F1200C01FA02F1D5
:1002D00020FA0CFCDCBF41EA0C019040E41AA2BFFA
:1002E00001EB0451294330BD6FEA04041F3C1CDAC2
:1002F0000C340EDC04F11404C4F1200220FA04F0E2
:1003000001FA02F340EA030021FA04F345EA03018B
:1003100030BDC4F10C04C4F1200220FA02F001FA4D
:1003200004F340EA0300294630BD21FA04F02946CF
:1003300030BD94F0000F83F4801306BF81F4801168
:100340000134013D4EE77FEA645C18BF7FEA655CDB
:1003500029D094EA050F08BF90EA020F05D054EAAD
:10036000000C04BF1946104630BD91EA030F1EBFB2
:100370000021002030BD5FEA545C05D140004941B6
:1003800028BF41F0004130BD14F580043CBF01F5A9
:10039000801130BD01F0004545F0FE4141F470018F
:1003A0004FF0000030BD7FEA645C1ABF194610466A
:1003B0007FEA655C1CBF0B46024650EA013406BF6B
:1003C00052EA033591EA030F41F4002130BD00BF2A
:1003D00090F0000F04BF0021704730B54FF48064E7
:1003E00004F132044FF000054FF0000150E700BF68
:1003F00090F0000F04BF0021704730B54FF48064C7
:1004000004F1320410F0004548BF40424FF00001B3
:100410003EE700BF42004FEAE2014FEA31014FEAF6
:1004200002701FBF12F07F4393F07F4F81F0605145
:10043000704792F0000F14BF93F07F4F704730B5B4
:100440004FF4607401F0004521F0004120E700BF47
:1004500050EA010208BF704730B54FF000050AE0CE
:1004600050EA010208BF704730B511F0004502D5CF
:10047000404261EB41014FF4806404F132045FEAD1
:10048000915C3FF4DCAE4FF003025FEADC0C18BF76
:1004900003325FEADC0C18BF033202EBDC02C2F16C
:1004A000200300FA03FC20FA02F001FA03FE40EAFE
:1004B0000E0021FA02F11444C1E600BF70B54FF0FE
:1004C000FF0C4CF4E06C1CEA11541DBF1CEA1355E0
:1004D00094EA0C0F95EA0C0F00F0DEF82C4481EA48
:1004E000030621EA4C5123EA4C5350EA013518BF68
:1004F00052EA033541F4801143F4801338D0A0FB55
:1005000002CE4FF00005E1FB02E506F00042E0FB01
:1005100003E54FF00006E1FB03569CF0000F18BF07
:100520004EF0010EA4F1FF04B6F5007F64F54074AF
:1005300004D25FEA4E0E6D4146EB060642EAC62142
:1005400041EA55514FEAC52040EA5E504FEACE2EAF
:10055000B4F1FD0C88BFBCF5E06F1ED8BEF1004FB2
:1005600008BF5FEA500E50F1000041EB045170BD2E
:1005700006F0004646EA010140EA020081EA030172
:10058000B4EB5C04C2BFD4EB0C0541EA045170BD6E
:1005900041F480114FF0000E013C00F3AB8014F1E8
:1005A000360FDEBF002001F0004170BDC4F1000431
:1005B000203C35DA0C341BDC04F11404C4F12005B2
:1005C00000FA05F320FA04F001FA05F240EA02000D
:1005D00001F0004221F0004110EBD37021FA04F643
:1005E00042EB06015EEA430E08BF20EAD37070BDFD
:1005F000C4F10C04C4F1200500FA04F320FA05F05C
:1006000001FA04F240EA020001F0004110EBD3705D
:1006100041F100015EEA430E08BF20EAD37070BDCD
:10062000C4F1200500FA05F24EEA020E20FA04F3A6
:1006300001FA05F243EA020321FA04F001F0004155
:1006400021FA04F220EA020000EBD3705EEA430EC6
:1006500008BF20EAD37070BD94F0000F0FD101F0F5
:100660000046400041EB010111F4801F08BF013C2E
:10067000F7D041EA060195F0000F18BF704703F06C
:100680000046520043EB030313F4801F08BF013DF3
:10069000F7D043EA0603704794EA0C0F0CEA1355AF
:1006A00018BF95EA0C0F0CD050EA410618BF52EA69
:1006B0004306D1D181EA030101F000414FF000006F
:1006C00070BD50EA410606BF1046194652EA43067D
:1006D00019D094EA0C0F02D150EA013613D195EAF1
:1006E0000C0F05D152EA03361CBF104619460AD139
:1006F00081EA030101F0004141F0FE4141F4700143
:100700004FF0000070BD41F0FE4141F4780170BD32
:1007100070B54FF0FF0C4CF4E06C1CEA11541DBF97
:100720001CEA135594EA0C0F95EA0C0F00F0A7F899
:10073000A4EB050481EA030E52EA03354FEA0131C6
:1007400000F088804FEA03334FF0805545EA1313D9
:1007500043EA12634FEA022245EA111545EA1065A1
:100760004FEA00260EF000419D4208BF964244F138
:10077000FD0404F5407402D25B084FEA3202B61A57
:1007800065EB03055B084FEA32024FF480104FF42B
:10079000002CB6EB020E75EB030E22BFB61A75469F
:1007A00040EA0C005B084FEA3202B6EB020E75EB32
:1007B000030E22BFB61A754640EA5C005B084FEA9A
:1007C0003202B6EB020E75EB030E22BFB61A754667
:1007D00040EA9C005B084FEA3202B6EB020E75EB72
:1007E000030E22BFB61A754640EADC0055EA060E33
:1007F00018D04FEA051545EA16754FEA06164FEA76
:10080000C30343EA52734FEAC2025FEA1C1CC0D121
:1008100011F4801F0BD141EA00014FF000004FF0AE
:10082000004CB6E711F4801F04BF01430020B4F16F
:10083000FD0C88BFBCF5E06F3FF6AFAEB5EB030C27
:1008400004BFB6EB020C5FEA500C50F1000041EB24
:10085000045170BD0EF0004E4EEA113114EB5C04F1
:10086000C2BFD4EB0C0541EA045170BD41F48011C4
:100870004FF0000E013C90E645EA060E8DE60CEACC
:10088000135594EA0C0F08BF95EA0C0F3FF43BAFE9
:1008900094EA0C0F0AD150EA01347FF434AF95EAA0
:1008A0000C0F7FF425AF104619462CE795EA0C0F84
:1008B00006D152EA03353FF4FDAE1046194622E751
:1008C00050EA410618BF52EA43067FF4C5AE50EA2B
:1008D00041047FF40DAF52EA43057FF4EBAE12E71B
:1008E0004FF0FF3C06E000BF4FF0010C02E000BFFC
:1008F0004FF0010C4DF804CD4FEA410C7FEA6C5CDF
:100900004FEA430C18BF7FEA6C5C1BD001B050EA81
:10091000410C0CBF52EA430C91EA030F02BF90EA6C
:10092000020F0020704710F1000F91EA030F58BF2B
:10093000994208BF90422CBFD8176FEAE37040F08D
:10094000010070474FEA410C7FEA6C5C02D150EA2B
:10095000013C07D14FEA430C7FEA6C5CD6D152EAE6
:10096000033CD3D05DF8040B704700BF84461046AB
:1009700062468C461946634600E000BF01B5FFF7AA
:10098000B7FF002848BF10F1000F01BD4DF808ED7A
:10099000FFF7F4FF0CBF012000205DF808FB00BF4B
:1009A0004DF808EDFFF7EAFF34BF012000205DF8A5
:1009B00008FB00BF4DF808EDFFF7E0FF94BF0120F2
:1009C00000205DF808FB00BF4DF808EDFFF7CEFFF3
:1009D00094BF012000205DF808FB00BF4DF808ED32
:1009E000FFF7C4FF34BF012000205DF808FB00BF03
:1009F0004FEA410212F5001215D211D56FF4787347
:100A0000B3EB625212D94FEAC12343F0004343EAE9
:100A1000505311F0004F23FA02F018BF40427047C4
:100A20004FF00000704750EA013005D111F000404E
:100A300008BF6FF0004070474FF00000704700BFE4
:100A40004FEA4102B2F1E04324BFB3F5001CDCF1F0
:100A5000FE5C0DD901F0004C4FEAC0024CEA507028
:100A6000B2F1004F40EB830008BF20F00100704757
:100A700011F0804F21D113F13872BCBF01F000405A
:100A8000704741F480114FEA5252C2F11802C2F18C
:100A9000200C10FA0CF320FA02F018BF40F001000D
:100AA0004FEAC1234FEAD32303FA0CFC40EA0C00BF
:100AB00023FA02F34FEA4303CCE77FEA625307D1FC
:100AC00050EA01331EBF4FF0FE4040F44000704733
:100AD00001F0004040F0FE4040F40000704700BFCD
:100AE00080F0004002E000BF81F0004142001FBFE3
:100AF0005FEA410392EA030F7FEA226C7FEA236CEC
:100B00006AD04FEA1262D2EB1363C1BFD2184140E0
:100B100048404140B8BF5B42192B88BF704710F076
:100B2000004F40F4000020F07F4018BF404211F019
:100B3000004F41F4000121F07F4118BF494292EA81
:100B4000030F3FD0A2F1010241FA03FC10EB0C00AD
:100B5000C3F1200301FA03F100F0004302D549423A
:100B600060EB4000B0F5000F13D3B0F1807F06D3E7
:100B700040084FEA310102F10102FE2A51D2B1F1DF
:100B8000004F40EBC25008BF20F0010040EA0300D4
:100B90007047490040EB000010F4000FA2F1010281
:100BA000EDD1B0FA80FCACF1080CB2EB0C0200FA0B
:100BB0000CF0AABF00EBC25052421843BCBFD04059
:100BC0001843704792F0000F81F4000106BF80F4D3
:100BD00000000132013BB5E74FEA41037FEA226C96
:100BE00018BF7FEA236C21D092EA030F04D092F061
:100BF000000F08BF0846704790EA010F1CBF002095
:100C0000704712F07F4F04D1400028BF40F00040F1
:100C1000704712F100723CBF00F50000704700F011
:100C2000004343F0FE4040F4000070477FEA226238
:100C300016BF08467FEA23630146420206BF5FEA09
:100C4000412390EA010F40F4800070474FF0000309
:100C500004E000BF10F0004348BF40425FEA000CD0
:100C600008BF704743F0964301464FF000001CE078
:100C700050EA010208BF70474FF000030AE000BFCE
:100C800050EA010208BF704711F0004302D540420C
:100C900061EB41015FEA010C02BF8446014600207E
:100CA00043F0B64308BFA3F18053A3F50003BCFA99
:100CB0008CF2083AA3EBC25310DB01FA02FC634446
:100CC00000FA02FCC2F12002BCF1004F20FA02F24D
:100CD00043EB020008BF20F00100704702F1200240
:100CE00001FA02FCC2F1200250EA4C0021FA02F2A1
:100CF00043EB020008BF20EADC7070474FF0FF0CA6
:100D00001CEAD0521EBF1CEAD15392EA0C0F93EAA0
:100D10000C0F6FD01A4480EA010C400218BF5FEA42
:100D200041211ED04FF0006343EA501043EA5111B5
:100D3000A0FB01310CF00040B1F5000F3EBF4900AF
:100D400041EAD3715B0040EA010062F17F02FD2AB3
:100D50001DD8B3F1004F40EBC25008BF20F0010096
:100D6000704790F0000F0CF0004C08BF49024CEAAD
:100D7000502040EA51207F3AC2BFD2F1FF0340EA3F
:100D8000C250704740F400004FF00003013A5DDCB0
:100D900012F1190FDCBF00F000407047C2F10002F1
:100DA000410021FA02F1C2F1200200FA02FC5FEADE
:100DB000310040F1000053EA4C0308BF20EADC7028
:100DC000704792F0000F00F0004C02BF400010F49A
:100DD000000F013AF9D040EA0C0093F0000F01F047
:100DE000004C02BF490011F4000F013BF9D041EA69
:100DF0000C018FE70CEAD15392EA0C0F18BF93EA6B
:100E00000C0F0AD030F0004C18BF31F0004CD8D194
:100E100080EA010000F00040704790F0000F17BF1B
:100E200090F0004F084691F0000F91F0004F14D061
:100E300092EA0C0F01D142020FD193EA0C0F03D1B9
:100E40004B0218BF084608D180EA010000F00040BC
:100E500040F0FE4040F40000704740F0FE4040F497
:100E6000400070474FF0FF0C1CEAD0521EBF1CEA36
:100E7000D15392EA0C0F93EA0C0F69D0A2EB030254
:100E800080EA010C49024FEA402037D04FF08053EE
:100E900043EA111143EA10130CF000408B4238BFB3
:100EA0005B0042F17D024FF4000C8B4224BF5B1AC1
:100EB00040EA0C00B3EB510F24BFA3EB510340EA0F
:100EC0005C00B3EB910F24BFA3EB910340EA9C00BD
:100ED000B3EBD10F24BFA3EBD10340EADC001B012D
:100EE00018BF5FEA1C1CE0D1FD2A3FF650AF8B42D1
:100EF00040EBC25008BF20F0010070470CF0004CDE
:100F00004CEA50207F32C2BFD2F1FF0340EAC25008
:100F1000704740F400004FF00003013A37E792F0C9
:100F2000000F00F0004C02BF400010F4000F013A27
:100F3000F9D040EA0C0093F0000F01F0004C02BF22
:100F4000490011F4000F013BF9D041EA0C0195E78B
:100F50000CEAD15392EA0C0F08D142027FF47DAF24
:100F600093EA0C0F7FF470AF084676E793EA0C0F14
:100F700004D14B023FF44CAF08466EE730F0004C12
:100F800018BF31F0004CCAD130F000427FF45CAFA2
:100F900031F000437FF43CAF5FE700BF4FF0FF3C10
:100FA00006E000BF4FF0010C02E000BF4FF0010C63
:100FB0004DF804CD4FEA40024FEA41037FEA226C2C
:100FC00018BF7FEA236C11D001B052EA530C18BF4E
:100FD00090EA010F58BFB2EB030088BFC81738BFB3
:100FE0006FEAE17018BF40F0010070477FEA226CA1
:100FF00002D15FEA402C05D17FEA236CE4D15FEA9D
:10100000412CE1D05DF8040B704700BF84460846D0
:101010006146FFE70FB5FFF7C9FF002848BF10F191
:10102000000F0FBD4DF808EDFFF7F4FF0CBF0120D6
:1010300000205DF808FB00BF4DF808EDFFF7EAFF60
:1010400034BF012000205DF808FB00BF4DF808ED1B
:10105000FFF7E0FF94BF012000205DF808FB00BF10
:101060004DF808EDFFF7D2FF94BF012000205DF896
:1010700008FB00BF4DF808EDFFF7C8FF34BF0120A3
:1010800000205DF808FB00BF4FEA4002B2F1FE4FBE
:101090000FD34FF09E03B3EB12620DD94FEA00233A
:1010A00043F0004310F0004F23FA02F018BF404213
:1010B00070474FF00000704712F1610F01D14202FA
:1010C00005D110F0004008BF6FF0004070474FF0AE
:1010D0000000704742000ED2B2F1FE4F0BD34FF02A
:1010E0009E03B3EB126209D44FEA002343F000439E
:1010F00023FA02F070474FF00000704712F1610FC1
:1011000001D1420202D14FF0FF3070474FF0000092
:10111000704700BF0B460146184600F001B800BFFB
:1011200013460A460146022000F0BCBE014B186877
:10113000704700BF4098FF1F70B50F4E0F4D761BD4
:10114000B61018BF002405D0013455F8043B984769
:10115000A642F9D10A4E0B4D761B03F0D3FDB61013
:1011600018BF002406D0013455F8043B9847A64226
:10117000F9D170BD70BD00BF104D0100104D0100D0
:10118000244D0100104D0100024B0146186800F08B
:101190000BB800BF4098FF1F024B0146186800F0D3
:1011A00045BF00BF4098FF1F2DE9F04F01F10B052F
:1011B000162D83B0064640F29F8035F0070500F1FA
:1011C000BF80A94200F2BC8000F058FBB5F5FC7F5F
:1011D000C0F09C826B0A00F0BA80042B00F283817D
:1011E000A80900F1390E4FEA4E033830C44F07EB1F
:1011F0008303A3F108015C68A14207D1ACE0002A97
:1012000080F2AC80E468A14200F0A680636823F01D
:1012100003035A1B0F2AF2DDB9493C6901F1080E9C
:10122000744500F0B381636823F003035A1B0F2A4F
:1012300000F39981002AC1F814E0C1F810E080F2AF
:101240009E80B3F5007F80F06781DB0803F1010C1D
:1012500001229B1002FA03F34A6851F83C80C4F85B
:10126000088001EBCC091A43A9F10803E3604A6046
:1012700041F83C40C8F80C40831001249C40944243
:1012800000F28A80144206D120F003006400144268
:1012900000F10400FAD007EBC009CC468046DCF828
:1012A0000C108C4507D173E1002A80F28181C96856
:1012B0008C4500F06D814B6823F003035A1B0F2A05
:1012C000F2DD0C46D1F80CC054F8088F4B1945F0EC
:1012D00001054D6042F00101C8F80CC03046CCF861
:1012E00008807B613B61C3F80CE0C3F808E05960FB
:1012F0009A5000F0C5FA1FE0102921D800F0BEFA7C
:101300001025062302207E4F07EB8303A3F108027A
:101310005C68944200F045816368E168A56823F049
:101320000303234430465A68E96042F001028D60AD
:101330005A6000F0A5FA0834204603B0BDE8F08FEB
:1013400000240C232046336003B0BDE8F08F8023D7
:101350004FF0400E3F2049E770465DE72344E168C7
:101360005A68A56842F00102E96030468D605A6013
:1013700000F086FA0834204603B0BDE8F08F23441D
:1013800030465A6842F001025A6000F079FA083497
:10139000204603B0BDE8F08FBC68636823F0030803
:1013A000A84504D3C5EB08030F2B00F38C80554BE5
:1013B000DFF860911A68D9F8003001332A4404EB51
:1013C000080A00F0608102F580520F3222F47F6239
:1013D00022F00F0211463046019200F04BFCB0F1B2
:1013E000FF3F8346019A00F05881824500F2FC805D
:1013F000454B1968DA451144196000F05381D9F85A
:101400000000DFF810E101301BBFCAEB0B0A5144AA
:10141000CEF800B019601BF0070100F01781C1F190
:101420000800C1F58051834408315A44C2F30B02CD
:10143000C2EB010949463046019300F01BFC431CF6
:10144000019B00F03F81CBEB00024A4442F00102D5
:101450001968C7F808B04944BC42CBF804201960A9
:10146000DFF8A49016D0B8F10F0F40F2FD8062684B
:10147000A8F10C0323F00703E01802F001024FF07B
:10148000050E1A430F2B6260C0F804E0C0F808E0B4
:1014900000F21C811D4BBC681A68914288BF19601C
:1014A0001B4B1A689142626888BF196022F00302E0
:1014B0009542A2EB050301D80F2B04DC304600F067
:1014C000DFF9002438E7621943F0010345F0010514
:1014D00065603046BA60536000F0D2F908342046A7
:1014E00003B0BDE8F08F142B71D9542B00F2A48007
:1014F000280B00F16F0E4FEA4E036E3076E600BF08
:101500004498FF1F18A3FF1F1CA3FF1F14A3FF1F56
:1015100010A3FF1F509CFF1F5A0A042A5ED9142AE9
:1015200000F2B38002F15C0149005B3207EB810CF1
:1015300057F82110DFF8DC81ACF1080C8C4500F085
:1015400088804A6822F00302934202D289688C455F
:10155000F7D1D1F80CC07A68C4F80CC0A160CCF8FF
:101560000840CC6088E6631942F0010745F00105A8
:10157000656030464B610B61C3F80CE0C3F808E0CE
:101580005F609A50083400F07BF9D5E64A6873E64C
:1015900008F1010818F0030F0CF1080C7FF47FAE7E
:1015A00030E0DC68A34208BF02303FF435AEB3E65A
:1015B0000B440C465A68C96854F8085F42F00102AF
:1015C0005A603046E9608D6000F05AF9B4E603F1E4
:1015D0005C0E03F15B004FEA4E0307E69A0902F145
:1015E000390149003832A1E7BC424A4B3FF400AF11
:1015F0009C68626822F003025AE759F80839994555
:1016000040F0828010F0030F00F1FF30F5D17B68CD
:1016100023EA04037B6064009C423FF6BDAE002CCD
:101620003FF4BAAE1C4240467FF435AE64001C4223
:1016300000F10400FAD02EE6B3F5AA7F18D8E80B23
:1016400000F1780E4FEA4E037730CFE54FF480512A
:10165000EBE60121D8F80430921001FA02F21A43A5
:10166000C8F80420614677E70123CBF8043025E76A
:1016700040F25452934220D8A80C00F17D0E4FEA5C
:101680004E037C30B2E51032A4E6542A26D81A0B59
:1016900002F16F0149006E3248E7BC68626822F0CF
:1016A000030205E7CAF30B0000287FF4A8AE42440A
:1016B000BB6842F001025A60ECE6FE234FF07F0E59
:1016C0007E2093E501224FF00009C1E604F10801F4
:1016D000304600F0ABFCD9F80010DBE6B2F5AA7F8B
:1016E00005D8DA0B02F17801490077321EE740F2A3
:1016F00054518A4205D89A0C02F17D0149007C328E
:1017000014E7FE217E2211E77B6884E7E808431C8A
:101710005B00F8E54498FF1F8842F0B50DD98B189F
:1017200098420AD28118002A51D09A1A13F8014D12
:1017300001F8014D9342F9D1F0BD0F2A48D941EA91
:1017400000039B0746D100F1100401F11003154678
:1017500053F8106C44F8106C53F80C6C44F80C6C93
:1017600053F8086C44F8086C103D53F8046C44F8C6
:10177000046C0F2D03F1100304F11004E8D8A2F15A
:10178000100323F00F0302F00F0E1033BEF1030F0E
:101790001944034421D91E1F0D467446043C55F8D4
:1017A000047B46F8047F032CF8D8AEF1040424F03F
:1017B000030404342344214402F0030262B1013BD8
:1017C0000A4411F8014B03F8014F8A42F9D1F0BDE8
:1017D0000346F3E70346F2E7F0BD7246EEE700BFCB
:1017E00070B4840746D0541E002A41D0CDB20346BF
:1017F00002E0621EE4B3144603F8015B9A07F8D1D5
:10180000032C2ED9CDB245EA05250F2C45EA054516
:1018100019D903F110022646103E0F2E42F8105C33
:1018200042F80C5C42F8085C42F8045C02F11002D9
:10183000F2D8A4F1100222F00F0204F00F041032CB
:10184000032C13440DD91E462246043A032A46F8B7
:10185000045BFAD8221F22F003020432134404F07E
:1018600003042CB1C9B21C4403F8011BA342FBD1F1
:1018700070BC704714460346C2E700BF704700BF04
:10188000704700BF024B0A460146186800F002B8D4
:101890004098FF1F2DE9F04F174683B0002900F054
:1018A000C1800E46814607F10B05FFF7E7FF56F8AA
:1018B00004EC162D2EF00304A6F1080840D81022DF
:1018C0001546AF4241D8944275DAC94B996808EB86
:1018D00004008842416800F0D98021F001030344EC
:1018E0005B68DB077DD51EF0010F35D039464846D1
:1018F000FFF75AFC0746E0B156F8043C23F0010319
:101900004344A0F108029A4200F04481221F242A95
:1019100000F23181132A00F2048103463246116835
:1019200019605168596092689A603146484600F0E3
:101930007DFB4846FFF7A4FF384603B0BDE8F08FB3
:1019400025F00705002D2A46BBDA0C230020C9F834
:10195000003003B0BDE8F08F56F8083CC3EB080A2E
:10196000DAF8043023F0030C04EB0C039342BDDBE4
:101970005746DAF80C1057F8080F221F242AC160C6
:10198000886000F21781132A40F212813168CAF888
:1019900008107168CAF80C101B2A00F22B81083657
:1019A0000AF110023168116071685160B16891608C
:1019B0003E461C46D046631B0F2B1DD8D8F804307A
:1019C00003F0010323434444C8F80430636843F040
:1019D000010363604846FFF753FF304603B0BDE89C
:1019E000F08F21F003012144914221DBC36882681A
:1019F0000C46D3609A60DEE7D8F8042008EB0501B6
:101A000002F00102154343F001020B44C8F80450F0
:101A10004A605A6842F0010208315A60484600F0B4
:101A200005FBD7E7114603B0BDE8F04FFFF7BCBB9D
:101A30001EF0010F7FF45AAF56F8083CC3EB080ABA
:101A4000DAF8043023F0030C01EB0C0E96458BDB27
:101A5000C36882685746D3609A6057F8081FDAF85F
:101A60000C30CB60221F242A996000F29980132A3F
:101A700062D93368CAF808307368CAF80C301B2A78
:101A800000F2A08008360AF1100356E021F0030BA3
:101A9000A34405F11000834559DA1EF0010F7FF4CD
:101AA00025AF56F8081CC1EB080ADAF8041021F03B
:101AB000030CE34458453FF757AF5746DAF80C108C
:101AC00057F8080F221F242AC160886000F2B480F2
:101AD000132A40F2A5803168CAF808107168CAF864
:101AE0000C101B2A00F2AF8008360AF11002316890
:101AF000116071685160B16891600AEB0501C5EB36
:101B00000B0242F0010299604A60DAF8043003F0F7
:101B100001031D434846CAF80450FFF7B1FE38469A
:101B20005CE733680360736843601B2A27D800F1C1
:101B3000080306F10802F2E63B4632681A60726852
:101B40005A60B2689A603E467446D04633E708EB66
:101B50000501C5EB0B0B4BF0010299604A6056F88A
:101B6000043C03F001031D43484646F8045CFFF7BC
:101B700087FE304632E73146FFF7CEFDD5E6B36843
:101B80008360F368C360242A28D000F1100306F1B3
:101B90001002C4E650F8043C23F003031C440AE797
:101BA000314638467446D046FFF7B6FD3E4602E75A
:101BB0003A46F7E6314638461C46D046FFF7ACFDBC
:101BC0003E46F8E6B368CAF81030F368CAF8143035
:101BD000242A1BD010360AF11803AEE733690361DB
:101BE0007369436106F1180200F1180397E600BF1C
:101BF0004498FF1FB168CAF81010F168CAF81410B1
:101C0000242A0FD010360AF11802CBE63369CAF83D
